:020000040000FA
:0400000053EF00F0CA
:020006000102F5
:0400080006EF04F00B
:080018007F6603EF04F0F0A085
:100020002DD0F09080A80DD083CFDEFF80A603D026
:100030007E82800E29D88A8681A2FED795688A960C
:10004000110080500F0B04E1010E8C6E956AF3D7FE
:10005000080A04E1020E8C6E956AEDD70C0A04E1E1
:100060007DC08CFF956AE7D7080A04E17CC08CFF4D
:10007000956AE1D74F0E8C6E956ADDD7F2A403D056
:10008000F2947B667B061100C96EC7A0FED78B80F9
:10009000C9508B901200DF38DEBC8F0FDF24DEBC2E
:1000A000F90FCD0F12007F6A7E6A8EEC01F0FE0E12
:1000B000F66EFF0EF76EF86A0900F5507D627E8CD1
:1000C0000900F5507C627E8C7EBC26D0030EAA6EA1
:1000D000FE0EA96EA69EA69CA680A8507D627E8E6E
:1000E000A92AA69EA69CA680A8507C627E8E7EBE73
:1000F00013D07F6800EF04F0030EAA6EFE0EA96E07
:100100007DC0A8FF040EA66EC3D8A92A7CC0A8FF94
:10011000040EA66EBDD8FF0094900F0EC16E8A9695
:100120009396F086F09CF19A8A9E939E8A9C939C6B
:100130009496949A400EC76E210EC66E870ED56EA9
:10014000F194F28A120E7B6ED08E8A8E8A8C856B29
:10015000846B21EE00F0F28CF28E400E95DF7EB2C1
:1001600005D87EBCFCD77B66FAD7C6D77E9221EE37
:1001700000F0DE503A0A37E18EDF806F040F816FA6
:100180008ADF8027812FFCD7806726D021EE01F0FF
:1001900082DF816F80DF836F7EDF826F7CDF866F1F
:1001A000070B88EC01F0F5EF00F064EF01F0EAEFE7
:1001B00000F0EAEF00F05BEF01F0EAEF00F066EF2D
:1001C00001F0EAEF00F040095FDF21EE00F01200DD
:1001D000000EF9D7020EF7D7030EF5D77E84050E71
:1001E000F2D7010EF0D7040EEED77EB4F3D78551C7
:1001F000F1E1845105E033D88451F00A18E0EAD7E0
:100200008251F65C876F8351F75808E38713E6E164
:1002100042DF8107F56E7E8649D801D0F5680D0072
:10022000F6503F0BD8B424D88167EAD7D1D7A6B20D
:10023000FED78451F008876F8351FC0B871185111D
:10024000D0E18351AA6E8251A96E25DF8107A86E85
:10025000040EA66E1DD82AD88167E9D7B9D77EA625
:100260001200F5680D00F6503F0BFCE101D81200BA
:100270007EA60CD07E960A00FF0EF65C070EF7589D
:1002800004E37E8C840EA66E03D80900A66A1200D1
:10029000F29EF29C550EA76EAA0EA76EA682F28C55
:1002A000F28E0000A6B2FED7A6941200E86A822B56
:1002B0008323842312008105E82C95D7ECDE856F1B
:1002C000EADE846F000E7FD7CADFFF0083298BE14F
:1002D000825101E00FD07E8C000EF66E080EF76E94
:1002E000F86A940EA66ED4DF400EF626E86AF7226E
:1002F000F8E16ED7A868AA6AA96A040EA66EC8DFDC
:10030000A6B2FED7A93EF9D7AA2AAA50F6E160D72D
:10031000E844E844FD26000EFE221200000EF66EB0
:10032000080EF76EF86A7C6A7D6A0900F55007D8F6
:10033000F750FF08FAE1F650FE08F7E112007C18CA
:100340007D187D1A7D187C6E7D507D3A7D1A7D3238
:100350007DB0D8707DB2D8707DB4D8707D6E010E3E
:10036000D8B07C1A400E7D32D8B07C1A7D347D1A0C
:0A0370007D32800ED8B07C1A000C1C
:06080000BEEF70F01200D3
:060806009CEF6CF01200F3
:04080C00F0900366FF
:100810005DD080501F0B186205D08338070B0F6E18
:10082000106A1F0F62EC04F06BEF04F071EF04F03C
:10083000A8EF04F09CEF04F081EF04F099EF04F0CE
:10084000B8EF04F0A2EF04F06EEF04F090EF04F0C4
:1008500093EF04F09FEF04F08DEF04F096EF04F0B7
:10086000B8EF04F001EF05F001EF05F0C9EF04F077
:1008700055EF05F018EF05F0E3EF04F012EF05F087
:1008800064EF05F01FEF05F0B9EF04F001EF05F09C
:1008900060EF05F01BEF05F02AEF05F015EF05F00E
:1008A00064EF05F001EF05F030EF05F036EF05F0ED
:1008B0003DEF05F04AEF05F051EF05F051EF05F07F
:1008C0004AEF05F0E844E844FD26120080B899D0CC
:1008D00004C08CFF95D00EC08CFF92D006C08CFF58
:1008E0008FD0E9CF49F0EACF4AF009EE00F010C00E
:1008F000E9FFEFCF8CFF103E7FD0500EC96E046E23
:1009000076D0E9CF49F0EACF4AF00AEE00F015C000
:10091000E9FF152AEFCF8CFF6FD013C08CFF70D08A
:1009200007C08CFF6DD012C08CFF6AD009C08CFF4D
:1009300067D008C08CFF64D00AC08CFF61D00BC0A8
:100940008CFF5ED00C44E844E8440D108C6E58D007
:10095000020E166203D017C08CFF08D016C0A9FF84
:10096000AA6AA69EA69CA680A8CF8CFF162A48D06D
:1009700048D08350066EE8B644D0056606D0510EC6
:10098000C96E046E100E076E42D0500EC96E046E12
:100990003ED00F50030A35E1E9CF49F0EACF4AF0E3
:1009A00009EE00F010C0E9FF83CFEFFF49C0E9FF77
:1009B0004AC0EAFF103E25D0820EC96E046E030EB7
:1009C000016E008424D0E9CF49F0EACF4AF00AEE64
:1009D00000F015C0E9FF83CFEFFF49C0E9FF4AC02F
:1009E000EAFF152A135015620CD0400E62D0C7A042
:1009F000FED78B8000008B9049C0E9FF4AC0EAFF18
:100A0000956A8A8681A2FED795688A961100C7A04A
:100A1000FED78B808A8681A2FED79568C9508B90BD
:100A20008A96110083CF08F0ECD783CF09F0E9D77D
:100A300083CF0AF0E6D78350030B0B6EE2D78344D3
:100A4000E838030B0C6E8350070B0D6E500EC96E09
:100A5000046EDDD7146A8350136ED3E1142AD1D704
:100A6000500EC96E046E0A6A0B6AD1D7820EC96E27
:100A7000046E020E016E0084CAD78350040B04E199
:100A8000580EC96E046EC3D7510EC96E046E040EA3
:100A9000076EBDD7820EC96E046E010E016E008412
:100AA000B6D7500EC96E046EB2D783CF11F0156A57
:100AB000800E1110016E820EC96E046E0084A7D7DD
:0A0AC00083CF17F0166A9DD79CD76C
:060ACA000100DAE100006A
:080AD000CD0000000100000050
:080AD800D9CFE6FFDACFE6FFFB
:100AE000E1CFD9FFE2CFDAFFE652E652E652E65214
:100AF000FC0EDBCFDEFFDBCFDDFFFA0EDBCF3DF000
:100B0000FB0EDBCF3EF0020E3DC0DBFF030E3EC00E
:100B1000DBFFF80EDBCF1DF0F90EDBCF1EF0020E6F
:100B20001D5C000E1E582BE3020EDBCFE9FF030E07
:100B3000DBCFEAFFEECF1DF0EFCF1EF0DECFE9FFF7
:100B4000DDCFEAFF1DC0EEFF1EC0EDFF020EDE2668
:100B5000000EDD22D950020FE96E000EDA20EA6E97
:100B6000020EEE26000EED22D950F80FE96EFF0EB0
:100B7000DA20EA6E020EEE5E000EED5ACAD7F80ECB
:100B8000DBCF1DF0DB06F90EDBCF1EF001E2DB064A
:100B90001D501E1017E0020EDBCFE9FFDB2A030E0B
:100BA000DBCFEAFF01E3DB2AEF50E66EDFCFE9FFA0
:100BB000DF2A010EDBCFEAFF01E3DB2AE552E75033
:100BC000EF6EDDD7040EE15C02E2E16AE552E16E10
:100BD000E552E5CFDAFFE7CFD9FF1200D9CFE6FF24
:100BE000DACFE6FFE1CFD9FFE2CFDAFFE652E652F5
:100BF000FC0EDBCFDEFFDBCFDDFFF80EDBCF1DF021
:100C0000DB06F90EDBCF1EF001E2DB061D501E10E5
:100C10000CE0DFCFE9FFDF2A010EDBCFEAFF01E3C3
:100C2000DB2AFA0EDBCFEFFFE8D7E552E552E552BB
:100C3000E5CFDAFFE7CFD9FF1200D9CFE6FFDACF51
:100C4000E6FFE1CFD9FFE2CFDAFF060EE12402E3AF
:100C5000E168E652E16EFC0EDBCFDEFFDBCFDDFFAD
:100C6000FA0EDBCF3DF0FB0EDBCF3EF0020E3DC0B7
:100C7000DBFF030E3EC0DBFF040EDB6A050EDB6A02
:100C8000F80EDBCF1DF0DB06F90EDBCF1EF001E224
:100C9000DB061D501E1020E0DFCFE9FFDF2A010E2A
:100CA000DBCFEAFF01E3DB2AEFCF21F0020EDBCF3F
:100CB000E9FFDB2A030EDBCFEAFF01E3DB2AEF507B
:100CC000215C1F6E206A040E1FC0DBFF050E20C0D2
:100CD000DBFF1F502010D4E0040EDBCF1DF0050E0B
:100CE000DBCF1EF01DC0F3FF1EC0F4FF060EE15C5B
:100CF00002E2E16AE552E16EE552E5CFDAFFE7CFC5
:100D0000D9FF1200D9CFE6FFDACFE6FFE1CFD9FF56
:100D1000E2CFDAFFFC0EDBCFF6FFFD0EDBCFF7FFF5
:100D20000800F5501AE0FC0EDBCFF6FFFD0EDBCF1E
:100D3000F7FF0800F5CF1DF01E6A1DBE1E68FA0EF3
:100D4000DB501D1803E1FB0EDB501E1806E0FC0E05
:100D5000DB2AFD0EDFE3DB2ADDD7FC0EDBCFF6FF5F
:100D6000FD0EDBCFF7FF0800F5CF1DF01E6A1DBE9C
:100D70001E681DC0F3FF1EC0F4FFE552E5CFDAFF89
:100D8000E7CFD9FF1200D9CFE6FFDACFE6FFE1CFF8
:100D9000D9FFE2CFDAFF060EE12402E3E168E65272
:100DA000E16EFC0EDBCFE9FFFD0EDBCFEAFF040EA8
:100DB000E926000EEA22EF5001E11ED1FC0EDBCF46
:100DC000E9FFFD0EDBCFEAFF2E0EE926000EEA2238
:100DD000EECFDFFF010EEECFDBFF020EEECFDBFF2B
:100DE000030EEECFDBFF010EE66ED9CFE9FFDACFBF
:100DF000EAFFEECFE6FFEECFE6FFEECFE6FFEFCF66
:100E0000E6FFFC0EDBCFE9FFFD0EDBCFEAFF320E83
:100E1000E926000EEA22E9CF1DF0EACF1EF0E9CF65
:100E2000E6FFEACFE6FFFC0EDBCFE9FFFD0EDBCFEE
:100E3000EAFFEE52EF50E66E65EC5EF01F6E080EB4
:100E4000E15C02E2E16AE552E16E1F50000902E056
:100E5000010ED3D0FC0EDBCFE9FFFD0EDBCFEAFFA6
:100E6000040EE926000EEA22EF6AFC0EDBCFE9FF52
:100E7000FD0EDBCFEAFF220EE926000EEA22EECFBE
:100E80001DF0EECF1EF0EECF1FF0EFCF20F0D9CF48
:100E9000E9FFDACFEAFF1D50EE5C1E50EE581F50FE
:100EA000EE582050EE5801E2A7D0FC0EDBCFE9FF50
:100EB000FD0EDBCFEAFF1A0EE926000EEA22EECF86
:100EC00021F0EECF22F0EECF23F0EFCF24F0FC0E96
:100ED000DBCFE9FFFD0EDBCFEAFF220EE926000E95
:100EE000EA22EE502126EE502222EE502322EE502E
:100EF0002422D9CFE9FFDACFEAFF2150EE5C22505D
:100F0000EE582350EE582450EE5876E2FC0EDBCF1C
:100F1000E9FFFD0EDBCFEAFF030EE926000EEA2211
:100F2000EF50E66ED950040FE96E000EDA20EA6E3B
:100F3000E552E750EE6EED6A040EDBCF1DF0050EB4
:100F4000DBCF1EF0020E1D5C000E1E5855E3FC0E9A
:100F5000DBCFE9FFFD0EDBCFEAFF1A0EE926000E1C
:100F6000EA22EECF1DF0EECF1EF0EECF1FF0EFCF56
:100F700020F01D50DE261E50DE221F50DE222050A3
:100F8000DD22DD52DD52010EE66ED9CFE9FFDACF68
:100F9000EAFFEECFE6FFEECFE6FFEECFE6FFEFCFC4
:100FA000E6FFFC0EDBCFE9FFFD0EDBCFEAFF320EE2
:100FB000E926000EEA22E9CF1DF0EACF1EF0E9CFC4
:100FC000E6FFEACFE6FFFC0EDBCFE9FFFD0EDBCF4D
:100FD000EAFFEE52EF50E66E65EC5EF01F6E080E13
:100FE000E15C02E2E16AE552E16E1F50040EDB06AD
:100FF000050EA2E2DB06A0D7000E1D6E060EE15C18
:1010000002E2E16AE552E16E1D50E552E5CFDAFFFA
:10101000E7CFD9FF1200D9CFE6FFDACFE6FFE1CF65
:10102000D9FFE2CFDAFFF80EDBCF1DF0F90EDBCFF0
:101030001EF0FA0EDBCF1FF0FB0EDBCF20F0FC0E14
:10104000DBCFE9FFFD0EDBCFEAFF2E0EE926000E17
:10105000EA221D50EE1808E11E50EE1805E11F505F
:10106000EE1802E12050EE185AE0FC0EDBCFE6FF4E
:10107000FD0EDBCFE6FF87DEE552E552000937E1E2
:10108000010EE66ED950F80FE96EFF0EDA20EA6E17
:10109000EECFE6FFEECFE6FFEECFE6FFEFCFE6FFC7
:1010A000FC0EDBCFE9FFFD0EDBCFEAFF320EE926B7
:1010B000000EEA22E9CF1DF0EACF1EF0E9CFE6FFED
:1010C000EACFE6FFFC0EDBCFE9FFFD0EDBCFEAFF48
:1010D000EE52EF50E66EF5EC5DF01F6E080EE15C2F
:1010E00002E2E16AE552E16E1F50000902E0010EE2
:1010F00017D0FC0EDBCFE9FFFD0EDBCFEAFF2E0E93
:10110000E926000EEA22F80EDBCFEEFFF90EDBCF68
:10111000EEFFFA0EDBCFEEFFFB0EDBCFEEFF000E95
:10112000E552E5CFDAFFE7CFD9FF1200D9CFE6FFCE
:10113000DACFE6FFE1CFD9FFE2CFDAFFE652FC0ECD
:10114000DBCFE6FFFD0EDBCFE6FF1DDEE552E5520D
:10115000DF6EDF5001E028D1FC0EDBCFE9FFFD0E92
:10116000DBCFEAFFEF50030801E007D1FC0EDBCF35
:10117000E9FFFD0EDBCFEAFF050EE926000EEA22AD
:10118000EF5001E1FAD0FC0EDBCFE9FFFD0EDBCF23
:10119000EAFF2E0EE926000EEA22EE6AEE6AEE6AF9
:1011A000EE6AE66A020EE66E000EE66EE66AFC0E77
:1011B000DBCFE9FFFD0EDBCFEAFF320EE926000EA2
:1011C000EA22E9CF1DF0EACF1EF0E9CFE6FFEACF31
:1011D000E6FF04DD1F6E060EE15C02E2E16AE55205
:1011E000E16E1F50FC0EDBCFE9FFFD0EDBCFEAFF07
:1011F000320EE926000EEA22FE0EE926010EEA2250
:10120000550EEE6EAA0EED6EFC0EDBCFE9FFFD0E65
:10121000DBCFEAFF320EE926000EEA22520EEE6E16
:10122000EE6E610EEE6E410EEE6EFC0EDBCFE9FF50
:10123000FD0EDBCFEAFF320EE926000EEA22E40EB5
:10124000E926010EEA22720EEE6EEE6E410EEE6E91
:10125000610EEE6EFC0EDBCFE9FFFD0EDBCFEAFF89
:101260000E0EE926000EEA22EECF1DF0EECF1EF0A4
:10127000EECF1FF0EFCF20F0FC0EDBCFE9FFFD0E2D
:10128000DBCFEAFF320EE926000EEA22E80EE9265D
:10129000010EEA221DC0EEFF1EC0EEFF1FC0EEFFD2
:1012A00020C0EEFFFC0EDBCFE9FFFD0EDBCFEAFF37
:1012B0000A0EE926000EEA22EECF1DF0EECF1EF058
:1012C000EECF1FF0EFCF20F0FC0EDBCFE9FFFD0EDD
:1012D000DBCFEAFF320EE926000EEA22EC0EE92609
:1012E000010EEA221DC0EEFF1EC0EEFF1FC0EEFF82
:1012F00020C0EEFFE66EFC0EDBCFE9FFFD0EDBCF7C
:10130000EAFF120EE926000EEA22EECFE6FFEECF4C
:10131000E6FFEECFE6FFEFCFE6FFFC0EDBCFE9FF07
:10132000FD0EDBCFEAFF320EE926000EEA22E9CFFE
:101330001DF0EACF1EF0E9CFE6FFEACFE6FFFC0E94
:10134000DBCFE9FFFD0EDBCFEAFFEE52EF50E66E9A
:1013500065EC5EF01F6E080EE15C02E2E16AE552A8
:10136000E16E1F50FC0EDBCFE9FFFD0EDBCFEAFF85
:10137000050EE926000EEA22EF6A000EE66EE66A26
:10138000E66AFC0EDBCFE9FFFD0EDBCFEAFFEE5293
:10139000EF50E66ED7EC5EF0E552E552E552E552CD
:1013A000000902E0010EDF6EDF50E552E552E5CFA5
:1013B000DAFFE7CFD9FF1200D9CFE6FFDACFE6FF99
:1013C000E1CFD9FFE2CFDAFFE150F80FE96EFF0E6F
:1013D000E220EA6E020EEE5E000EEE5AEE5AEE5A71
:1013E000FC0EDBCFE9FFFD0EDBCFEAFF160EE92690
:1013F000000EEA22EECF1DF0EECF1EF0EECF1FF072
:10140000EFCF20F0020E1D5E000E1E5A1F5A205A0A
:10141000D950F80FE96EFF0EDA20EA6E1D50EE5C2F
:101420001E50EE581F50EE582050EE5805E33B6A10
:101430003C6A3D6A3E6A4AD0FC0EDBCFE9FFFD0EF6
:10144000DBCFEAFF2A0EE926000EEA22EECF25F0D6
:10145000EECF26F0EECF27F0EFCF28F0FC0EDBCF5B
:10146000E9FFFD0EDBCFEAFF020EE926000EEA22BD
:10147000EFCF21F0226A236A246A21C03BF022C008
:101480003CF023C03DF024C03EF0F80EDBCF40F02E
:10149000F90EDBCF41F0FA0EDBCF42F0FB0EDBCFD3
:1014A00043F0CEEC6FF0375025241D6E38502620C7
:1014B0001E6E395027201F6E3A502820206E1DC006
:1014C0003BF01EC03CF01FC03DF03E6EE552E5CF44
:1014D000DAFFE7CFD9FF1200D9CFE6FFDACFE6FF78
:1014E000E1CFD9FFE2CFDAFF060EE12402E3E168A3
:1014F000E652E16ED950F80FE96EFF0EDA20EA6E7F
:10150000020EEE5C000EEE58000EEE58000EEE5885
:101510001FE3F80EDBCF1DF0F90EDBCF1EF0FA0E45
:10152000DBCF1FF0FB0EDBCF20F0FC0EDBCFE9FFA3
:10153000FD0EDBCFEAFF160EE926000EEA22EE5082
:101540001D5CEE501E58EE501F58EE50205806E31A
:10155000010E3B6E3C6A3D6A3E6A29D2FC0EDBCF2F
:10156000E9FFFD0EDBCFEAFFEF50030A01E18AD16C
:10157000010A01E108D1030A01E015D2F80EDBCF20
:101580003DF0F90EDBCF3EF0020E3DC0DBFF030E57
:101590003EC0DBFF020EDBCF1DF0030EDBCF1EF0E3
:1015A000010E0F0B05E0D8901E321D32E806FBE15C
:1015B000D950020FE96E000EDA20EA6E1D50EE26B9
:1015C0001E50ED22020EDBCF1DF0030EDBCF1EF00E
:1015D000090E0F0B05E0D8901E321D32E806FBE124
:1015E0001F6A206AFC0EDBCFE9FFFD0EDBCFEAFFAE
:1015F000220EE926000EEA22EE501D26EE501E2293
:10160000EE501F22EE5020221DC0E6FF1EC0E6FF56
:101610001FC0E6FF20C0E6FFFC0EDBCFE6FFFD0E9D
:10162000DBCFE6FFF8DC216E060EE15C02E2E16A48
:10163000E552E16E2150000901E0B5D1FC0EDBCF8F
:10164000E9FFFD0EDBCFEAFF320EE926000EEA22AB
:10165000020EDBCF1FF0030EDBCF20F00001010EE6
:101660002016E9501F24E96EEA502020EA6EEF5060
:10167000DE6EDD6A020EDB2A030E01E3DB2A020EB8
:10168000DBCF1DF0030EDBCF1EF0090E0F0B05E0C4
:10169000D8901E321D32E806FBE11F6A206AFC0E5C
:1016A000DBCFE9FFFD0EDBCFEAFF220EE926000EBD
:1016B000EA22EE501D26EE501E22EE501F22EE5062
:1016C00020221DC0E6FF1EC0E6FF1FC0E6FF20C0AF
:1016D000E6FFFC0EDBCFE6FFFD0EDBCFE6FF9BDC7B
:1016E000216E060EE15C02E2E16AE552E16E2150F4
:1016F000000901E058D1FC0EDBCFE9FFFD0EDBCF86
:10170000EAFF320EE926000EEA22020EDBCF1FF0BE
:10171000030EDBCF20F0010E2016E9501F24E96EE6
:10172000EA502020EA6EEF50000EF350DF12010E57
:10173000216E226A236A246AD950F80FE96EFF0EDF
:10174000DA20EA6EEE502116EE502216EE502316E5
:10175000EE50241621502210231024100BE0DECF6F
:101760001DF0DDCF1EF0040ED8901E321D32E804AD
:10177000FBE185D0DECF1DF0DDCF1EF0FF0E1D1684
:101780000F0E1E167CD0F80EDBCF1DF0F90EDBCF4E
:101790001EF0FA0EDBCF1FF0FB0EDBCF20F0080EA1
:1017A000D89020321F321E321D32E806F9E1FC0EBD
:1017B000DBCFE9FFFD0EDBCFEAFF220EE926000EAC
:1017C000EA22EE501D26EE501E22EE501F22EE5051
:1017D00020221DC0E6FF1EC0E6FF1FC0E6FF20C09E
:1017E000E6FFFC0EDBCFE6FFFD0EDBCFE6FF13DCF2
:1017F000216E060EE15C02E2E16AE552E16E2150E3
:10180000000901E0D0D0FC0EDBCFE9FFFD0EDBCFFD
:10181000EAFF320EE926000EEA22E9CF1FF0EACFF6
:1018200020F0F80EDBCF3BF0F90EDBCF3CF0FA0EE8
:10183000DBCF3DF0FB0EDBCF3EF0D8903B363C36A5
:101840003D363E36406A020E416E426A436A2BECD8
:1018500070F01F5037241D6E205038201E6E040E6D
:101860001DC0DBFF050E1EC0DBFF040EDBCFE9FF52
:10187000050EDBCFEAFFEECF1DF0EFCF1EF01F6AA3
:10188000206A88D0F80EDBCF1DF0F90EDBCF1EF0FA
:10189000FA0EDBCF1FF0FB0EDBCF20F0070ED89047
:1018A00020321F321E321D32E806F9E1FC0EDBCF7A
:1018B000E9FFFD0EDBCFEAFF220EE926000EEA2249
:1018C000EE501D26EE501E22EE501F22EE5020221A
:1018D0001DC0E6FF1EC0E6FF1FC0E6FF20C0E6FFFA
:1018E000FC0EDBCFE6FFFD0EDBCFE6FF0BEC08F0D6
:1018F000216E060EE15C02E2E16AE552E16E2150E2
:10190000000951E1FC0EDBCFE9FFFD0EDBCFEAFF62
:10191000320EE926000EEA22E9CF1FF0EACF20F0CE
:10192000F80EDBCF3BF0F90EDBCF3CF0FA0EDBCF4D
:101930003DF0FB0EDBCF3EF0020ED8903B363C363E
:101940003D363E36E806F9E1406A020E416E426AD3
:10195000436A2BEC70F01F5037241D6E2050382046
:101960001E6E040E1DC0DBFF050E1EC0DBFF1D68D2
:101970001E681F680F0E206E040EDBCFE9FF050EF8
:10198000DBCFEAFFEE501D16EE501E16EE501F166E
:10199000EE5020161DC03BF01EC03CF01FC03DF0B5
:1019A00020C03EF004D03B683C683D683E68060EAF
:1019B000E15C02E2E16AE552E16EE552E5CFDAFF71
:1019C000E7CFD9FF1200D9CFE6FFDACFE6FFE1CFAC
:1019D000D9FFE2CFDAFFE652E652E652E652E6528D
:1019E000D950F80FE96EFF0EDA20EA6E020EEE5CB7
:1019F000000EEE58000EEE58000EEE581FE3F80EE3
:101A0000DBCF1DF0F90EDBCF1EF0FA0EDBCF1FF09F
:101A1000FB0EDBCF20F0FC0EDBCFE9FFFD0EDBCFB2
:101A2000EAFF160EE926000EEA22EE501D5CEE508B
:101A30001E58EE501F58EE50205806E3020EF36E6B
:101A4000040EF3CFDBFFBDD2FC0EDBCFE9FFFD0EB2
:101A5000DBCFEAFFEF50030A01E1F5D1010A01E112
:101A60006ED1030A01E09CD2F80EDBCFDEFFDBCFA4
:101A7000DDFFDECF1DF0DDCF1EF0010E0F0B05E008
:101A8000D8901E321D32E806FBE1D9CFE9FFDACF4C
:101A9000EAFF1D50EE261E50ED22DECF1DF0DDCFF9
:101AA0001EF0090E0F0B05E0D8901E321D32E8061D
:101AB000FBE11F6A206AFC0EDBCFE9FFFD0EDBCFE6
:101AC000EAFF220EE926000EEA22EE501D26EE5015
:101AD0001E22EE501F22EE5020221DC0E6FF1EC027
:101AE000E6FF1FC0E6FF20C0E6FFFC0EDBCFE6FFEF
:101AF000FD0EDBCFE6FF0BEC08F0216E060EE15C7D
:101B000002E2E16AE552E16E2150E76E040EE7CF92
:101B1000DBFFDB5001E049D2FC0EDBCFE9FFFD0E1D
:101B2000DBCFEAFF320EE926000EEA22DECF21F0FB
:101B3000DDCF22F00001010E2216E95021241D6E96
:101B4000EA5022201E6E020E1DC0DBFF030E1EC0D7
:101B5000DBFF010E1D6E1E6A1F6A206AD950F80F46
:101B6000E96EFF0EDA20EA6EEE501D16EE501E16DC
:101B7000EE501F16EE5020161D501E101F10201084
:101B80000EE0F40EDB38F00B216E020EDBCFE9FF26
:101B9000030EDBCFEAFFEF500F0B211002D0F40E43
:101BA000DB50E66E020EDBCFE9FF030EDBCFEAFF70
:101BB000E552E750EF6EDF2A010E01E3DB2AFC0E4F
:101BC000DBCFE9FFFD0EDBCFEAFF040EE926000EB6
:101BD000EA22010EEF6EDECF1DF0DDCF1EF0090E02
:101BE0000F0B05E0D8901E321D32E806FBE11F6A9C
:101BF000206AFC0EDBCFE9FFFD0EDBCFEAFF220EF1
:101C0000E926000EEA22EE501D26EE501E22EE506E
:101C10001F22EE5020221DC0E6FF1EC0E6FF1FC09F
:101C2000E6FF20C0E6FFFC0EDBCFE6FFFD0EDBCFBC
:101C3000E6FF0BEC08F0216E060EE15C02E2E16AC1
:101C4000E552E16E2150E76E040EE7CFDBFFDB507B
:101C500001E0ABD1FC0EDBCFE9FFFD0EDBCFEAFFED
:101C6000320EE926000EEA22DECF21F0DDCF22F08F
:101C7000010E2216E95021241D6EEA5022201E6E0C
:101C8000020E1DC0DBFF030E1EC0DBFF010E1D6E2A
:101C90001E6A1F6A206AD950F80FE96EFF0EDA201B
:101CA000EA6EEE501D16EE501E16EE501F16EE5048
:101CB00020161D501E101F10201016E0F40EDBCF52
:101CC00021F0F50EDBCF22F0F60EDBCF23F0F70E7E
:101CD000DBCF24F0040ED89024322332223221327A
:101CE000E806F9E1215020D0F40EDBCF26F0F50E06
:101CF000DBCF27F0F60EDBCF28F0F70EDBCF29F095
:101D0000080ED8902932283227322632E806F9E127
:101D10000F0E2614256E020EDBCFE9FF030EDBCF7C
:101D2000EAFFEF50F00B2510E66E020EDBCFE9FF65
:101D3000030EDBCFEAFFE552E750EF6E36D1F80E27
:101D4000DBCF1DF0F90EDBCF1EF0FA0EDBCF1FF05C
:101D5000FB0EDBCF20F0080ED89020321F321E324F
:101D60001D32E806F9E1FC0EDBCFE9FFFD0EDBCF0B
:101D7000EAFF220EE926000EEA22EE501D26EE5062
:101D80001E22EE501F22EE5020221DC0E6FF1EC074
:101D9000E6FF1FC0E6FF20C0E6FFFC0EDBCFE6FF3C
:101DA000FD0EDBCFE6FF0BEC08F0216E060EE15CCA
:101DB00002E2E16AE552E16E2150E76E040EE7CFE0
:101DC000DBFFDB5001E0F1D0FC0EDBCFE9FFFD0EC5
:101DD000DBCFEAFF320EE926000EEA22E9CF1FF040
:101DE000EACF20F0F80EDBCF3BF0F90EDBCF3CF072
:101DF000FA0EDBCF3DF0FB0EDBCF3EF0D8903B364A
:101E00003C363D363E36406A020E416E426A436AB7
:101E10002BEC70F01F5037241D6E205038201E6EA2
:101E2000020E1DC0DBFF030E1EC0DBFF020EDBCF68
:101E3000E9FF030EDBCFEAFFF40EDBCFEEFFF50E7A
:101E4000DBCFEDFFB2D0F80EDBCF1DF0F90EDBCF0C
:101E50001EF0FA0EDBCF1FF0FB0EDBCF20F0070EDB
:101E6000D89020321F321E321D32E806F9E1FC0EF6
:101E7000DBCFE9FFFD0EDBCFEAFF220EE926000EE5
:101E8000EA22EE501D26EE501E22EE501F22EE508A
:101E900020221DC0E6FF1EC0E6FF1FC0E6FF20C0D7
:101EA000E6FFFC0EDBCFE6FFFD0EDBCFE6FF0BEC23
:101EB00008F0216E060EE15C02E2E16AE552E16E95
:101EC0002150E76E040EE7CFDBFFDB506EE1FC0E26
:101ED000DBCFE9FFFD0EDBCFEAFF320EE926000E75
:101EE000EA22E9CF1FF0EACF20F0F80EDBCF3BF07B
:101EF000F90EDBCF3CF0FA0EDBCF3DF0FB0EDBCF73
:101F00003EF0020ED8903B363C363D363E36E80673
:101F1000F9E1406A020E416E426A436A2BEC70F0AE
:101F20001F5037241D6E205038201E6E020E1DC01B
:101F3000DBFF030E1EC0DBFF1D6A1E6A1F6AF00E68
:101F4000206E020EDBCFE9FF030EDBCFEAFFEE507F
:101F50001D16EE501E16EE501F16EE502016D950CC
:101F6000F40FE96EFF0EDA20EA6E1D50EE121E50DD
:101F7000EE121F50EE122050EE12020EDBCFE9FFE0
:101F8000030EDBCFEAFFF40EDBCFEEFFF50EDBCF67
:101F9000EEFFF60EDBCFEEFFF70EDBCFEEFF05D048
:101FA000020EF36E040EF3CFDBFFFC0EDBCFE9FF76
:101FB000FD0EDBCFEAFF040EE926000EEA22010E39
:101FC000EF6E040EDB501D6E050EE15C02E2E16A6D
:101FD000E552E16E1D50E552E5CFDAFFE7CFD9FFBC
:101FE0001200D9CFE6FFDACFE6FFE1CFD9FFE2CF8B
:101FF000DAFFE652E652E652E652E652D950F80FC0
:10200000E96EFF0EDA20EA6E020EEE5C000EEE586C
:10201000000EEE58000EEE5801E28BD0F80EDBCF2A
:102020001DF0F90EDBCF1EF0FA0EDBCF1FF0FB0E1A
:10203000DBCF20F0FC0EDBCFE9FFFD0EDBCFEAFFAC
:10204000160EE926000EEA22EE501D5CEE501E58D8
:10205000EE501F58EE5020586CE2DF6AF80EDBCFCE
:102060001DF0F90EDBCF1EF0FA0EDBCF1FF0FB0EDA
:10207000DBCF20F0FC0EDBCFE9FFFD0EDBCFEAFF6C
:10208000160EE926000EEA22EE501D5CEE501E5898
:10209000EE501F58EE50205801E3C9D0D950F80F28
:1020A000E96EFF0EDA20EA6EEECFE6FFEECFE6FF36
:1020B000EECFE6FFEFCFE6FFFC0EDBCFE6FFFD0E37
:1020C000DBCFE6FF6CEC0AF01D6E060EE15C02E26F
:1020D000E16AE552E16E1D50010E3BC0DBFF020ECE
:1020E0003CC0DBFF030E3DC0DBFF040E3EC0DBFF48
:1020F000010EDBCF1DF0020EDBCF1EF0030EDBCF97
:102100001FF0040EDBCF20F01D501E101F102010FA
:1021100001E18DD0D950010FE96E000EDA20EA6E90
:10212000010EEE1808E1EE5006E1EE5004E1EE502B
:1021300002E1020E13D0D950010FE96E000EDA2031
:10214000EA6EE868EE180CE1E868EE1809E1E86864
:10215000EE1806E1E868EE1803E1010EDF6E67D0C5
:10216000E66AE66AE66AE66AD950F80FE96EFF0E9B
:10217000DA20EA6EEECFE6FFEECFE6FFEECFE6FF27
:10218000EFCFE6FFFC0EDBCFE6FFFD0EDBCFE6FF79
:102190001ADC1D6E0A0EE15C02E2E16AE552E16EB4
:1021A0001D50DF6EDF5043E1FC0EDBCFE9FFFD0E7B
:1021B000DBCFEAFF0E0EE926000EEA22E868EE18F1
:1021C00008E1E868EE1805E1E868EE1802E1E86861
:1021D000EE181AE0FC0EDBCFE9FFFD0EDBCFEAFFC5
:1021E0000E0EE926000EEA22EE2AEE22EE22EE2262
:1021F000FC0EDBCFE9FFFD0EDBCFEAFF050EE92683
:10220000000EEA22010EEF6ED950010FE96E000EAA
:10221000DA20EA6EF80EEECFDBFFF90EEECFDBFF31
:10222000FA0EEECFDBFFFB0EEECFDBFF17D7DF5052
:102230001D6E050EE15C02E2E16AE552E16E1D50A1
:10224000E552E5CFDAFFE7CFD9FF1200D9CFE6FF9D
:10225000DACFE6FFE1CFD9FFE2CFDAFF0D0EE124BE
:1022600002E3E168E652E16EF80EDBCF1DF0F90EF5
:10227000DBCF1EF0FA0EDBCF1FF0FB0EDBCF20F022
:102280001D501E101F10201053E1FC0EDBCFE9FF84
:10229000FD0EDBCFEAFF0A0EE926000EEA22080E49
:1022A000EECFDBFF090EEECFDBFF0A0EEECFDBFF3A
:1022B0000B0EEECFDBFF080EDBCF1DF0090EDBCFE0
:1022C0001EF00A0EDBCF1FF00B0EDBCF20F01D50EF
:1022D0001E101F10201020E0080EDBCF21F0090E89
:1022E000DBCF22F00A0EDBCF23F00B0EDBCF24F086
:1022F000FC0EDBCFE9FFFD0EDBCFEAFF160EE92671
:10230000000EEA22EE50215CEE502258EE50235887
:10231000EE50245801E276D0010EF36E080EF3CF92
:10232000DBFF090EDB6A0A0EDB6A0B0EDB6A6AD082
:10233000D950F80FE96EFF0EDA20EA6EEECFE6FF15
:10234000EECFE6FFEECFE6FFEFCFE6FFFC0EDBCFF2
:10235000E6FFFD0EDBCFE6FF6CEC0AF01D6E060E0D
:10236000E15C02E2E16AE552E16E1D503BC0DEFF36
:102370003CC0DEFF3DC0DEFF3EC0DDFFDD52DD5272
:10238000D9CFE9FFDACFEAFF020EEE5C000EEE587D
:10239000000EEE58000EEE5803E2010E3B6E3CD1EB
:1023A000FC0EDBCFE9FFFD0EDBCFEAFF160EE926C0
:1023B000000EEA22EECF1DF0EECF1EF0EECF1FF0A2
:1023C000EFCF20F0D9CFE9FFDACFEAFF1D50EE5C66
:1023D0001E50EE581F50EE582050EE5801E2ECD03F
:1023E000D950F80FE96EFF0EDA20EA6E080EEECF34
:1023F000DBFF090EEECFDBFF0A0EEECFDBFF0B0E8D
:10240000EECFDBFFD950080FE96E000EDA20EA6E3E
:10241000040EEECFDBFF050EEECFDBFF060EEECF98
:10242000DBFF070EEECFDBFFD950040FE96E000E85
:10243000DA20EA6EEE2A000EEE22EE22EE22040EE2
:10244000DBCF1DF0050EDBCF1EF0060EDBCF1FF03D
:10245000070EDBCF20F0FC0EDBCFE9FFFD0EDBCF5C
:10246000EAFF160EE926000EEA22EE501D5CEE5041
:102470001E58EE501F58EE50205828E3020EF36EFF
:10248000040EF3CFDBFF050EDB6A060EDB6A070ED8
:10249000DB6A080EDBCF1DF0090EDBCF1EF00A0E43
:1024A000DBCF1FF00B0EDBCF20F0D950040FE96E0D
:1024B000000EDA20EA6EEE501D5CEE501E58EE5013
:1024C0001F58EE50205802E23B6AA6D0D950040FA4
:1024D000E96E000EDA20EA6EEECFE6FFEECFE6FF01
:1024E000EECFE6FFEFCFE6FFFC0EDBCFE6FFFD0E03
:1024F000DBCFE6FF6CEC0AF01D6E060EE15C02E23B
:10250000E16AE552E16E1D503BC0DEFF3CC0DEFFDC
:102510003DC0DEFF3EC0DDFFDD52DD52D9CFE9FF19
:10252000DACFEAFFEECF1DF0EECF1EF0EECF1FF0B8
:10253000EFCF20F01D501E101F10201020E1E66884
:10254000E668E6680F0EE66ED950040FE96E000EDD
:10255000DA20EA6EEECFE6FFEECFE6FFEECFE6FF43
:10256000EFCFE6FFFC0EDBCFE6FFFD0EDBCFE6FF95
:10257000E3EC0CF01D6E0A0EE15C54E251D0D9CFB1
:10258000E9FFDACFEAFFE868EE1808E1E868EE183C
:1025900005E1E868EE1802E1E868EE180DE0D9CF31
:1025A000E9FFDACFEAFF010EEE1811E1EE500FE17C
:1025B000EE500DE1EE500BE1DECF3BF0DECF3CF014
:1025C000DECF3DF0DDCF3EF0DD52DD52EBD0040E2C
:1025D000DBCF1DF0050EDBCF1EF0060EDBCF1FF0AC
:1025E000070EDBCF20F0D950080FE96E000EDA207D
:1025F000EA6E1D50EE1801E017D71E50EE1801E0EC
:1026000013D71F50EE1801E00FD72050EE1801E04D
:102610000BD701E009D73B6A3C6A3D6A3E6AC2D0EB
:10262000E16AE552E16E1D50E76E0C0EE7CFDBFF6D
:10263000DB5041E1F80EDBCF1DF0F90EDBCF1EF0D1
:10264000FA0EDBCF1FF0FB0EDBCF20F01D501E106B
:102650001F10201030E0D950040FE96E000EDA2070
:10266000EA6EEECFE6FFEECFE6FFEECFE6FFEFCF6E
:10267000E6FFD950F80FE96EFF0EDA20EA6EEECFD2
:10268000E6FFEECFE6FFEECFE6FFEFCFE6FFFC0E74
:10269000DBCFE6FFFD0EDBCFE6FFE3EC0CF01D6EBB
:1026A0000A0EE15C02E2E16AE552E16E1D50E76E5E
:1026B0000C0EE7CFDBFF0C0EDB5047E1FC0EDBCF4F
:1026C000E9FFFD0EDBCFEAFF0A0EE926000EEA2243
:1026D000040EDBCFEEFF050EDBCFEEFF060EDBCFE9
:1026E000EEFF070EDBCFEEFFFC0EDBCFE9FFFD0EAA
:1026F000DBCFEAFF0E0EE926000EEA22E868EE18AC
:1027000008E1E868EE1805E1E868EE1802E1E8681B
:10271000EE1834E0FC0EDBCFE9FFFD0EDBCFEAFF65
:102720000E0EE926000EEA22EE06EE5AEE5AEE5A98
:10273000FC0EDBCFE9FFFD0EDBCFEAFF050EE9263D
:10274000000EEA22010EEF6E19D00C0EDB0405E13B
:102750001D681E681F68206805D0010E1D6E1E6A68
:102760001F6A206A040E1DC0DBFF050E1EC0DBFFC2
:10277000060E1FC0DBFF070E20C0DBFF040EDBCF01
:102780001DF0050EDBCF1EF0060EDBCF1FF0070E8F
:10279000DBCF20F01DC03BF01EC03CF01FC03DF061
:1027A00020C03EF00D0EE15C02E2E16AE552E16E0E
:1027B000E552E5CFDAFFE7CFD9FF1200D9CFE6FF28
:1027C000DACFE6FFE1CFD9FFE2CFDAFF0A0EE1244C
:1027D00002E3E168E652E16EFC0EDBCFE9FFFD0E9D
:1027E000DBCFEAFF200EE926000EEA22EECF1DF035
:1027F000EFCF1EF0040E1D26000E1E22080E1DC077
:10280000DBFF090E1EC0DBFFFC0EDBCFE9FFFD0E78
:10281000DBCFEAFFEE50EFCFEAFFE96E020EE926CA
:10282000000EEA22EFCF1DF01E6A1F6A206AF80E22
:10283000DBCF3BF0F90EDBCF3CF0FA0EDBCF3DF007
:10284000FB0EDBCF3EF0406A020E416E426A436AE5
:102850002BEC70F01DC040F01EC041F01FC042F0D4
:1028600020C043F02BEC70F03BC0DEFF3CC0DEFF2D
:102870003DC0DEFF3EC0DDFFDD52DD52D950080F06
:10288000E96E000EDA20EA6EEECFF3FFEDCFF4FF33
:10289000040EEE26000EEF22F3CFE9FFF4CFEAFF9D
:1028A000040EEECFDBFF050EEECFDBFF060EEECF04
:1028B000DBFF070EEECFDBFF040EDBCF1DF0050EB6
:1028C000DBCF1EF0060EDBCF1FF0070EDBCF20F0B4
:1028D0001D501E101F10201005E13B6A3C6A3D6A26
:1028E0003E6A56D0040EDBCF1DF0050EDBCF1EF086
:1028F000060EDBCF1FF0070EDBCF20F0D9CFE9FFAC
:10290000DACFEAFF1D50EE5C1E50EE581F50EE5815
:102910002050EE581BE3D9CFE9FFDACFEAFF040ECF
:10292000DB50EE5E050EDB50EE5A060EDB50EE5A23
:10293000070EDB50EE5AD950080FE96E000EDA2070
:10294000EA6E040EEE26000EEF2298D7080EDBCFBB
:10295000E9FF090EDBCFEAFFEECF1DF0EECF1EF050
:10296000EECF1FF0EFCF20F0D9CFE9FFDACFEAFFAB
:10297000EE501D26EE501E22EE501F22EE50202259
:102980001DC03BF01EC03CF01FC03DF020C03EF01B
:102990000A0EE15C02E2E16AE552E16EE552E5CF42
:1029A000DAFFE7CFD9FF1200D9CFE6FFDACFE6FF93
:1029B000E1CFD9FFE2CFDAFF060EE12402E3E168BE
:1029C000E652E16EFC0EDBCFE9FFFD0EDBCFEAFF46
:1029D000040EE926000EEA22FA0EDBCFEEFFFB0E14
:1029E000DBCFEDFFFC0EDBCFE9FFFD0EDBCFEAFF17
:1029F000060EE926000EEA22EECFDFFF010EEECF33
:102A0000DBFF020EEECFDBFF030EEECFDBFFD9CFF5
:102A1000E9FFDACFEAFF010EEE1805E1EE5003E11F
:102A2000EE5001E1EE5001E164D1FC0EDBCFE9FF95
:102A3000FD0EDBCFEAFFEE50EFCFEAFFE96E160E98
:102A4000E926000EEA22EECF1DF0EECF1EF0EECF0B
:102A50001FF0EFCF20F0D9CFE9FFDACFEAFF1D500A
:102A6000EE5C1E50EE581F50EE582050EE5801E319
:102A700040D1D9CFE9FFDACFEAFFEECF1DF0EECF9C
:102A80001EF0EECF1FF0EFCF20F01D501E101F10D4
:102A9000201026E1FC0EDBCFE9FFFD0EDBCFEAFFC5
:102AA000EE50EFCFEAFFE96EEF50030819E1FC0E9C
:102AB000DBCFE9FFFD0EDBCFEAFFEE50EFCFEAFF01
:102AC000E96E260EE926000EEA22EECFDFFF010EA8
:102AD000EECFDBFF020EEECFDBFF030EEECFDBFF10
:102AE000D9CFE9FFDACFEAFFEECF1DF0EECF1EF02F
:102AF000EECF1FF0EFCF20F01D501E101F10201042
:102B00005AE1FC0EDBCFE9FFFD0EDBCFEAFF0A0E38
:102B1000E926000EEA22DFCFEEFF010EDBCFEEFF4B
:102B2000020EDBCFEEFF030EDBCFEEFFFA0EDBCFA4
:102B30001DF0FB0EDBCF1EF0FC0EDBCFE9FFFD0E20
:102B4000DBCFEAFFEE50EFCFEAFFE96E080EE92691
:102B5000000EEA22EECF1FF0EFCF20F01F501D5CD9
:102B600020501E5801E3C5D0FA0EDBCF1DF0FB0E3E
:102B7000DBCF1EF0040E0F0B05E0D8901E321D3285
:102B8000E806FBE11F6A206AFC0EDBCFE9FFFD0EC1
:102B9000DBCFEAFFEE50EFCFEAFFE96E260EE92623
:102BA000000EEA22EE501D26EE501E22EE501F228D
:102BB000EE50202216D1FC0EDBCFE9FFFD0EDBCF5D
:102BC000EAFFEE50EFCFEAFFE96E020EE926000EB3
:102BD000EA22EF501D6E1E6A100E3D6E3E6A1DC049
:102BE00042F01EC043F04FEC70F0040E3BC0DBFF20
:102BF000050E3CC0DBFFFA0EDBCF1DF0FB0EDBCF7A
:102C00001EF0040EDBCF1FF0050EDBCF20F01F50AF
:102C10001D5C20501E5801E27FD0D9CFE9FFDACFEA
:102C2000EAFFEECFE6FFEECFE6FFEECFE6FFEFCF17
:102C3000E6FFFC0EDBCFE9FFFD0EDBCFEAFFEECFB8
:102C4000E6FFEFCFE6FF6CEC0AF01D6E060EE15CCE
:102C500002E2E16AE552E16E1D503BC0DEFF3CC07E
:102C6000DEFF3DC0DEFF3EC0DDFFDD52DD52D9CFCD
:102C7000E9FFDACFEAFFE868EE180BE1E868EE1842
:102C800008E1E868EE1805E1E868EE1802E1010ED7
:102C9000EDD0D9CFE9FFDACFEAFF020EEE5C000EED
:102CA000EE58000EEE58000EEE5823E3FC0EDBCF7C
:102CB000E9FFFD0EDBCFEAFFEE50EFCFEAFFE96E52
:102CC000160EE926000EEA22EECF1DF0EECF1EF022
:102CD000EECF1FF0EFCF20F0D9CFE9FFDACFEAFF38
:102CE0001D50EE5C1E50EE581F50EE582050EE580E
:102CF00002E3020EBBD0040EDBCF1DF0050EDBCFCE
:102D00001EF0D950FA0FE96EFF0EDA20EA6E1D5060
:102D1000EE5E1E50ED5A6FD7FC0EDBCFE9FFFD0EC5
:102D2000DBCFEAFF0A0EE926000EEA22DFCFEEFF34
:102D3000010EDBCFEEFF020EDBCFEEFF030EDBCF8B
:102D4000EEFFFA0EDBCF22F0FB0EDBCF23F0040EFA
:102D50000F0B05E0D89023322232E806FBE1246A0B
:102D6000256A22C0E6FF23C0E6FF24C0E6FF25C097
:102D7000E6FFD9CFE9FFDACFEAFFEECFE6FFEECFED
:102D8000E6FFEECFE6FFEFCFE6FFFC0EDBCFE9FF7D
:102D9000FD0EDBCFEAFFEECFE6FFEFCFE6FFDCEC88
:102DA00009F0216E060EE15C02E2E16AE552E16E95
:102DB0002150E552E7CF25F0E552E7CF24F0E55268
:102DC000E7CF23F0E552E7CF22F03B5022241D6EDF
:102DD0003C5023201E6E3D5024201F6E3E50252067
:102DE000206EFC0EDBCFE9FFFD0EDBCFEAFF0E0EFF
:102DF000E926000EEA221DC0EEFF1EC0EEFF1FC036
:102E0000EEFF20C0EEFFFC0EDBCFE9FFFD0EDBCFB7
:102E1000EAFFEE50EFCFEAFFE96E320EE926000E30
:102E2000EA22E9CF1FF0EACF20F0FA0EDBCF21F043
:102E3000FB0E226A0F0E2116050ED890213622367F
:102E4000E806FBE11F5021241D6E205022201E6E3B
:102E5000FC0EDBCFE9FFFD0EDBCFEAFF120EE92609
:102E6000000EEA221DC0EEFF1EC0EDFF1D6E060E15
:102E7000E15C02E2E16AE552E16E1D50E552E5CF08
:102E8000DAFFE7CFD9FF1200D9CFE6FFDACFE6FFAE
:102E9000E1CFD9FFE2CFDAFF070EE12402E3E168D8
:102EA000E652E16EFA0EDBCF3DF0FB0EDBCF3EF0DB
:102EB000FA0E3DC0DBFFFB0E3EC0DBFFFC0EDBCF9E
:102EC000E9FFFD0EDBCFEAFF040EE926000EEA2241
:102ED000EECF1DF0EFCF1EF0010E1D26000E1E22BC
:102EE000040E1DC0DBFF050E1EC0DBFFD950040F12
:102EF000E96E000EDA20EA6EEE50ED1001E109D124
:102F0000FC0EDBCFE9FFFD0EDBCFEAFF0E0EE9265C
:102F1000000EEA22EECF1DF0EECF1EF0EECF1FF036
:102F2000EFCF20F01D501E101F10201001E1F1D036
:102F3000040EDBCF1DF0050E1E6A0F0E1D161D5070
:102F40001E1001E078D2FC0EDBCFE9FFFD0EDBCFD7
:102F5000EAFF0E0EE926000EEA22EE2AEE22EE220B
:102F6000EE22FC0EDBCFE9FFFD0EDBCFEAFF0A0EFF
:102F7000E926000EEA22EECF1DF0EECF1EF0EECFD6
:102F80001FF0EFCF20F01D501E101F1020101FE16A
:102F9000040EDBCF1DF0050EDBCF1EF0FC0EDBCFE9
:102FA000E9FFFD0EDBCFEAFFEE50EFCFEAFFE96E5F
:102FB000080EE926000EEA22EECF1FF0EFCF20F038
:102FC0001F501D5C20501E5801E235D2A2D0040EC5
:102FD000DBCF1FF0050EDBCF20F0040E0F0B05E05A
:102FE000D89020321F32E806FBE1FC0EDBCFE9FF70
:102FF000FD0EDBCFEAFFEE50EFCFEAFFE96E020EE7
:10300000E926000EEA22EF0400011F141D6E1E6A5D
:10301000E8501E1001E00FD2FC0EDBCFE9FFFD0EE1
:10302000DBCFEAFF0A0EE926000EEA22EECFE6FF2A
:10303000EECFE6FFEECFE6FFEFCFE6FFFC0EDBCFF5
:10304000E9FFFD0EDBCFEAFFEECFE6FFEFCFE6FFB5
:103050006CEC0AF01D6E060EE15C02E2E16AE552DC
:10306000E16E1D503BC0DEFF3CC0DEFF3DC0DEFF19
:103070003EC0DDFFDD52DD52D9CFE9FFDACFEAFFF6
:10308000D880010EEE54000EEE54000EEE54000EE9
:10309000EE5401E390D0D9CFE9FFDACFEAFFE86838
:1030A000EE180AE1E868EE1807E1E868EE1804E1B6
:1030B000E868EE1801E13FD1FC0EDBCFE9FFFD0E21
:1030C000DBCFEAFFEE50EFCFEAFFE96E160EE926FE
:1030D000000EEA22EECF1DF0EECF1EF0EECF1FF075
:1030E000EFCF20F0D9CFE9FFDACFEAFF1D50EE5C39
:1030F0001E50EE581F50EE582050EE5801E24ED1AF
:10310000D950FA0FE96EFF0EDA20EA6EEE50ED109C
:1031100002E1040ED3D1FC0EDBCFE9FFFD0EDBCFC5
:10312000EAFF0A0EE926000EEA22EECFE6FFEECF16
:10313000E6FFEECFE6FFEFCFE6FFFC0EDBCFE9FFC9
:10314000FD0EDBCFEAFFEECFE6FFEFCFE6FF26EC8A
:1031500011F01D6E060EE15C02E2E16AE552E16EDD
:103160001D503BC0DEFF3CC0DEFF3DC0DEFF3EC069
:10317000DDFFDD52DD52D9CFE9FFDACFEAFFEECF36
:103180001DF0EECF1EF0EECF1FF0EFCF20F01D5060
:103190001E101F10201002E1070E90D1D9CFE9FFB9
:1031A000DACFEAFF010EEE1808E1EE5006E1EE502C
:1031B00004E1EE5002E1020E81D1D9CFE9FFDACF6E
:1031C000EAFFE868EE180AE1E868EE1807E1E86847
:1031D000EE1804E1E868EE1801E1ADD0FC0EDBCF9B
:1031E000E9FFFD0EDBCFEAFFEECFE6FFEFCFE6FF14
:1031F000C3EC06F0E552E552000901E09CD0E66A16
:10320000020EE66E000EE66EE66AFC0EDBCFE9FF0C
:10321000FD0EDBCFEAFFEE50EFCFEAFFE96E320E94
:10322000E926000EEA22E9CF1DF0EACF1EF0E9CF31
:10323000E6FFEACFE6FFEEEC05F01F6E060EE15C5E
:1032400002E2E16AE552E16E1F50D9CFE9FFDACF21
:10325000EAFFEECFE6FFEECFE6FFEECFE6FFEFCFE1
:10326000E6FFFC0EDBCFE9FFFD0EDBCFEAFFEECF82
:10327000E6FFEFCFE6FFDCEC09F0216E060EE15C25
:1032800002E2E16AE552E16E21503BC01DF03CC014
:103290001EF03DC01FF03EC020F0FC0EDBCFE9FF6A
:1032A000FD0EDBCFEAFFEE50EFCFEAFFE96E2E0E08
:1032B000E926000EEA223BC0EEFF1EC0EEFF1FC053
:1032C000EEFF20C0EEFF060EDB6AFC0EDBCFE9FF4F
:1032D000FD0EDBCFEAFFEE50EFCFEAFFE96E020E04
:1032E000E926000EEA22EF50F36E060EDBCFF4FF64
:1032F000F350F45C37E2FC0EDBCFE9FFFD0EDBCFD1
:10330000EAFFEE50EFCFEAFFE96E040EE926000E69
:10331000EA22010EEF6EFC0EDBCFE9FFFD0EDBCFE4
:10332000EAFFEECFE6FFEFCFE6FFC3EC06F0E55293
:10333000E552000902E0010EC1D0FC0EDBCFE9FF2F
:10334000FD0EDBCFEAFFEE50EFCFEAFFE96E2E0E67
:10335000E926000EEA22EE2AEE22EE22EE22060EE8
:10336000DB2AB3D7060EDBCF1DF01E6A1F6A206A68
:10337000FC0EDBCFE9FFFD0EDBCFEAFFEE50EFCF17
:10338000EAFFE96E2E0EE926000EEA221D50EE5EDF
:103390001E50EE5A1F50EE5A2050EE5AFC0EDBCF54
:1033A000E9FFFD0EDBCFEAFF0A0EE926000EEA2256
:1033B000DFCFEEFF010EDBCFEEFF020EDBCFEEFF25
:1033C000030EDBCFEEFFD9CFE9FFDACFEAFFEECF76
:1033D000E6FFEECFE6FFEECFE6FFEFCFE6FFFC0E17
:1033E000DBCFE9FFFD0EDBCFEAFFEECFE6FFEFCF4D
:1033F000E6FFDCEC09F0216E060EE15C02E2E16A18
:10340000E552E16E21503CC01EF03DC01FF03EC0B1
:1034100020F0FC0EDBCFE9FFFD0EDBCFEAFF0E0E46
:10342000E926000EEA223BC0EEFF1EC0EEFF1FC0E1
:10343000EEFF20C0EEFFFC0EDBCFE9FFFD0EDBCF81
:10344000EAFF040EE926000EEA22040EDBCFEEFFAF
:10345000050EDBCFEDFFFC0EDBCFE9FFFD0EDBCF72
:10346000EAFFEE50EFCFEAFFE96E320EE926000EDA
:10347000EA22E9CF1FF0EACF20F0040EDBCF21F0E3
:10348000050E226A0F0E2116050ED890213622361F
:10349000E806FBE11F5021241D6E205022201E6EE5
:1034A000FC0EDBCFE9FFFD0EDBCFEAFF120EE926B3
:1034B000000EEA221DC0EEFF1EC0EDFF1D6E070EBE
:1034C000E15C02E2E16AE552E16E1D50E552E5CFB2
:1034D000DAFFE7CFD9FF1200D9CFE6FFDACFE6FF58
:1034E000E1CFD9FFE2CFDAFFE652E652E652000E14
:1034F000E66EE66AFC0EDBCFE6FFFD0EDBCFE6FFF5
:10350000D4EC14F0E552E552E552E552DF6EDF509F
:1035100075E1010EDB6A020EDB6AFC0EDBCFE9FF10
:10352000FD0EDBCFEAFF0E0EE926000EEA22EECFFB
:10353000E6FFEECFE6FFEECFE6FFEFCFE6FFFC0EB5
:10354000DBCFE9FFFD0EDBCFEAFFEECFE6FFEFCFEB
:10355000E6FF0BEC08F01D6E060EE15C02E2E16A8C
:10356000E552E16E1D50DF6EDF5048E1FC0EDBCF0F
:10357000E9FFFD0EDBCFEAFF120EE926000EEA227C
:10358000EE50EFCFEAFFE96EEF50E50810E0FC0ED9
:10359000DBCFE9FFFD0EDBCFEAFF120EE926000EBE
:1035A000EA22EE50EFCFEAFFE96EEF5012E1010E92
:1035B000DB2ADBCF1DF0020E01E3DB2ADBCF1EF09E
:1035C000FA0EDB501D1809E1FB0EDB501E1805E159
:1035D00015D0010EDB6A020EDB6A010EE66EE66AAA
:1035E000FC0EDBCFE6FFFD0EDBCFE6FF4DDCE55248
:1035F000E552E552E552DF6EDF508FE0040EDF5CEE
:1036000002E1070EDF6EDF50E552E552E552E5526A
:10361000E5CFDAFFE7CFD9FF1200D9CFE6FFDACF47
:10362000E6FFE1CFD9FFE2CFDAFFE652E652E652FB
:10363000E6521A0EE76EFA0EDBCFE9FFFB0EDBCF88
:10364000EAFFE750E926000EEA22EECF1DF0EFCFA9
:103650001EF01DC0DFFF010E1EC0DBFF020EDB6A85
:10366000030EDB6AFC0EDBCFE9FFFD0EDBCFEAFFCA
:10367000EF50030826E1140EE76EFA0EDBCFE9FFE8
:10368000FB0EDBCFEAFFE750E926000EEA22EECF81
:103690001DF0EFCF1EF01F6A206A100E1F0B07E00F
:1036A000D8901D361E361F362036E806F9E11D502B
:1036B000DE121E50DE121F50DE122050DD12DD52CF
:1036C000DD52DECF3BF0DECF3CF0DECF3DF0DDCF94
:1036D0003EF0DD52DD52040EE15C02E2E16AE552A9
:1036E000E16EE552E5CFDAFFE7CFD9FF1200D9CF7F
:1036F000E6FFDACFE6FFE1CFD9FFE2CFDAFF1A0E1D
:10370000E76EFC0EDBCFE9FFFD0EDBCFEAFFE750F3
:10371000E926000EEA22F80EDBCFEEFFF90EDBCF32
:10372000EDFFF80EDBCF1DF0F90EDBCF1EF0FA0E29
:10373000DBCF1FF0FB0EDBCF20F0100ED890203235
:103740001F321E321D32E806F9E1140EE76EFC0E40
:10375000DBCFE9FFFD0EDBCFEAFFE750E926000EE5
:10376000EA221DC0EEFF1EC0EDFFE552E5CFDAFFF5
:10377000E7CFD9FF1200D9CFE6FFDACFE6FFE1CFDE
:10378000D9FFE2CFDAFFE652E652E652E652000EE9
:10379000E66EE66AFC0EDBCFE6FFFD0EDBCFE6FF52
:1037A000D4EC14F0E552E552E552E552DF6EDF50FD
:1037B00002E0DF5092D0FC0EDBCFE9FFFD0EDBCF45
:1037C000EAFF0E0EE926000EEA22EECFE6FFEECF6C
:1037D000E6FFEECFE6FFEFCFE6FFFC0EDBCFE9FF23
:1037E000FD0EDBCFEAFFEECFE6FFEFCFE6FF0BECFF
:1037F00008F01D6E060EE15C02E2E16AE552E16E40
:103800001D50DF6EDF5068E1FC0EDBCFE9FFFD0EDF
:10381000DBCFEAFF120EE926000EEA22020EEECFFF
:10382000DBFF030EEDCFDBFF020EDBCFE9FF030E64
:10383000DBCFEAFF010EEFCFDBFFDB5003E1040E2D
:10384000DF6E4AD00B0EE76E020EDBCFE9FF030EF0
:10385000DBCFEAFFE750E926000EEA22EF50080B23
:1038600028E10B0EE66EE66AFC0EDBCFE9FFFD0EEB
:10387000DBCFEAFF140EE926000EEA22EECFE6FFC8
:10388000EFCFE6FF020EDBCFE6FF030EDBCFE6FF56
:103890001DEC06F01F6E060EE15C02E2E16AE552E5
:1038A000E16E1F50F3CF1DF0F4CF1EF0F350F41073
:1038B00013E0000EE66EE66AFC0EDBCFE6FFFD0EBF
:1038C000DBCFE6FF44EC17F0E552E552E552E55256
:1038D000DF6EDF5001E16FD7DF501D6E040EE15C3B
:1038E00002E2E16AE552E16E1D50E552E5CFDAFFF2
:1038F000E7CFD9FF1200D9CFE6FFDACFE6FFE1CF5D
:10390000D9FFE2CFDAFFE652E652E652E652E6523D
:10391000040EDF6EFC0EDBCFE9FFFD0EDBCFEAFF0E
:103920000E0EE926000EEA22EECF1DF0EECF1EF0BD
:10393000EECF1FF0EFCF20F01D501E101F102010F3
:1039400001E18BD0FC0EDBCFE9FFFD0EDBCFEAFF00
:103950000E0EE926000EEA22EECFE6FFEECFE6FFDE
:10396000EECFE6FFEFCFE6FFFC0EDBCFE9FFFD0E6B
:10397000DBCFEAFFEECFE6FFEFCFE6FF0BEC08F080
:103980001D6E060EE15C02E2E16AE552E16E1D5039
:10399000DF6EDF5062E1FC0EDBCFE9FFFD0EDBCF17
:1039A000EAFF120EE926000EEA22030EEECFDBFF3D
:1039B000040EEDCFDBFF030EDBCFE9FF040EDBCF00
:1039C000EAFF020EEFCFDBFFDB5003E1040EDF6EF8
:1039D00044D00B0EE76E030EDBCFE9FF040EDBCF06
:1039E000EAFFE750E926000EEA22EF503F0BE76EB0
:1039F000010EE7CFDBFF020EDB50E5081BE0020EF5
:103A0000DB502E0817E0010EDB500F0813E0010E0B
:103A1000DB50080802E0000E01D0010E1D6E1E6A88
:103A20001DBE1E68FA0EDB501D1804E1FB0EDB50B4
:103A30001E1813E0000EE66EE66AFC0EDBCFE6FF12
:103A4000FD0EDBCFE6FF44EC17F0E552E552E55200
:103A5000E552DF6EDF5001E15DD7DF500EE0FC0E76
:103A6000DBCFE9FFFD0EDBCFEAFF0E0EE926000EED
:103A7000EA22EE6AEE6AEE6AEE6ADF501D6E050E0D
:103A8000E15C02E2E16AE552E16E1D50E552E5CFEC
:103A9000DAFFE7CFD9FF1200D9CFE6FFDACFE6FF92
:103AA000E1CFD9FFE2CFDAFFE652010EE66EE66A19
:103AB000FC0EDBCFE6FFFD0EDBCFE6FF0DDDE552B2
:103AC000E552E552E552DF6EDF5001E080D0FC0E9A
:103AD000DBCFE9FFFD0EDBCFEAFF0E0EE926000E7D
:103AE000EA22EECFE6FFEECFE6FFEECFE6FFEFCF26
:103AF000E6FFFC0EDBCFE9FFFD0EDBCFEAFFEECFEA
:103B0000E6FFEFCFE6FF0BEC08F01D6E060EE15C62
:103B100002E2E16AE552E16E1D50DF6EDF5057E1CF
:103B2000200EE66EE66A000EE66EE66AFC0EDBCF5D
:103B3000E9FFFD0EDBCFEAFF120EE926000EEA22B6
:103B4000EECFE6FFEFCFE6FFEEEC05F01D6E060EC2
:103B5000E15C02E2E16AE552E16E1D500B0EE66E99
:103B6000E66AFC0EDBCFE9FFFD0EDBCFEAFF140EA9
:103B7000E926000EEA22EECFE6FFEFCFE6FFFC0ECD
:103B8000DBCFE9FFFD0EDBCFEAFF120EE926000EC8
:103B9000EA22EECFE6FFEFCFE6FF6CEC05F01D6EFC
:103BA000060EE15C02E2E16AE552E16E1D50FC0E98
:103BB000DBCFE9FFFD0EDBCFEAFFEE50EFCFEAFFF0
:103BC000E96E040EE926000EEA22010EEF6EDF50C8
:103BD000E552E552E5CFDAFFE7CFD9FF1200D9CFA2
:103BE000E6FFDACFE6FFE1CFD9FFE2CFDAFF0D0E35
:103BF000E12402E3E168E652E16EFA0EDBCFE9FF71
:103C0000FB0EDBCFEAFF0B0EEECFDBFF0C0EEDCF92
:103C1000DBFF0B0EDBCFE9FF0C0EDBCFEAFFEF5033
:103C20002F0809E00B0EDBCFE9FF0C0EDBCFEAFF1C
:103C3000EF505C0806E10B0EDB2A0C0EEAE3DB2AF0
:103C4000E8D7FC0EDBCFE9FFFD0EDBCFEAFF140E59
:103C5000E926000EEA22030EEECFDBFF040EEDCFC5
:103C6000DBFF0B0EE66EE66A200EE66EE66A030EDA
:103C7000DBCFE6FF040EDBCFE6FFEEEC05F01D6EBA
:103C8000060EE15C02E2E16AE552E16E1D50000EB3
:103C9000DF6EE66ED950090FE96E000EDA20EA6E8B
:103CA000E552E750EE6EED6AE66ED950070FE96E09
:103CB000000EDA20EA6EE552E750EE6EED6A080E6D
:103CC000F36E050EF3CFDBFF060EDB6A070EDBCFCC
:103CD0001DF0DB2A080EDBCF1EF001E3DB2A0B0E02
:103CE000DB501D24E96E0C0EDB501E20EA6E010E27
:103CF000EFCFDBFFDB50200801E39CD0010EDB504F
:103D00002F0801E197D0010EDB505C0801E192D051
:103D1000010EDB502E0811E0090EDBCF1DF00A0E5C
:103D2000DBCF1EF0050EDBCF1FF0060EDBCF20F041
:103D30001F501D5C20501E5825E3D950050FE96E19
:103D4000000EDA20EA6E080EEE1801E09FD0ED506A
:103D500001E09CD0010EDB502E0801E097D0080E48
:103D6000F36E090EF3CFDBFF0A0EDB6A0B0EF36E68
:103D7000050EF3CFDBFF060EDB6A040EDF02F3CF86
:103D8000DFFFA4D7800EF36E010EDBCFF4FFF350FC
:103D9000F45C04E3000EDF80DF8278D0010EDBCF1D
:103DA000E6FFE66A3C0EE66EE10EE66E82EC06F099
:103DB000E552E552E552E552F350F41067E1410E49
:103DC000F36E010EDBCFF4FFF350F45C06E3010E5B
:103DD000DB505A0802E3DF8218D0610EF36E010E49
:103DE000DBCFF4FFF350F45C10E3010EDB507A08F4
:103DF0000CE3000EDF80200E1D6E010EDBCFE7FF0F
:103E00001D50E75E010EE7CFDBFF090EDBCF1DF093
:103E1000DB2A0A0EDBCF1EF001E3DB2A030EDB50A8
:103E20001D24E96E040EDB501E20EA6E010EDBCF6E
:103E3000EFFF4CD7070EDBCF1FF0080EDBCF20F0D3
:103E40000B0EDB501F241D6E0C0EDB5020201E6E4F
:103E5000FA0EDBCFE9FFFB0EDBCFEAFF1DC0EEFF62
:103E60001EC0EDFF010EDB50200802E3040E01D05E
:103E7000000EE76E010EE7CFDBFFD950090FE96EA8
:103E8000000EDA20EA6EEE50ED1002E1060E3CD094
:103E9000030EDBCFE9FF040EDBCFEAFFEF50E508AE
:103EA00008E1030EDBCFE9FF040EDBCFEAFF050ECE
:103EB000EF6ED950050FE96E000EDA20EA6E080E9B
:103EC000EE1806E1ED5004E1040EDF02F3CFDFFF50
:103ED000030EDF14010802E1010EDB880C0EDF1473
:103EE000040802E1010EDB860B0EE76E030EDBCF4A
:103EF000E9FF040EDBCFEAFFE750E926000EEA22D5
:103F0000010EDBCFEFFF000E1D6E0D0EE15C02E235
:103F1000E16AE552E16E1D50E552E5CFDAFFE7CFE9
:103F2000D9FF1200D9CFE6FFDACFE6FFE1CFD9FF04
:103F3000E2CFDAFF080EE12402E3E168E652E16E27
:103F4000FA0EDBCFE9FFFB0EDBCFEAFF090EE92615
:103F5000000EEA22050EE9CFDBFF060EEACFDBFFFB
:103F6000FC0EDBCFE9FFFD0EDBCFEAFF0E0EE926EC
:103F7000000EEA22EECF1DF0EECF1EF0EECF1FF0C6
:103F8000EFCF20F01D501E101F10201001E118D19E
:103F9000FC0EDBCFE9FFFD0EDBCFEAFF120EE926B8
:103FA000000EEA22030EEECFDBFF040EEDCFDBFFA7
:103FB0000C0EE76E030EDBCFE9FF040EDBCFEAFF4A
:103FC000E750E926000EEA22020EEFCFDBFFDE6AA1
:103FD000DD6ADECF1DF0DDCF1EF0080E1D5C000E89
:103FE0001E582CE2030EDBCF1DF0040EDBCF1EF0BB
:103FF000DE501D24E96EDD501E20EA6E070EEFCF65
:10400000DBFFDB5020081AE0070EDB50050805E156
:10401000E50EF36E070EF3CFDBFF050EDBCFE9FFF6
:10402000DB2A060EDBCFEAFF01E3DB2A070EDBCF3C
:10403000EFFFDF2A010ECDE3DB2ACBD7080EE76EB8
:10404000030EDBCFE9FF040EDBCFEAFFE750E926E2
:10405000000EEA22EF5020083AE0050EDBCFE9FF20
:10406000DB2A060EDBCFEAFF01E3DB2A2E0EEF6E22
:10407000080EDE6EDD6ADECF1DF0DDCF1EF00B0E0A
:104080001D5C000E1E5823E2030EDBCF1DF0040E54
:10409000DBCF1EF0DE501D24E96EDD501E20EA6EDF
:1040A000070EEFCFDBFFDB50200811E0050EDBCF62
:1040B000E9FFDB2A060EDBCFEAFF01E3DB2A070E6E
:1040C000DBCFEFFFDF2A010ED6E3DB2AD4D70B0EBE
:1040D000E76E030EDBCFE9FF040EDBCFEAFFE7500C
:1040E000E926000EEA22EF50E66EFA0EDBCFE9FF7A
:1040F000FB0EDBCFEAFF080EE926000EEA22E552AE
:10410000E750EF6E1C0EE76E030EDBCFE9FF040EE7
:10411000DBCFEAFFE750E926000EEA22EECF1DF0E2
:10412000EECF1EF0EECF1FF0EFCF20F0FA0EDBCF78
:10413000E9FFFB0EDBCFEAFF1DC0EEFF1EC0EEFF66
:104140001FC0EEFF20C0EEFF180EE76E030EDBCFA0
:10415000E9FF040EDBCFEAFFE750E926000EEA2272
:10416000EECF1DF0EFCF1EF0FA0EDBCFE9FFFB0E16
:10417000DBCFEAFF040EE926000EEA221DC0EEFFA7
:104180001EC0EDFF160EE76E030EDBCFE9FF040E37
:10419000DBCFEAFFE750E926000EEA22EECF1DF062
:1041A000EFCF1EF0FA0EDBCFE9FFFB0EDBCFEAFF0D
:1041B000060EE926000EEA221DC0EEFF1EC0EDFF2E
:1041C000050EDBCFE9FF060EDBCFEAFFEF6A080E34
:1041D000E15C02E2E16AE552E16EE552E5CFDAFF29
:1041E000E7CFD9FF1200D9CFE6FFDACFE6FFE1CF64
:1041F000D9FFE2CFDAFFE652E652E652E652FA0E75
:10420000DBCFE9FFFB0EDBCFEAFFEF502F0809E021
:10421000FA0EDBCFE9FFFB0EDBCFEAFFEF505C08C5
:1042200005E1FA0EDB2AFB0E01E3DB2AFC0EDBCFF5
:10423000E9FFFD0EDBCFEAFF060EE926000EEA22BB
:10424000EE6AEE6AEE6AEE6AFA0EDBCFE9FFFB0E6B
:10425000DBCFEAFFEFCF1DF01E6A1DBE1E68200EE9
:104260001D5C000E1E581BE2000EE66EE66AFC0E98
:10427000DBCFE6FFFD0EDBCFE6FFD4EC14F0E5521A
:10428000E552E552E552DF6EFC0EDBCFE9FFFD0E95
:10429000DBCFEAFF120EEB6A130EEB6A94D0D95013
:1042A000FA0FE66EFF0EDA20E66EFC0EDBCFE6FFBD
:1042B000FD0EDBCFE6FF93DCE552E552E552E55219
:1042C000DF6EDF5001E07FD0FC0EDBCFE6FFFD0E9E
:1042D000DBCFE6FFBBEC1BF0E552E552DF6EFC0ED8
:1042E000DBCFE9FFFD0EDBCFEAFF140EE926000E5F
:1042F000EA22EE50EFCFEAFFE96E0B0EE926000E40
:10430000EA22030EEFCFDBFFDF5007E0040EDF5C95
:104310005AE1030EDBB457D022D0030EDBB453D0E6
:10432000FC0EDBCFE9FFFD0EDBCFEAFF120EE92624
:10433000000EEA22010EEECFDBFF020EEDCFDBFF17
:104340000B0EE76E010EDBCFE9FF020EDBCFEAFFBB
:10435000E750E926000EEA22EF50100B03E1050EAC
:10436000DF6E31D0010EDBCFE6FF020EDBCFE6FFC2
:10437000FC0EDBCFE9FFFD0EDBCFEAFFEECFE6FF61
:10438000EFCFE6FF0DEC1BF0E552E552E552E552AA
:104390003BC01DF03CC01EF03DC01FF03EC020F0F1
:1043A000FC0EDBCFE9FFFD0EDBCFEAFF060EE926B0
:1043B000000EEA223BC0EEFF1EC0EEFF1FC0EEFF64
:1043C00020C0EEFF6CD7DF501D6E040EE15C02E2F0
:1043D000E16AE552E16E1D50E552E5CFDAFFE7CF25
:1043E000D9FF1200D9CFE6FFDACFE6FFE1CFD9FF40
:1043F000E2CFDAFF010EE66ED950F80FE96EFF0E3C
:10440000DA20EA6EEECFE6FFEECFE6FFEECFE6FF74
:10441000EFCFE6FFFC0EDBCFE9FFFD0EDBCFEAFFBF
:10442000320EE926000EEA22E9CF1DF0EACF1EF097
:10443000E9CFE6FFEACFE6FFFC0EDBCFE9FFFD0E9A
:10444000DBCFEAFFEE52EF50E66EF5EC5DF01F6E4B
:10445000080EE15C02E2E16AE552E16E1F500009DC
:1044600002E0030E63D0FC0EDBCFE9FFFD0EDBCFD5
:10447000EAFF320EE926000EEA22FE0EE926010EC0
:10448000EA22550EEE1802E1AA0EED1802E0020E25
:104490004DD01D681E681F68206AFC0EDBCFE9FF47
:1044A000FD0EDBCFEAFF320EE926000EEA22360EC1
:1044B000E926000EEA22EE501D16EE501E16EE50B2
:1044C0001F16EE502016460E1D1808E1410E1E184C
:1044D00005E1540E1F1802E1205025E01D681E68FA
:1044E0001F68206AFC0EDBCFE9FFFD0EDBCFEAFF81
:1044F000320EE926000EEA22520EE926000EEA22CA
:10450000EE501D16EE501E16EE501F16EE502016E1
:10451000460E1D180AE1410E1E1807E1540E1F1821
:1045200004E1205002E1000E01D0010EE552E5CF7A
:10453000DAFFE7CFD9FF1200D9CFE6FFDACFE6FFE7
:10454000E1CFD9FFE2CFDAFF260EE12402E3E168F2
:10455000E652E16EFC0EDBCFE9FFFD0EDBCFEAFF9A
:10456000220EEECFDBFF230EEDCFDBFF220EDBCFE3
:10457000E9FF230EDBCFEAFFEF50D00FE66ED950F4
:10458000050FE96E000EDA20EA6EE552E750EE6E96
:10459000ED6AD950050FE96E000EDA20EA6E090EB9
:1045A000D880EE54000EED5426E3010EE76E220E85
:1045B000DBCFE9FF230EDBCFEAFFE750E926000E51
:1045C000EA22EF503A0817E1D950220FE96E000EA7
:1045D000DA20EA6E020EEE26000EED22FC0EDBCF94
:1045E000E9FFFD0EDBCFEAFF220EDBCFEEFF230E4D
:1045F000DBCFEDFF04D0050EDB6A060EDB6AFA0E98
:10460000DBCFE9FFFB0EDBCFEAFFEE6AED6A050EBA
:10461000DBCF1DF0060EDBCF1EF0010E1D5C000E81
:104620001E5803E30B0EC1EF29F0050EDBCFE9FFA7
:10463000060EDBCFEAFF010ED890E936EA36E8062F
:10464000FBE1C60EE926000EEA22240EEECFDBFFC8
:10465000250EEDCFDBFFD950240FE96E000EDA20D6
:10466000EA6EEE50ED1003E10C0EC1EF29F0FA0EE8
:10467000DBCFE9FFFB0EDBCFEAFF240EDBCFEEFF43
:10468000250EDBCFEDFF240EDBCFE9FF250EDBCFC0
:10469000EAFFEF501CE0240EDBCFE9FF250EDBCF55
:1046A000EAFFEE52EF50E66EE0EC5DF0E552E76EA9
:1046B000070EE7CFDBFFDBB00AD0F90EDB5004E0DA
:1046C000070EDB50040B30E1000EC1EF29F0240E81
:1046D000DBCFE9FF250EDBCFEAFFEF6A240EDBCF4D
:1046E000E9FF250EDBCFEAFFEE52050EDBCFEFFF31
:1046F000240EDBCFE9FF250EDBCFEAFFEE52EF50B1
:10470000E66E9FEC5CF0E552E76E070EE7CFDBFF4D
:10471000DBA003D0030EC1EF29F0F90EDB5007E058
:10472000070EDB50040B03E00A0EC1EF29F0080E60
:10473000DB6A090EDB6A0A0EDB6A0B0EDB6AE66ACD
:10474000E66AE66AE66A240EDBCFE6FF250EDBCFDB
:10475000E6FF48DE1D6E060EE15C02E2E16AE5520C
:10476000E16E1D50DF6EDF046CE1020EDB6ADB5090
:1047700002E0020EDB06240EDBCFE9FF250EDBCFC5
:10478000EAFF320EE926000EEA22E9CF1FF0EACF57
:1047900020F0020EDB50100DF350226ABE0F216E86
:1047A000010E2222E95021241D6EEA5022201E6EA5
:1047B000030E1DC0DBFF040E1EC0DBFFE76E030E01
:1047C000DBCFE9FF040EDBCFEAFFE750E926000E5E
:1047D000EA22EF5036E0080EE76E030EDBCFE9FF6A
:1047E000040EDBCFEAFFE750E926000EEA22080EAE
:1047F000EECFDBFF090EEECFDBFF0A0EEECFDBFFC5
:104800000B0EEECFDBFFD950080FE96E000EDA2059
:10481000EA6EEECFE6FFEECFE6FFEECFE6FFEFCF9C
:10482000E6FF240EDBCFE6FF250EDBCFE6FFDADD69
:104830001D6E060EE15C02E2E16AE552E16E1D507A
:10484000DF6E030EDF5C03E1010EC1EF29F0DF50E4
:1048500002E05BEF28F0240EDBCFE9FF250EDBCF73
:10486000EAFF320EE926000EEA220B0EE926000EC0
:10487000EA22EE5002E05BEF28F0020EED1802E0B3
:104880005BEF28F0240EDBCFE9FF250EDBCFEAFF3C
:10489000320EE926000EEA22160EE926000EEA2262
:1048A000EECF1DF0EFCF1EF00C0E1DC0DBFF0D0E86
:1048B0001EC0DBFF0E0EDB6A0F0EDB6A0C0EDBCFB9
:1048C0001DF00D0EDBCF1EF00E0EDBCF1FF00F0E16
:1048D000DBCF20F01D501E101F1020101AE1240EF7
:1048E000DBCFE9FF250EDBCFEAFF320EE926000E13
:1048F000EA22240EE926000EEA220C0EEECFDBFFA0
:104900000D0EEECFDBFF0E0EEECFDBFF0F0EEECF68
:10491000DBFF240EDBCFE9FF250EDBCFEAFF1A0E0B
:10492000E926000EEA220C0EDBCFEEFF0D0EDBCFE8
:10493000EEFF0E0EDBCFEEFF0F0EDBCFEEFF240EF1
:10494000DBCFE9FF250EDBCFEAFF320EE926000EB2
:10495000EA22100EE926000EEA22010EEFCFDBFF5D
:10496000240EDBCFE9FF250EDBCFEAFF030EE9269D
:10497000000EEA22010EDBCFEFFFDB0405E0010EA3
:10498000DB50020801E097D3010EDBCF1DF01E6A59
:104990001F6A206AD9500C0FE96E000EDA20EA6E09
:1049A0001DC040F01EC041F01FC042F020C043F0C7
:1049B000EECF3BF0EECF3CF0EECF3DF0EFCF3EF050
:1049C000CEEC6FF03AC0EDFF39C0EDFF38C0EDFF1F
:1049D00037C0EFFF240EDBCFE9FF250EDBCFEAFF68
:1049E000320EE926000EEA220D0EE926000EEA221A
:1049F000010EEFCFDBFF240EDBCFE9FF250EDBCF6F
:104A0000EAFF020EE926000EEA22010EDBCFEFFFDD
:104A1000DB5001E150D3010EDBCFE6FFDB04E552B2
:104A2000E71401E048D3240EDBCFE9FF250EDBCFEE
:104A3000EAFF320EE926000EEA22110EE926000EE8
:104A4000EA22EECF1DF0EFCF1EF0240EDBCFE9FF00
:104A5000250EDBCFEAFF080EE926000EEA221DC074
:104A6000EEFF1EC0EDFF240EDBCFE9FF250EDBCFEE
:104A7000EAFF080EE926000EEA22EECF1DF0000143
:104A80001E6A0F0E1D161D501E1001E014D3240EB9
:104A9000DBCFE9FF250EDBCFEAFF320EE926000E61
:104AA000EA22130EE926000EEA22EECF1DF0EFCF28
:104AB0001EF0100E1DC0DBFF110E1EC0DBFF120E1C
:104AC000DB6A130EDB6A100EDBCF1DF0110EDBCF9D
:104AD0001EF0120EDBCF1FF0130EDBCF20F01D50A7
:104AE0001E101F1020101AE1240EDBCFE9FF250E47
:104AF000DBCFEAFF320EE926000EEA22200EE9267D
:104B0000000EEA22100EEECFDBFF110EEECFDBFF20
:104B1000120EEECFDBFF130EEECFDBFF240EDBCF4A
:104B2000E9FF250EDBCFEAFF320EE926000EEA226E
:104B30000E0EE926000EEA22200EEECFDBFF210E3C
:104B4000EDCFDBFFD950200FE96E000EDA20EA6EC0
:104B5000EE50ED1001E1AFD2200EDBCF21F0210E9F
:104B6000DBCF22F0236A246AD9500C0FE96E000EC5
:104B7000DA20EA6E2150EE241D6E2250EE201E6EC9
:104B80002350EE201F6E2450EE20206E240EDBCF2B
:104B9000E9FF250EDBCFEAFF080EE926000EEA2228
:104BA000EECF25F0EFCF26F0040E0F0B05E0D890E6
:104BB00026322532E806FBE1276A286A25501D26A1
:104BC00026501E2227501F2228502022140E1DC0BE
:104BD000DBFF150E1EC0DBFF160E1FC0DBFF170E1E
:104BE00020C0DBFF140EDBCF1DF0150EDBCF1EF057
:104BF000160EDBCF1FF0170EDBCF20F0D950100FB1
:104C0000E96E000EDA20EA6E1D50EE5C1E50EE5882
:104C10001F50EE582050EE5801E24DD2240EDBCF4B
:104C2000E9FF250EDBCFEAFF020EE926000EEA229D
:104C3000EFCF25F0266A276A286A100EDBCF21F015
:104C4000110EDBCF22F0120EDBCF23F0130EDBCFE1
:104C500024F0D950140FE96E000EDA20EA6EEE50FF
:104C6000215C1D6EEE5022581E6EEE5023581F6EB2
:104C7000EE502458206E1DC03BF01EC03CF01FC0FB
:104C80003DF03E6E25C040F026C041F027C042F006
:104C900028C043F02BEC70F0180E3BC0DBFF190E60
:104CA0003CC0DBFF1A0E3DC0DBFF1B0E3EC0DBFF2E
:104CB000180EDBCF1DF0190EDBCF1EF01A0EDBCF66
:104CC0001FF01B0EDBCF20F01D501E101F102010F8
:104CD00001E1F1D1010EDF6ED950180FE96E000E1F
:104CE000DA20EA6EF60EEE5C0F0EEE58000EEE586D
:104CF000000EEE5802E3020EDF6ED950180FE96E77
:104D0000000EDA20EA6EF60EEE5CFF0EEE58000E94
:104D1000EE58000EEE5802E3030EDF6E020E1D6E1B
:104D20001E6A1F6A206AD950180FE96E000EDA2039
:104D3000EA6EEE501D26EE501E22EE501F22EE505F
:104D40002022240EDBCFE9FF250EDBCFEAFF160E73
:104D5000E926000EEA221DC0EEFF1EC0EEFF1FC0B6
:104D6000EEFF20C0EEFF240EDBCFE9FF250EDBCFE8
:104D7000EAFF1E0EE926000EEA22080EDBCFEEFF48
:104D8000090EDBCFEEFF0A0EDBCFEEFF0B0EDBCF03
:104D9000EEFF200EDBCF1DF0210EDBCF1EF01F6AD1
:104DA000206AD950080FE96E000EDA20EA6EEE5044
:104DB0001D26EE501E22EE501F22EE502022240E01
:104DC000DBCFE9FF250EDBCFEAFF220EE926000E3E
:104DD000EA221DC0EEFF1EC0EEFF1FC0EEFF20C086
:104DE000EEFF140EDBCF1DF0150EDBCF1EF0160EFE
:104DF000DBCF1FF0170EDBCF20F0D950080FE96E84
:104E0000000EDA20EA6EEE501D26EE501E22EE5005
:104E10001F22EE502022240EDBCFE9FF250EDBCF30
:104E2000EAFF2A0EE926000EEA221DC0EEFF1EC090
:104E3000EEFF1FC0EEFF20C0EEFF030EDF5C5CE163
:104E4000240EDBCFE9FF250EDBCFEAFF080EE926B3
:104E5000000EEA22EE50ED1001E02DD1240EDBCF42
:104E6000E9FF250EDBCFEAFF320EE926000EEA222B
:104E70002C0EE926000EEA22EECF1DF0EECF1EF03A
:104E8000EECF1FF0EFCF20F0240EDBCFE9FF250E91
:104E9000DBCFEAFF260EE926000EEA221DC0EEFF58
:104EA0001EC0EEFF1FC0EEFF20C0EEFF240EDBCFC2
:104EB000E9FF250EDBCFEAFF160EE926000EEA22F7
:104EC000EECF3BF0EECF3CF0EECF3DF0EFCF3EF03B
:104ED000040E406E416A426A436ACEEC6FF01C0ECB
:104EE00037C0DBFF1D0E38C0DBFF1E0E39C0DBFFF5
:104EF0001F0E3AC0DBFFB1D0240EDBCFE9FF250E39
:104F0000DBCFEAFF080EE926000EEA22EE50ED1094
:104F100001E1D1D00C0EDBCF1DF00D0EDBCF1EF06A
:104F20000E0EDBCF1FF00F0EDBCF20F0240EDBCFF9
:104F3000E9FF250EDBCFEAFF220EE926000EEA226A
:104F4000EE501D26EE501E22EE501F22EE50202263
:104F5000240EDBCFE9FF250EDBCFEAFF260EE92684
:104F6000000EEA221DC0EEFF1EC0EEFF1FC0EEFFC6
:104F700020C0EEFF020EDF5C18E1240EDBCFE9FF5C
:104F8000250EDBCFEAFF160EE926000EEA22EECF51
:104F90001DF0EECF1EF0EECF1FF0EFCF20F0D89037
:104FA0001D361E361F3620364CD0010E216E226A69
:104FB000236A246A240EDBCFE9FF250EDBCFEAFF4C
:104FC000160EE926000EEA22EE502116EE502216A9
:104FD000EE502316EE502416240EDBCFE9FF250EEB
:104FE000DBCFEAFF160EE926000EEA22EECF3BF0F9
:104FF000EECF3CF0EECF3DF0EFCF3EF0030E406E33
:10500000416A426A436ACEEC6FF037C03BF038C069
:105010003CF039C03DF03AC03EF0020E406E416AAD
:10502000426A436A2BEC70F03B50000121241D6E54
:105030003C5022201E6E3D5023201F6E3E502420E7
:10504000206E1C0E1DC0DBFF1D0E1EC0DBFF1E0EE2
:105050001FC0DBFF1F0E20C0DBFF1C0EDBCF1DF0CF
:105060001D0EDBCF1EF01E0EDBCF1FF01F0EDBCFA1
:1050700020F0FF0E1D26010E1E22000E1F222022F0
:10508000090ED89020321F321E321D32E806F9E197
:10509000240EDBCFE9FF250EDBCFEAFF1A0EE9264F
:1050A000000EEA221D50EE5C1E50EE581F50EE58C6
:1050B0002050EE5802E20D0E64D1240EDBCFE9FF42
:1050C000250EDBCFEAFF0E0EE926000EEA22EE687F
:1050D000EE68EE68EE68240EDBCFE9FF250EDBCF2D
:1050E000EAFF0A0EE926000EEA22EE6AEE6AEE6A8E
:1050F000EE6A030EDF5C01E011D1240EDBCFE9FF85
:10510000250EDBCFEAFF050EE926000EEA22EF6A44
:10511000240EDBCFE9FF250EDBCFEAFF320EE926B6
:10512000000EEA22300EE926000EEA22EECF1DF034
:10513000EFCF1EF01F6A206AD950080FE96E000EEB
:10514000DA20EA6EEE501D26EE501E22EE501F228F
:10515000EE502022240EDBCFE9FF250EDBCFEAFF45
:10516000120EE926000EEA221DC0EEFF1EC0EEFF61
:105170001FC0EEFF20C0EEFF010EE66E240EDBCF57
:10518000E9FF250EDBCFEAFF120EE926000EEA2228
:10519000EECFE6FFEECFE6FFEECFE6FFEFCFE6FF86
:1051A000240EDBCFE9FF250EDBCFEAFF320EE92626
:1051B000000EEA22E9CF1DF0EACF1EF0E9CFE6FFAC
:1051C000EACFE6FF240EDBCFE9FF250EDBCFEAFFB7
:1051D000EE52EF50E66EF5EC5DF01F6E080EE15CEE
:1051E00002E2E16AE552E16E1F50000901E096D04B
:1051F000240EDBCFE9FF250EDBCFEAFF320EE926D6
:10520000000EEA22FE0EE926010EEA22550EEE18E5
:1052100001E084D0AA0EED1801E080D0240EDBCF8F
:10522000E9FF250EDBCFEAFF320EE926000EEA2267
:10523000520EEE1873E1520EEE1870E1610EEE1888
:105240006DE1410EEE186AE1240EDBCFE9FF250E79
:10525000DBCFEAFF320EE926000EEA22E40EE92651
:10526000010EEA22720EEE1859E1720EEE1856E1A6
:10527000410EEE1853E1610EEE1850E1240EDBCF23
:10528000E9FF250EDBCFEAFF320EE926000EEA2207
:10529000EC0EE926010EEA22EECF1DF0EECF1EF055
:1052A000EECF1FF0EFCF20F0240EDBCFE9FF250E6D
:1052B000DBCFEAFF0A0EE926000EEA221DC0EEFF50
:1052C0001EC0EEFF1FC0EEFF20C0EEFF240EDBCF9E
:1052D000E9FF250EDBCFEAFF320EE926000EEA22B7
:1052E000E80EE926010EEA22EECF1DF0EECF1EF009
:1052F000EECF1FF0EFCF20F0240EDBCFE9FF250E1D
:10530000DBCFEAFF0E0EE926000EEA221DC0EEFFFB
:105310001EC0EEFF1FC0EEFF20C0EEFF240EDBCF4D
:10532000E9FF250EDBCFEAFFDFCFEFFF0001C82B3F
:10533000000EC923240EDBCFE9FF250EDBCFEAFFE9
:10534000060EE926000EEA22C8C0EEFFC9C0EDFF36
:10535000240EDBCFE9FF250EDBCFEAFF2E0EE92678
:10536000000EEA22EE6AEE6AEE6AEE6A240EDBCFE7
:10537000E9FF250EDBCFEAFF040EE926000EEA2244
:10538000EF6A1D6E260EE15C02E2E16AE552E16E13
:105390001D50E552E5CFDAFFE7CFD9FF1200D9CF94
:1053A000E6FFDACFE6FFE1CFD9FFE2CFDAFFE65240
:1053B000E652FC0EDBCFDEFFDBCFDDFFD9CFE9FF0E
:1053C000DACFEAFFEE50ED1033E0DECFE9FFDDCFBC
:1053D000EAFFEE50ED102CE0DECFE9FFDDCFEAFF73
:1053E000EE50EFCFEAFFE96EEF5022E0DECFE9FFAB
:1053F000DDCFEAFFEE50EFCFEAFFE96E060EE926B9
:10540000000EEA22EECF1DF0EFCF1EF0DECFE9FF57
:10541000DDCFEAFF020EE926000EEA22EECF1FF0F2
:10542000EFCF20F01F501D1802E120501E1802E09F
:10543000090E13D0DECFE9FFDDCFEAFFEE50EFCF4C
:10544000EAFFE96EEE52EF50E66EE0EC5DF0E552F9
:10545000010B02E0030E01D0000EE552E552E552C9
:10546000E5CFDAFFE7CFD9FF1200D9CFE6FFDACFD9
:10547000E6FFE1CFD9FFE2CFDAFFE652E652010EB6
:10548000F36EFD0EDBCFF4FFF350F45C02E30B0E82
:105490003BD0FD0EEA6ADB34FE0BEA36E96EC60E3F
:1054A000E926000EEA22EECFDEFFEDCFDDFFD9CFF9
:1054B000E9FFDACFEAFFEE50ED1005E0DECFE9FFBD
:1054C000DDCFEAFFEF6AD950FB0FE96EFF0EDA205D
:1054D000EA6EEE50ED1007E0FB0EDBCFE9FFFC0EAD
:1054E000DBCFEAFFEF6AFD0EEA6ADB34FE0BEA3639
:1054F000E96EC60EE926000EEA22FB0EDBCFEEFFB8
:10550000FC0EDBCFEDFF000EE552E552E552E5CF94
:10551000DAFFE7CFD9FF1200D9CFE6FFDACFE6FFF7
:10552000E1CFD9FFE2CFDAFF2D0EE12402E3E168FB
:10553000E652E16ED950FC0FE96EFF0EDA20EA6EFA
:10554000EE50ED1002E1090EBFD2FC0EDBCFE9FFF9
:10555000FD0EDBCFEAFFEE6AED6AF90EDB9ADB9C0B
:10556000DB9EDB50FE0BE66ED950010FE66E000E9F
:10557000DA20E66ED950FA0FE66EFF0EDA20E66EFC
:105580009CEC22F01D6E050EE15C02E2E16AE55240
:10559000E16E1D50DF6EDF5001E095D2D950190F3A
:1055A0001D6E000EDA201E6E150E1DC0DBFF160EDE
:1055B0001EC0DBFFFA0EDBCFE6FFFB0EDBCFE6FF04
:1055C000D950010FE66E000EDA20E66EF3EC20F003
:1055D000E552E552E552E552DF6E130EDBCF3DF0AA
:1055E000140EDBCF3EF0170E3DC0DBFF180E3EC0A1
:1055F000DBFFDF500BE1D950170FE96E000EDA2008
:10560000EA6EEE50ED1002E1060EDF6EF90EDB5091
:105610001C0B01E149D1DF501DE0040EDF5C0BE102
:10562000D950010FE66E000EDA20E66E4CEC1DF04C
:10563000E552E552DF6EF90EDB86130EDBCF3DF04F
:10564000140EDBCF3EF0170E3DC0DBFF180E3EC040
:10565000DBFF16D00B0EE76E170EDBCFE9FF180E3F
:10566000DBCFEAFFE750E926000EEA22EF50110BEC
:1056700002E0070E04D0F90EDBA402D0080EDF6EA4
:10568000DF5001E039D1F90EDB50080B01E134D1D4
:105690007AEC68F0250E3BC0DBFF260E3CC0DBFF3A
:1056A000270E3DC0DBFF280E3EC0DBFF0E0EE76E6F
:1056B000170EDBCFE9FF180EDBCFEAFFE750E92634
:1056C000000EEA22250EDBCFEEFF260EDBCFEEFF2B
:1056D000270EDBCFEEFF280EDBCFEEFF0B0EE76EC3
:1056E000170EDBCFE9FF180EDBCFEAFFE750E92604
:1056F000000EEA22EF6A1C0EE76E170EDBCFE9FF01
:10570000180EDBCFEAFFE750E926000EEA22EE6A28
:10571000EE6AEE6AEE6A170EDBCFE6FF180EDBCFFD
:10572000E6FF010EDBCFE6FF020EDBCFE6FF0DEC5E
:105730001BF0E552E552E552E552290E3BC0DBFF76
:105740002A0E3CC0DBFF2B0E3DC0DBFF2C0E3EC003
:10575000DBFFE66AE66AE66AE66A170EDBCFE6FF7B
:10576000180EDBCFE6FF77EC1BF01D6E060EE15C3A
:1057700002E2E16AE552E16E1D50010EDBCFE9FF66
:10578000020EDBCFEAFF040EE926000EEA22010E2C
:10579000EF6E290EDBCF1DF02A0EDBCF1EF02B0E95
:1057A000DBCF1FF02C0EDBCF20F01D501E101F1082
:1057B000201001E1A1D0010EDBCFE9FF020EDBCF0B
:1057C000EAFF2E0EE926000EEA22250EEECFDBFFC1
:1057D000260EEECFDBFF270EEECFDBFF280EEECF3F
:1057E000DBFFD950290FE96E000EDA20EA6EEECF0A
:1057F000E6FFEECFE6FFEECFE6FFEFCFE6FF010ECE
:10580000DBCFE6FF020EDBCFE6FFF1EC0FF01D6E03
:10581000060EE15C02E2E16AE552E16E1D50DF6EC8
:10582000DF506AE1290EDBCF1DF02A0EDBCF1EF020
:105830002B0EDBCF1FF02C0EDBCF20F01D06000E51
:105840001E5A1F5A205A010EDBCFE9FF020EDBCF92
:10585000EAFF0A0EE926000EEA221DC0EEFF1EC076
:10586000EEFF1FC0EEFF20C0EEFFD950250FE96EFE
:10587000000EDA20EA6EEECFE6FFEECFE6FFEECFC7
:10588000E6FFEFCFE6FF010EDBCFE6FF020EDBCF38
:10589000E6FF0BEC08F01D6E060EE15C02E2E16A29
:1058A000E552E16E1D5027D0DF5026E10B0EE76E6A
:1058B000170EDBCFE9FF180EDBCFEAFFE750E92632
:1058C000000EEA22EF50100B02E0040E14D0F90E85
:1058D000DB50020B11E00B0EE76E170EDBCFE9FF7A
:1058E000180EDBCFEAFFE750E926000EEA22EF5060
:1058F000010B02E0070EDF6EDF5037E1F90EDBB679
:10590000DB8A010EDBCFE9FF020EDBCFEAFF2E0EB2
:10591000E926000EEA22EECF1DF0EECF1EF0EECF0C
:105920001FF0EFCF20F0FC0EDBCFE9FFFD0EDBCF49
:10593000EAFF1A0EE926000EEA221DC0EEFF1EC085
:10594000EEFF1FC0EEFF20C0EEFFFC0EDBCFE9FF35
:10595000FD0EDBCFEAFF1E0EE926000EEA22170E2F
:10596000DBCFEEFF180EDBCFEDFFDF5001E0ABD059
:10597000FC0EDBCFE9FFFD0EDBCFEAFF040EE926CC
:10598000000EEA22F90EDBCFEFFF170EDBCFE6FFAA
:10599000180EDBCFE6FF010EDBCFE6FF020EDBCFFA
:1059A000E6FF0DEC1BF0E552E552E552E5523CC036
:1059B0001EF03DC01FF03EC020F0FC0EDBCFE9FF23
:1059C000FD0EDBCFEAFF0E0EE926000EEA223BC0F9
:1059D000EEFF1EC0EEFF1FC0EEFF20C0EEFF1C0E4C
:1059E000E76E170EDBCFE9FF180EDBCFEAFFE750BB
:1059F000E926000EEA22EECF1DF0EECF1EF0EECF2C
:105A00001FF0EFCF20F0FC0EDBCFE9FFFD0EDBCF68
:105A1000EAFF0A0EE926000EEA221DC0EEFF1EC0B4
:105A2000EEFF1FC0EEFF20C0EEFFFC0EDBCFE9FF54
:105A3000FD0EDBCFEAFF060EE926000EEA22EE6A33
:105A4000EE6AEE6AEE6AFC0EDBCFE9FFFD0EDBCFFD
:105A5000EAFF160EE926000EEA22EE6AEE6AEE6A08
:105A6000EE6AFC0EDBCFE9FFFD0EDBCFEAFF200E76
:105A7000EB6A210EEB6AFC0EDBCFE9FFFD0EDBCFFC
:105A8000EAFF010EDBCFEEFF020EDBCFEDFF010ED2
:105A9000DBCFE9FF020EDBCFEAFF060EE926000EA0
:105AA000EA22EECF1DF0EFCF1EF0FC0EDBCFE9FFB8
:105AB000FD0EDBCFEAFF020EE926000EEA221DC032
:105AC000EEFF1EC0EDFFDF501D6E2D0EE15C02E209
:105AD000E16AE552E16E1D50E552E5CFDAFFE7CF0E
:105AE000D9FF1200D9CFE6FFDACFE6FFE1CFD9FF29
:105AF000E2CFDAFF140EE12402E3E168E652E16E40
:105B0000FA0EDBCF3DF0FB0EDBCF3EF0120E3DC0B8
:105B1000DBFF130E3EC0DBFFF60EDBCFE9FFF70E17
:105B2000DBCFEAFFEE6AED6AFC0EDBCFE6FFFD0E8F
:105B3000DBCFE6FF34DCE552E552DF6EDF5003E0F9
:105B4000DF50FFEF31F0FC0EDBCFE9FFFD0EDBCFC6
:105B5000EAFF040EE926000EEA22EF50800B01E076
:105B6000D6D1FC0EDBCFE9FFFD0EDBCFEAFF040E42
:105B7000E926000EEA22EF50010B03E1070EFFEFCA
:105B800031F0FC0EDBCFE9FFFD0EDBCFEAFF0A0EA2
:105B9000E926000EEA22EECF21F0EECF22F0EECF82
:105BA00023F0EFCF24F0FC0EDBCFE9FFFD0EDBCFBF
:105BB000EAFF060EE926000EEA22EE50215C1D6E79
:105BC000EE5022581E6EEE5023581F6EEE50245891
:105BD000206E090E1DC0DBFF0A0E1EC0DBFF0B0E80
:105BE0001FC0DBFF0C0E20C0DBFFF80EDBCF1DF06B
:105BF000F90EDBCF1EF01F6A206AD950090FE96E3B
:105C0000000EDA20EA6E1D50EE5C1E50EE581F505A
:105C1000EE582050EE580CE2090EDBCF3DF00A0E94
:105C2000DBCF3EF0F80E3DC0DBFFF90E3EC0DBFFE0
:105C3000D950F80FE96EFF0EDA20EA6EEE50ED1043
:105C400001E1DCD3FC0EDBCFE9FFFD0EDBCFEAFF89
:105C5000060EE926000EEA22EECF1DF0EECF1EF072
:105C6000010E1E161F6A206A1D501E101F102010E4
:105C700001E0C1D2FC0EDBCFE9FFFD0EDBCFEAFF76
:105C8000060EE926000EEA22EECF1DF0EECF1EF042
:105C9000EECF1FF0EFCF20F0090ED89020321F3248
:105CA0001E321D32E806F9E1FC0EDBCFE9FFFD0EE6
:105CB000DBCFEAFFEE50EFCFEAFFE96E020EE926F6
:105CC000000EEA22EF04216E226A236A246AE85059
:105CD0001D1622501E1623501F1624502016110E7A
:105CE0001DC0DBFFDB5001E0C4D0FC0EDBCFE9FFC1
:105CF000FD0EDBCFEAFF060EE926000EEA22EECF0C
:105D00001DF0EECF1EF0EECF1FF0EFCF20F01D50B4
:105D10001E101F10201017E1FC0EDBCFE9FFFD0E57
:105D2000DBCFEAFF0E0EE926000EEA22010EEECFCF
:105D3000DBFF020EEECFDBFF030EEECFDBFF040E28
:105D4000EECFDBFF5ED0FC0EDBCFE9FFFD0EDBCF3D
:105D5000EAFF200EE926000EEA22EE50ED101FE0C9
:105D6000FC0EDBCFE9FFFD0EDBCFEAFF060EE926D6
:105D7000000EEA22EECFE6FFEECFE6FFEECFE6FF23
:105D8000EFCFE6FFFC0EDBCFE6FFFD0EDBCFE6FF3D
:105D9000DEEC13F01D6E060EE15C25E222D0FC0E57
:105DA000DBCFE9FFFD0EDBCFEAFF120EE926000E86
:105DB000EA22EECFE6FFEECFE6FFEECFE6FFEFCF33
:105DC000E6FFFC0EDBCFE9FFFD0EDBCFEAFFEECFF7
:105DD000E6FFEFCFE6FF6CEC0AF01D6E060EE15C0D
:105DE00002E2E16AE552E16E1D50010E3BC0DBFFAD
:105DF000020E3CC0DBFF030E3DC0DBFF040E3EC0C5
:105E0000DBFFD950010FE96E000EDA20EA6E020EB8
:105E1000EE5C000EEE58000EEE58000EEE586CE3ED
:105E2000D950010FE96E000EDA20EA6EE868EE182C
:105E30000AE1E868EE1807E1E868EE1804E1E868AE
:105E4000EE1801E139D2FC0EDBCFE9FFFD0EDBCF0E
:105E5000EAFF120EE926000EEA22010EDBCFEEFF6A
:105E6000020EDBCFEEFF030EDBCFEEFF040EDBCF27
:105E7000EEFFFC0EDBCFE9FFFD0EDBCFEAFF120EDB
:105E8000E926000EEA22EECFE6FFEECFE6FFEECFE8
:105E9000E6FFEFCFE6FFFC0EDBCFE9FFFD0EDBCF29
:105EA000EAFFEECFE6FFEFCFE6FFDCEC09F01D6E78
:105EB000060EE15C02E2E16AE552E16E1D50050E5C
:105EC0003BC0DBFF060E3CC0DBFF070E3DC0DBFF27
:105ED000080E3EC0DBFF050EDBCF1DF0060EDBCF4C
:105EE0001EF0070EDBCF1FF0080EDBCF20F01D5099
:105EF0001E101F1020100DE1FC0EDBCFE9FFFD0E80
:105F0000DBCFEAFF040EE926000EEA22EF8E020E36
:105F100076D2110EDBCF1DF01E6A1F6A206AD9509F
:105F2000050FE96E000EDA20EA6E1D50EE261E50B7
:105F3000EE221F50EE222050EE221D6A020E1E6E2F
:105F4000F80EDBCF3DF0F90EDBCF3EF01DC042F086
:105F50001EC043F088EC70F00F0E3DC0DBFF100E4A
:105F60003EC0DBFFD9500F0FE96E000EDA20EA6E5B
:105F7000EE50ED1001E129D1110EDB501F6E206AA9
:105F80000F0EDB501F241D6E100EDB5020201E6EE6
:105F9000FC0EDBCFE9FFFD0EDBCFEAFFEE50EFCFCB
:105FA000EAFFE96E020EE926000EEA22EF50216EAA
:105FB000226A1D50215C1E50225820E2110EDBCFB8
:105FC000E6FFFC0EDBCFE9FFFD0EDBCFEAFFEE5074
:105FD000EFCFEAFFE96E020EE926000EEA22EF504B
:105FE000E552D880E754E66ED9500F0FE96E000EE7
:105FF000DA20EA6EE552E750EE6EED6A0F0EDBCF67
:10600000E6FFD950050FE96E000EDA20EA6EEECFFA
:10601000E6FFEECFE6FFEECFE6FFEFCFE6FF120E94
:10602000DBCFE6FF130EDBCFE6FFFC0EDBCFE9FF95
:10603000FD0EDBCFEAFFEE50EFCFEAFFE96EEE5246
:10604000EF50E66EF5EC5DF01D6E080EE15C02E2CD
:10605000E16AE552E16E1D50000901E02DD1FC0E10
:10606000DBCFE9FFFD0EDBCFEAFFEE50EFCFEAFF1B
:10607000E96E040EE926000EEA22EF5001E193D00A
:10608000050EDBCF21F0060EDBCF22F0070EDBCFB3
:1060900023F0080EDBCF24F0FC0EDBCFE9FFFD0E72
:1060A000DBCFEAFFEE50EFCFEAFFE96E2E0EE926D6
:1060B000000EEA222150EE5C1D6E2250EE581E6E3C
:1060C0002350EE581F6E2450EE58206E0F0EDBCF7B
:1060D00025F0100EDBCF26F0276A286A25501D5CBC
:1060E00026501E5827501F58285020585CE2E66A58
:1060F000020EE66EFC0EDBCFE9FFFD0EDBCFEAFF02
:10610000EE50EFCFEAFFE96E320EE926000EEA22EA
:10611000E9CF1DF0EACF1EF0E9CFE6FFEACFE6FFB8
:10612000050EDBCF25F0060EDBCF26F0070EDBCF0A
:1061300027F0080EDBCF28F0FC0EDBCFE9FFFD0EC9
:10614000DBCFEAFFEE50EFCFEAFFE96E2E0EE92635
:10615000000EEA222550EE5C216E2650EE58226E8B
:106160002750EE58236E2850EE58246E090ED89012
:106170002136223623362436E806F9E1120EDB50AA
:1061800021241F6E130EDB502220206E1FC0E6FF5D
:10619000E66E6CEC05F0296E060EE15C02E2E16A47
:1061A000E552E16E29503D6A020E3E6E0F0EDBCFC6
:1061B00042F0100EDBCF43F04FEC70F00D0E3BC001
:1061C000DBFF0E0E3CC0DBFFCED0FC0EDBCFE9FFC9
:1061D000FD0EDBCFEAFF160EE926000EEA22050EC1
:1061E000DBCFEEFF060EDBCFEEFF070EDBCFEEFFC1
:1061F000080EDBCFEEFFFC0EDBCFE9FFFD0EDBCFA1
:10620000EAFF060EE926000EEA22EECF1DF0EFCFE0
:106210001EF00001010E1E16000ED8801D56020E43
:106220001E560D0E1DC0DBFF0E0E1EC0DBFF0D0E39
:10623000DBCF1DF00E0EDBCF1EF0F80EDBCF1FF014
:10624000F90EDBCF20F01D501F5C1E5020580CE2D1
:10625000F80EDBCF3DF0F90EDBCF3EF00D0E3DC06A
:10626000DBFF0E0E3EC0DBFFFC0EDBCFE9FFFD0EB9
:10627000DBCFEAFF160EE926000EEA22EECFE6FF9C
:10628000EECFE6FFEECFE6FFEFCFE6FFFC0EDBCF73
:10629000E9FFFD0EDBCFEAFFEECFE6FFEFCFE6FF33
:1062A0000BEC08F01D6E060EE15C02E2E16AE552BD
:1062B000E16E1D5000090DE0FC0EDBCFE9FFFD0E85
:1062C000DBCFEAFF040EE926000EEA22EF8E010E74
:1062D00096D00D0EDBCFE6FF0E0EDBCFE6FFFC0EF9
:1062E000DBCFE9FFFD0EDBCFEAFFEE50EFCFEAFF99
:1062F000E96E320EE926000EEA22E9CF1FF0EACF5E
:1063000020F0FC0EDBCFE9FFFD0EDBCFEAFF060E2F
:10631000E926000EEA22EECF3BF0EECF3CF0EECFC6
:106320003DF0EFCF3EF0406A020E416E426A436A92
:106330002BEC70F01F5037241D6E205038201E6E3D
:106340001DC0E6FFE66E120EDBCFE6FF130EDBCFBD
:10635000E6FF6CEC05F0216E060EE15C02E2E16AFC
:10636000E552E16E21500D0EDBCF1DF00E0EDBCF9E
:106370001EF0D950120FE96E000EDA20EA6E1D50A1
:10638000EE261E50ED220D0EDBCF1FF00E0EDBCFE2
:1063900020F0216A226AFC0EDBCFE9FFFD0EDBCF85
:1063A000EAFF060EE926000EEA221F50EE262050D4
:1063B000EE222150EE222250EE220D0EDBCF23F0F2
:1063C0000E0EDBCF24F0F60EDBCFE9FFF70EDBCFAE
:1063D000EAFF2350EE262450ED220D0EDBCF25F0F0
:1063E0000E0EDBCF26F0D950F80FE96EFF0EDA2043
:1063F000EA6E2550EE5E2650ED5A1AD4000E1D6E40
:10640000140EE15C02E2E16AE552E16E1D50E552D4
:10641000E5CFDAFFE7CFD9FF1200D9CFE6FFDACF19
:10642000E6FFE1CFD9FFE2CFDAFF100EE12402E36D
:10643000E168E652E16EFA0EDBCF3DF0FB0EDBCFFA
:106440003EF00D0E3DC0DBFF0E0E3EC0DBFFF60E34
:10645000DBCFE9FFF70EDBCFEAFFEE6AED6AFC0E59
:10646000DBCFE6FFFD0EDBCFE6FFCFEC29F0E552F8
:10647000E552DF6EDF5003E0DF50C3EF37F0FC0E74
:10648000DBCFE9FFFD0EDBCFEAFF040EE926000EAD
:10649000EA22EF50800B01E04CD2FC0EDBCFE9FF8B
:1064A000FD0EDBCFEAFF040EE926000EEA22EF50D4
:1064B000020B03E1070EC3EF37F0F80EDBCF1DF040
:1064C000F90EDBCF1EF01F6A206AFC0EDBCFE9FF5E
:1064D000FD0EDBCFEAFF0A0EE926000EEA22EE509F
:1064E0001D26EE501E22EE501F22EE502022FC0EE2
:1064F000DBCFE9FFFD0EDBCFEAFF0A0EE926000E37
:10650000EA22EE501D5CEE501E58EE501F58EE5021
:10651000205804E2F80EDB6AF90EDB6AD950F80F56
:10652000E96EFF0EDA20EA6EEE50ED1002E16FEF39
:1065300037F0FC0EDBCFE9FFFD0EDBCFEAFF060EE6
:10654000E926000EEA22EECF1DF0EECF1EF0010E7E
:106550001E161F6A206A1D501E101F10201001E019
:10656000AAD3FC0EDBCFE9FFFD0EDBCFEAFF060E60
:10657000E926000EEA22EECF1DF0EECF1EF0EECFA0
:106580001FF0EFCF20F0090ED89020321F321E32BC
:106590001D32E806F9E1FC0EDBCFE9FFFD0EDBCF93
:1065A000EAFFEE50EFCFEAFFE96E020EE926000E99
:1065B000EA22EF04216E226A236A246AE8501D163B
:1065C00022502350245020160F0E1DC0DBFFDB503D
:1065D00001E023D1FC0EDBCFE9FFFD0EDBCFEAFFAC
:1065E000060EE926000EEA22EECF1DF0EECF1EF0D9
:1065F000EECF1FF0EFCF20F01D501E101F10201007
:1066000063E1FC0EDBCFE9FFFD0EDBCFEAFF0E0EF0
:10661000E926000EEA22010EEECFDBFF020EEECFDE
:10662000DBFF030EEECFDBFF040EEECFDBFF010E30
:10663000DBCF1DF0020EDBCF1EF0030EDBCF1FF011
:10664000040EDBCF20F01D501E101F10201001E0A3
:1066500099D0E66AE66AE66AE66AFC0EDBCFE9FFF5
:10666000FD0EDBCFEAFFEECFE6FFEFCFE6FF26EC35
:1066700011F01D6E060EE15C02E2E16AE552E16E88
:106680001D50010E3BC0DBFF020E3CC0DBFF030EC2
:106690003DC0DBFF040E3EC0DBFFFC0EDBCFE9FF9D
:1066A000FD0EDBCFEAFF0E0EE926000EEA22010EF8
:1066B000DBCFEEFF020EDBCFEEFF030EDBCFEEFFF4
:1066C000040EDBCFEEFF5ED0FC0EDBCFE9FFFD0E4C
:1066D000DBCFEAFF200EE926000EEA22EE50ED1095
:1066E0001FE0FC0EDBCFE9FFFD0EDBCFEAFF060E5D
:1066F000E926000EEA22EECFE6FFEECFE6FFEECF70
:10670000E6FFEFCFE6FFFC0EDBCFE6FFFD0EDBCFB3
:10671000E6FFDEEC13F01D6E060EE15C25E222D0F2
:10672000FC0EDBCFE9FFFD0EDBCFEAFF120EE92600
:10673000000EEA22EECFE6FFEECFE6FFEECFE6FF59
:10674000EFCFE6FFFC0EDBCFE9FFFD0EDBCFEAFF6C
:10675000EECFE6FFEFCFE6FF26EC11F01D6E060E42
:10676000E15C02E2E16AE552E16E1D50010E3BC0C0
:10677000DBFF020E3CC0DBFF030E3DC0DBFF040E5F
:106780003EC0DBFF010EDBCF1DF0020EDBCF1EF0A3
:10679000030EDBCF1FF0040EDBCF20F01D501E10C8
:1067A0001F10201001E19BD3D950010FE96E000E9C
:1067B000DA20EA6E010EEE1807E1EE5005E1EE5028
:1067C00003E1EE5001E1AAD0D950010FE96E000EAD
:1067D000DA20EA6EE868EE180AE1E868EE1807E1E8
:1067E000E868EE1804E1E868EE1801E1C5D2FC0E95
:1067F000DBCFE9FFFD0EDBCFEAFF120EE926000E2C
:10680000EA22010EDBCFEEFF020EDBCFEEFF030E1E
:10681000DBCFEEFF040EDBCFEEFFFC0EDBCFE9FF9C
:10682000FD0EDBCFEAFFEE50EFCFEAFFE96E2E0E52
:10683000E926000EEA22EECF1DF0EECF1EF0EECFDD
:106840001FF0EFCF20F0FC0EDBCFE9FFFD0EDBCF1A
:10685000EAFF160EE926000EEA221D50EE181BE193
:106860001E50EE1818E11F50EE1815E12050EE18DA
:1068700012E111E1FC0EDBCFE9FFFD0EDBCFEAFFF9
:10688000EECFE6FFEFCFE6FFC3EC06F0E552E552B0
:10689000000901E071D2FC0EDBCFE9FFFD0EDBCF7A
:1068A000EAFF120EE926000EEA22EECFE6FFEECF57
:1068B000E6FFEECFE6FFEFCFE6FFFC0EDBCFE9FF12
:1068C000FD0EDBCFEAFFEECFE6FFEFCFE6FFDCEC1D
:1068D00009F01D6E060EE15C02E2E16AE552E16E2E
:1068E0001D50050E3BC0DBFF060E3CC0DBFF070E54
:1068F0003DC0DBFF080E3EC0DBFF050EDBCF1DF009
:10690000060EDBCF1EF0070EDBCF1FF0080EDBCF2D
:1069100020F01D501E101F1020100DE1FC0EDBCFCB
:10692000E9FFFD0EDBCFEAFF040EE926000EEA22A6
:10693000EF8E020E28D30F0EDBCF1DF01E6A1F6AEA
:10694000206AD950050FE96E000EDA20EA6E1D505C
:10695000EE261E50EE221F50EE222050EE221D6A1F
:10696000020E1E6EF80EDBCF3DF0F90EDBCF3EF0CF
:106970001DC042F01EC043F088EC70F00B0E3DC00D
:10698000DBFF0C0E3EC0DBFFD9500B0FE96E000E93
:10699000DA20EA6EEE50ED1001E127D10F0EDB5048
:1069A0001F6E206A0B0EDB501F241D6E0C0EDB5079
:1069B00020201E6EFC0EDBCFE9FFFD0EDBCFEAFFD1
:1069C000EE50EFCFEAFFE96E020EE926000EEA2252
:1069D000EF50216E226A1D50215C1E50225820E289
:1069E0000F0EDBCFE6FFFC0EDBCFE9FFFD0EDBCFAA
:1069F000EAFFEE50EFCFEAFFE96E020EE926000E45
:106A0000EA22EF50E552D880E754E66ED9500B0FDA
:106A1000E96E000EDA20EA6EE552E750EE6EED6A9E
:106A20000B0EDBCFE6FFD950050FE96E000EDA2022
:106A3000EA6EEECFE6FFEECFE6FFEECFE6FFEFCF5A
:106A4000E6FF0D0EDBCFE6FF0E0EDBCFE6FFFC0E02
:106A5000DBCFE9FFFD0EDBCFEAFFEE50EFCFEAFF21
:106A6000E96EEE52EF50E66E65EC5EF01D6E080EBC
:106A7000E15C02E2E16AE552E16E1D50000901E0CD
:106A80007BD1050EDBCF21F0060EDBCF22F0070E07
:106A9000DBCF23F0080EDBCF24F0FC0EDBCFE9FFC9
:106AA000FD0EDBCFEAFFEE50EFCFEAFFE96E2E0ED0
:106AB000E926000EEA222150EE5C1D6E2250EE58AF
:106AC0001E6E2350EE581F6E2450EE58206E0B0E93
:106AD000DBCF25F00C0EDBCF26F0276A286A255085
:106AE0001D5C26501E5827501F58285020586BE216
:106AF000E66A020EE66E050EDBCF23F0060EDBCF54
:106B000024F0070EDBCF25F0080EDBCF26F0FC0EBD
:106B1000DBCFE9FFFD0EDBCFEAFFEE50EFCFEAFF60
:106B2000E96E2E0EE926000EEA222350EE5C1F6E5F
:106B30002450EE58206E2550EE58216E2650EE5807
:106B4000226E090ED8901F36203621362236E806EE
:106B5000F9E10D0EDB501F241D6E0E0EDB502020C0
:106B60001E6E1DC0E6FFE66EFC0EDBCFE9FFFD0EDC
:106B7000DBCFEAFFEE50EFCFEAFFE96E320EE926F7
:106B8000000EEA22E9CF27F0EACF28F0E9CFE6FFAE
:106B9000EACFE6FF6CEC05F0296E060EE15C02E23E
:106BA000E16AE552E16E2950FC0EDBCFE9FFFD0EF4
:106BB000DBCFEAFFEE50EFCFEAFFE96E040EE926E5
:106BC000000EEA22EF6A3D6A020E3E6E0B0EDBCF2C
:106BD00042F00C0EDBCF43F04FEC70F0090E3BC0DF
:106BE000DBFF0A0E3CC0DBFF2ED1FC0EDBCFE9FF42
:106BF000FD0EDBCFEAFF0A0EE926000EEA22EECFF9
:106C00001DF0EECF1EF0EECF1FF0EFCF20F0FC0E08
:106C1000DBCFE9FFFD0EDBCFEAFF060EE926000E13
:106C2000EA221D50EE5C1E50EE581F50EE582050C8
:106C3000EE582BE3FC0EDBCFE9FFFD0EDBCFEAFFC6
:106C4000EECFE6FFEFCFE6FFC3EC06F0E552E552EC
:106C5000000901E091D0FC0EDBCFE9FFFD0EDBCF98
:106C6000EAFFEE50EFCFEAFFE96E2E0EE926000EA6
:106C7000EA22050EDBCFEEFF060EDBCFEEFF070E9E
:106C8000DBCFEEFF080EDBCFEEFFFC0EDBCFE9FF24
:106C9000FD0EDBCFEAFF160EE926000EEA22050EF6
:106CA000DBCFEEFF060EDBCFEEFF070EDBCFEEFFF6
:106CB000080EDBCFEEFFFC0EDBCFE9FFFD0EDBCFD6
:106CC000EAFF060EE926000EEA22EECF1DF0EFCF16
:106CD0001EF00001010E1E16000ED8801D56020E79
:106CE0001E56090E1DC0DBFF0A0E1EC0DBFF090E7B
:106CF000DBCF1DF00A0EDBCF1EF0F80EDBCF1FF04E
:106D0000F90EDBCF20F01D501F5C1E5020580CE206
:106D1000F80EDBCF3DF0F90EDBCF3EF0090E3DC0A3
:106D2000DBFF0A0E3EC0DBFFFC0EDBCFE9FFFD0EF2
:106D3000DBCFEAFF160EE926000EEA22EECFE6FFD1
:106D4000EECFE6FFEECFE6FFEFCFE6FFFC0EDBCFA8
:106D5000E9FFFD0EDBCFEAFFEECFE6FFEFCFE6FF68
:106D60000BEC08F01D6E060EE15C02E2E16AE552F2
:106D7000E16E1D5000090DE0FC0EDBCFE9FFFD0EBA
:106D8000DBCFEAFF040EE926000EEA22EF8E010EA9
:106D9000FAD0090EDBCFE6FF0A0EDBCFE6FF0D0EC1
:106DA000DBCFE6FF0E0EDBCFE6FFFC0EDBCFE9FF0D
:106DB000FD0EDBCFEAFFEE50EFCFEAFFE96E320EB9
:106DC000E926000EEA22E9CF1FF0EACF20F0FC0E00
:106DD000DBCFE9FFFD0EDBCFEAFF060EE926000E52
:106DE000EA22EECF3BF0EECF3CF0EECF3DF0EFCF1E
:106DF0003EF0406A020E416E426A436A2BEC70F02C
:106E00001F5037241D6E205038201E6E1DC0E6FF17
:106E1000E66E6CEC05F0216E060EE15C02E2E16AC2
:106E2000E552E16E2150FC0EDBCFE9FFFD0EDBCF1A
:106E3000EAFFEE50EFCFEAFFE96E040EE926000EFE
:106E4000EA22010EEF6E090EDBCF1DF00A0EDBCF3A
:106E50001EF0D9500D0FE96E000EDA20EA6E1D50BB
:106E6000EE261E50ED22090EDBCF1FF00A0EDBCFFF
:106E700020F0216A226AFC0EDBCFE9FFFD0EDBCF9A
:106E8000EAFF060EE926000EEA221F50EE262050E9
:106E9000EE222150EE222250EE22090EDBCF23F00B
:106EA0000A0EDBCF24F0F60EDBCFE9FFF70EDBCFC7
:106EB000EAFF2350EE262450ED22090EDBCF25F009
:106EC0000A0EDBCF26F0D950F80FE96EFF0EDA205C
:106ED000EA6E2550EE5E2650ED5A8EEF32F0FC0E33
:106EE000DBCFE9FFFD0EDBCFEAFF0A0EE926000E3D
:106EF000EA22EECF1DF0EECF1EF0EECF1FF0EFCF67
:106F000020F0FC0EDBCFE9FFFD0EDBCFEAFF060E23
:106F1000E926000EEA22EE501D5CEE501E58EE509F
:106F20001F58EE50205824E2FC0EDBCFE9FFFD0E87
:106F3000DBCFEAFF060EE926000EEA22EECF1DF0B7
:106F4000EECF1EF0EECF1FF0EFCF20F0FC0EDBCF28
:106F5000E9FFFD0EDBCFEAFF0A0EE926000EEA226A
:106F60001DC0EEFF1EC0EEFF1FC0EEFF20C0EEFFF3
:106F7000FC0EDBCFE9FFFD0EDBCFEAFF040EE926B6
:106F8000000EEA22EF8A1D6E100EE15C02E2E16A59
:106F9000E552E16E1D50E552E5CFDAFFE7CFD9FFAC
:106FA0001200D9CFE6FFDACFE6FFE1CFD9FFE2CF7B
:106FB000DAFF070EE12402E3E168E652E16EFC0E1F
:106FC000DBCFE6FFFD0EDBCFE6FFCFEC29F0E5528D
:106FD000E552DF6EDF5001E0FBD0FC0EDBCFE9FFB6
:106FE000FD0EDBCFEAFF040EE926000EEA22EF5089
:106FF000200B01E1EDD0FC0EDBCFE9FFFD0EDBCF76
:10700000EAFF1A0EE926000EEA22EECFE6FFEECFE7
:10701000E6FFEECFE6FFEFCFE6FFFC0EDBCFE9FFAA
:10702000FD0EDBCFEAFFEECFE6FFEFCFE6FF0BEC86
:1070300008F01D6E060EE15C02E2E16AE552E16EC7
:107040001D50DF6EDF5001E0C3D0FC0EDBCFE9FF47
:10705000FD0EDBCFEAFF1E0EE926000EEA22050E2A
:10706000EECFDBFF060EEDCFDBFF0B0EE76E050E5E
:10707000DBCFE9FF060EDBCFEAFFE750E926000E83
:10708000EA22EF8AFC0EDBCFE9FFFD0EDBCFEAFF41
:107090000A0EE926000EEA22EECF1DF0EECF1EF01A
:1070A000EECF1FF0EFCF20F01C0EE76E050EDBCF0A
:1070B000E9FF060EDBCFEAFFE750E926000EEA22E1
:1070C0001DC0EEFF1EC0EEFF1FC0EEFF20C0EEFF92
:1070D000FC0EDBCFE9FFFD0EDBCFEAFF0E0EE9264B
:1070E000000EEA22EECFE6FFEECFE6FFEECFE6FFA0
:1070F000EFCFE6FF050EDBCFE6FF060EDBCFE6FFA8
:1071000077EC1BF01D6E060EE15C02E2E16AE552CF
:10711000E16E1D507AEC68F0010E3BC0DBFF020E01
:107120003CC0DBFF030E3DC0DBFF040E3EC0DBFFB7
:10713000160EE76E050EDBCFE9FF060EDBCFEAFF8A
:10714000E750E926000EEA22010EDBCFEEFF020E29
:10715000DBCFEEFF030EDBCFEEFF040EDBCFEEFF47
:10716000120EE76E050EDBCFE9FF060EDBCFEAFF5E
:10717000E750E926000EEA22EE6AED6AFC0EDBCF4C
:10718000E9FFFD0EDBCFEAFF040EE926000EEA223E
:10719000EF9AFC0EDBCFE9FFFD0EDBCFEAFFEE50EE
:1071A000EFCFEAFFE96E040EE926000EEA22010E97
:1071B000EF6EFC0EDBCFE9FFFD0EDBCFEAFFEECF7B
:1071C000E6FFEFCFE6FF96EC08F0E552E552DF6E02
:1071D000DF501D6E070EE15C02E2E16AE552E16EEE
:1071E0001D50E552E5CFDAFFE7CFD9FF1200D9CF26
:1071F000E6FFDACFE6FFE1CFD9FFE2CFDAFFE652D2
:10720000FC0EDBCFE6FFFD0EDBCFE6FFCADEE5526C
:10721000E552DF6EDF5008E1FC0EDBCFE9FFFD0E2B
:10722000DBCFEAFFEE6AED6ADF50E552E552E5CFCB
:10723000DAFFE7CFD9FF1200D9CFE6FFDACFE6FFBA
:10724000E1CFD9FFE2CFDAFF2F0EE12402E3E168BC
:10725000E652E16EFC0EDBCFE6FFFD0EDBCFE6FF74
:10726000CFEC29F0E552E552DF6EDF5003E0DF504E
:1072700078EF41F0FC0EDBCFE9FFFD0EDBCFEAFF3C
:10728000040EE926000EEA22EF50800B02E0B0EF78
:1072900040F0FC0EDBCFE9FFFD0EDBCFEAFF200E56
:1072A000E926000EEA22EE50ED1001E172D3D9502A
:1072B000F80FE96EFF0EDA20EA6EE868EE1801E0DA
:1072C000EAD1E868EE1801E0E6D1E868EE1801E0DE
:1072D000E2D1E868EE1801E0DED1FC0EDBCFE9FF79
:1072E000FD0EDBCFEAFF200EE926000EEA221D0E7E
:1072F000EECFDBFF1E0EEDCFDBFFD9501D0FE96E89
:10730000000EDA20EA6EEECFF3FFEDCFF4FF040EAD
:10731000EE26000EEF22F3CFE9FFF4CFEAFF150EC1
:10732000EECFDBFF160EEECFDBFF170EEECFDBFF4F
:10733000180EEECFDBFF020EF36E190EF3CFDBFF5C
:107340001A0EDB6A1B0EDB6A1C0EDB6AFC0EDBCF3F
:10735000E9FFFD0EDBCFEAFF0E0EE926000EEA2262
:10736000010EEECFDBFF020EEECFDBFF030EEECF02
:10737000DBFF040EEECFDBFF010EDBCF1DF0020EB4
:10738000DBCF1EF0030EDBCF1FF0040EDBCF20F0AF
:107390001D501E101F10201001E138D1D950010FCF
:1073A000E96E000EDA20EA6E0D0EEECFDBFF0E0E58
:1073B000EECFDBFF0F0EEECFDBFF100EEECFDBFFCD
:1073C000090EDB6A0A0EDB6A0B0EDB6A0C0EDB6A47
:1073D000D950190FE96E000EDA20EA6E020EEE2681
:1073E000000EEE22EE22EE22D950010FE96E000EC1
:1073F000DA20EA6E050EEECFDBFF060EEECFDBFFE6
:10740000070EEECFDBFF080EEECFDBFFD950090FE2
:10741000E96E000EDA20EA6EEE2A000EEE22EE226F
:10742000EE22D950010FE96E000EDA20EA6EEECF9F
:10743000E6FFEECFE6FFEECFE6FFEFCFE6FFFC0E76
:10744000DBCFE9FFFD0EDBCFEAFFEECFE6FFEFCFAC
:10745000E6FF6CEC0AF01D6E060EE15C02E2E16AEA
:10746000E552E16E1D50010E3BC0DBFF020E3CC039
:10747000DBFF030E3DC0DBFF040E3EC0DBFFD95037
:10748000010FE96E000EDA20EA6ED880010EEE548C
:10749000000EEE54000EEE54000EEE5402E3A5EF83
:1074A00040F0D950010FE96E000EDA20EA6EE8686C
:1074B000EE180BE1E868EE1808E1E868EE1805E15F
:1074C000E868EE1802E1BEEF3FF0010E1D6E1E6A85
:1074D0001F6A206AD950050FE96E000EDA20EA6EA5
:1074E000EE501D26EE501E22EE501F22EE5020229E
:1074F000D950010FE96E000EDA20EA6EEE501D1829
:1075000008E1EE501E1805E1EE501F1802E1EE50A2
:10751000201801E169D7150EDBCF1DF0160EDBCF69
:107520001EF0170EDBCF1FF0180EDBCF20F0D95066
:10753000190FE96E000EDA20EA6EEE501D5CEE5077
:107540001E58EE501F58EE5020583CE3D9501D0FE6
:10755000E96E000EDA20EA6EEECFF3FFEDCFF4FF16
:10756000040EEE26000EEF22F3CFE9FFF4CFEAFF80
:10757000090EDBCFEEFF0A0EDBCFEEFF0B0EDBCFEB
:10758000EEFF0C0EDBCFEEFFD9501D0FE96E000EA3
:10759000DA20EA6EEECFF3FFEDCFF4FF040EEE2615
:1075A000000EEF22F3CFE9FFF4CFEAFF0D0EDBCFA1
:1075B000EEFF0E0EDBCFEEFF0F0EDBCFEEFF100E59
:1075C000DBCFEEFF010EDBCF1DF0020EDBCF1EF096
:1075D000030EDBCF1FF0040EDBCF20F0FC0EDBCF61
:1075E000E9FFFD0EDBCFEAFFEE50EFCFEAFFE96ED9
:1075F000160EE926000EEA22EE501D5CEE501E58D3
:10760000EE501F58EE50205801E2C8D6FC0EDBCFDA
:10761000E9FFFD0EDBCFEAFF200EE926000EEA228D
:10762000EE50EFCFEAFFE96E190EDBCFEEFF1A0E38
:10763000DBCFEEFF1B0EDBCFEEFF1C0EDBCFEEFF32
:10764000150EDBCF1DF0160EDBCF1EF0170EDBCFB5
:107650001FF0180EDBCF20F0D950190FE96E000E85
:10766000DA20EA6EEE501D5CEE501E58EE501F58A8
:10767000EE5020580CE31D0EDBCFE9FF1E0EDBCFD2
:10768000EAFFEE6AEE6AEE6AEE6A77EF41F0110EFB
:10769000DF6E77EF41F0F80EDBCF1DF0F90EDBCF98
:1076A0001EF0FA0EDBCF1FF0FB0EDBCF20F0FC0E3E
:1076B000DBCFE9FFFD0EDBCFEAFF0A0EE926000E65
:1076C000EA221D50EE5C1E50EE581F50EE5820501E
:1076D000EE5816E2FC0EDBCFE9FFFD0EDBCFEAFF32
:1076E0000A0EE926000EEA22F80EEECFDBFFF90EB5
:1076F000EECFDBFFFA0EEECFDBFFFB0EEECFDBFFB4
:10770000FC0EDBCFE9FFFD0EDBCFEAFF060EE9261C
:10771000000EEA22F80EDBCFEEFFF90EDBCFEEFF14
:10772000FA0EDBCFEEFFFB0EDBCFEEFFF80EDBCF6A
:107730001DF0F90EDBCF1EF0FA0EDBCF1FF0FB0EB3
:10774000DBCF20F01D501E101F10201002E177EF3C
:1077500041F0F80EDBCF21F0F90EDBCF22F0FA0E6C
:10776000DBCF23F0FB0EDBCF24F02106000E225AE4
:10777000235A245A21C0E6FF22C0E6FF23C0E6FFB9
:1077800024C0E6FFFC0EDBCFE6FFFD0EDBCFE6FFFD
:10779000DEEC13F0256E060EE15C02E2E16AE552D2
:1077A000E16E25503BC01DF03CC01EF03DC01FF0F7
:1077B0003EC020F0FC0EDBCFE9FFFD0EDBCFEAFF81
:1077C000120EE926000EEA223BC0EEFF1EC0EEFFBD
:1077D0001FC0EEFF20C0EEFFFC0EDBCFE9FFFD0E69
:1077E000DBCFEAFF120EE926000EEA22EECFE6FF1B
:1077F000EECFE6FFEECFE6FFEFCFE6FFFC0EDBCFEE
:10780000E9FFFD0EDBCFEAFFEECFE6FFEFCFE6FFAD
:10781000DCEC09F01D6E060EE15C02E2E16AE55265
:10782000E16E1D50110E3BC0DBFF120E3CC0DBFFB2
:10783000130E3DC0DBFF140E3EC0DBFF110EDBCF8D
:107840001DF0120EDBCF1EF0130EDBCF1FF0140E57
:10785000DBCF20F01D501E101F10201002E1A5EFFD
:1078600040F0F80EDBCF1DF0F90EDBCF1EF0FA0E64
:10787000DBCF1FF0FB0EDBCF20F01D06000E1E5AE3
:107880001F5A205A090ED89020321F321E321D3244
:10789000E806F9E1FC0EDBCFE9FFFD0EDBCFEAFFE6
:1078A000EE50EFCFEAFFE96E020EE926000EEA2263
:1078B000EF04226A236A246AE8501D1622501E161D
:1078C00023501F1624502016D950110FE96E000EB8
:1078D000DA20EA6E1D50EE261E50EE221F50EE22D8
:1078E0002050EE22FC0EDBCFE9FFFD0EDBCFEAFFDE
:1078F000060EE926000EEA22EECF1DF0EECF1EF0B6
:10790000EECF1FF0010E1E161F6A206A1D501E10BA
:107910001F10201002E177EF41F0110EDBCF21F0B4
:10792000120EDBCF22F0130EDBCF23F0140EDBCFD1
:1079300024F0FC0EDBCFE9FFFD0EDBCFEAFF160ED5
:10794000E926000EEA222150EE1808E12250EE1836
:1079500005E12350EE1802E12450EE1802E177EF22
:1079600041F0FC0EDBCFE9FFFD0EDBCFEAFF160E88
:10797000E926000EEA22110EDBCFEEFF120EDBCF5E
:10798000EEFF130EDBCFEEFF140EDBCFEEFF77EF33
:1079900041F0F80EDBCF1DF0F90EDBCF1EF0FA0E32
:1079A000DBCF1FF0FB0EDBCF20F0FC0EDBCFE9FFBF
:1079B000FD0EDBCFEAFF0A0EE926000EEA221D507B
:1079C000EE5C1E50EE581F50EE582050EE5823E249
:1079D000FC0EDBCFE9FFFD0EDBCFEAFF040EE9264C
:1079E000000EEA22EF50020B16E1FC0EDBCFE9FF9E
:1079F000FD0EDBCFEAFF0A0EE926000EEA22F80EA2
:107A0000EECFDBFFF90EEECFDBFFFA0EEECFDBFFA2
:107A1000FB0EEECFDBFFFC0EDBCFE9FFFD0EDBCF75
:107A2000EAFF060EE926000EEA222B0EEECFDBFF60
:107A30002C0EEECFDBFF2D0EEECFDBFF2E0EEECFAA
:107A4000DBFF270EDB6A280EDB6A290EDB6A2A0EB3
:107A5000DB6AFC0EDBCFE9FFFD0EDBCFEAFF060E93
:107A6000E926000EEA22EE6AEE6AEE6AEE6AF80E87
:107A7000DBCF1DF0F90EDBCF1EF0FA0EDBCF1FF0CF
:107A8000FB0EDBCF20F01D501E101F10201001E157
:107A90008BD3FC0EDBCFE9FFFD0EDBCFEAFFEE5010
:107AA000EFCFEAFFE96E020EE926000EEA22EFCFE1
:107AB0003BF03C6A3D6A3E6A406A020E416E426A91
:107AC000436ACEEC6FF0230E37C0DBFF240E38C0C4
:107AD000DBFF250E39C0DBFF260E3AC0DBFFD95095
:107AE0002B0FE96E000EDA20EA6ED880000EEE54FD
:107AF000000EEE54000EEE54000EEE5401E3D7D00B
:107B00002B0EDBCF25F02C0EDBCF26F02D0EDBCF9E
:107B100027F02E0EDBCF28F02506000E265A275A16
:107B2000285A25C03BF026C03CF027C03DF028C0B5
:107B30003EF0230EDBCF40F0240EDBCF41F0250ECC
:107B4000DBCF42F0260EDBCF43F02BEC70F03BC0D6
:107B500021F03CC022F03DC023F03EC024F0F80EDE
:107B6000DBCF1DF0F90EDBCF1EF0FA0EDBCF1FF0DE
:107B7000FB0EDBCF20F01D06000E1E5A1F5A205AA6
:107B80001DC03BF01EC03CF01FC03DF020C03EF0C9
:107B9000230EDBCF40F0240EDBCF41F0250EDBCFF0
:107BA00042F0260EDBCF43F02BEC70F021503B5C13
:107BB00022503C5823503D5824503E5801E277D083
:107BC0002B0EDBCF1DF02C0EDBCF1EF02D0EDBCFEE
:107BD0001FF02E0EDBCF20F01D06000E1E5A1F5A7E
:107BE000205A230EDBCF21F0240EDBCF22F0250E0E
:107BF000DBCF23F0260EDBCF24F02106000E225A25
:107C0000235A245A211E221E231E241E21501D16D3
:107C100022501E1623501F1624502016FC0EDBCFB8
:107C2000E9FFFD0EDBCFEAFF060EE926000EEA2291
:107C30001DC0EEFF1EC0EEFF1FC0EEFF20C0EEFF16
:107C4000FC0EDBCFE9FFFD0EDBCFEAFF060EE926D7
:107C5000000EEA22EECF1DF0EECF1EF0EECF1FF0A9
:107C6000EFCF20F0D950F80FE96EFF0EDA20EA6E60
:107C70001D50EE5E1E50EE5A1F50EE5A2050EE5A26
:107C8000FC0EDBCFE9FFFD0EDBCFEAFF120EE9268B
:107C9000000EEA221F0EEECFDBFF200EEECFDBFF41
:107CA000210EEECFDBFF220EEECFDBFF9AD0FC0ED3
:107CB000DBCFE9FFFD0EDBCFEAFF0E0EE926000E5B
:107CC000EA221F0EEECFDBFF200EEECFDBFF210EF0
:107CD000EECFDBFF220EEECFDBFF1F0EDBCF1DF062
:107CE000200EDBCF1EF0210EDBCF1FF0220EDBCFEC
:107CF00020F01D501E101F1020105DE1E66AE66A9C
:107D0000E66AE66AFC0EDBCFE9FFFD0EDBCFEAFF99
:107D1000EECFE6FFEFCFE6FF26EC11F01D6E060E6C
:107D2000E15C02E2E16AE552E16E1D501F0E3BC0CC
:107D3000DBFF200E3CC0DBFF210E3DC0DBFF220E2F
:107D40003EC0DBFFD9501F0FE96E000EDA20EA6E4D
:107D5000010EEE1807E1EE5005E1EE5003E1EE50A2
:107D600001E1F3D1D9501F0FE96E000EDA20EA6E5F
:107D7000E868EE180AE1E868EE1807E1E868EE182E
:107D800004E1E868EE1801E1F9D0FC0EDBCFE9FF71
:107D9000FD0EDBCFEAFF0E0EE926000EEA221F0ED3
:107DA000DBCFEEFF200EDBCFEEFF210EDBCFEEFFB1
:107DB000220EDBCFEEFFFC0EDBCFE9FFFD0EDBCFAB
:107DC000EAFF120EE926000EEA221F0EDBCFEEFFBD
:107DD000200EDBCFEEFF210EDBCFEEFF220EDBCF3E
:107DE000EEFF1F0EDBCF1DF0200EDBCF1EF0210EAD
:107DF000DBCF1FF0220EDBCF20F01D501E101F1016
:107E0000201001E1D1D1230EDBCF1DF0240EDBCFFA
:107E10001EF0250EDBCF1FF0260EDBCF20F0D95051
:107E2000F80FE96EFF0EDA20EA6EEE501D5CEE50A0
:107E30001E58EE501F58EE50205801E320D1FC0E82
:107E4000DBCFE9FFFD0EDBCFEAFF040EE926000ED3
:107E5000EA22EF50020B52E0D9501F0FE96E000EDC
:107E6000DA20EA6EEECFE6FFEECFE6FFEECFE6FFDA
:107E7000EFCFE6FFFC0EDBCFE9FFFD0EDBCFEAFF25
:107E8000EECFE6FFEFCFE6FF26EC11F01D6E060EFB
:107E9000E15C02E2E16AE552E16E1D501F0E3BC05B
:107EA000DBFF200E3CC0DBFF210E3DC0DBFF220EBE
:107EB0003EC0DBFF1F0EDBCF1DF0200EDBCF1EF020
:107EC000210EDBCF1FF0220EDBCF20F01D501E1045
:107ED0001F10201041E1D950230FE96E000EDA2067
:107EE000EA6EF80EEECFDBFFF90EEECFDBFFFA0EF7
:107EF000EECFDBFFFB0EEECFDBFFC1D0D9501F0F63
:107F0000E96E000EDA20EA6EEECFE6FFEECFE6FF76
:107F1000EECFE6FFEFCFE6FFFC0EDBCFE9FFFD0E75
:107F2000DBCFEAFFEECFE6FFEFCFE6FF6CEC0AF027
:107F30001D6E060EE15C02E2E16AE552E16E1D5043
:107F40001F0E3BC0DBFF200E3CC0DBFF210E3DC0FF
:107F5000DBFF220E3EC0DBFFD9501F0FE96E000E83
:107F6000DA20EA6EE868EE1816E1E868EE1813E128
:107F7000E868EE1810E1E868EE180DE1FC0EDBCFC2
:107F8000E9FFFD0EDBCFEAFF040EE926000EEA2230
:107F9000EF8E010EADD1D9501F0FE96E000EDA2021
:107FA000EA6ED880010EEE54000EEE54000EEE5430
:107FB000000EEE5401E3C9D01F0EDBCF1DF0200EE2
:107FC000DBCF1EF0210EDBCF1FF0220EDBCF20F027
:107FD000FC0EDBCFE9FFFD0EDBCFEAFFEE50EFCF6B
:107FE000EAFFE96E160EE926000EEA22EE501D5C4D
:107FF000EE501E58EE501F58EE50205801E3A5D009
:10800000FC0EDBCFE9FFFD0EDBCFEAFF120EE92607
:10801000000EEA221F0EDBCFEEFF200EDBCFEEFFBD
:10802000210EDBCFEEFF220EDBCFEEFFFC0EDBCF0F
:10803000E9FFFD0EDBCFEAFF060EE926000EEA227D
:10804000230EDB50EE26240EDB50EE22250EDB50F5
:10805000EE22260EDB50EE22D950F80FE96EFF0E0D
:10806000DA20EA6E230EDB50EE5E240EDB50EE5A71
:10807000250EDB50EE5A260EDB50EE5AC4D6FC0E0F
:10808000DBCFE9FFFD0EDBCFEAFF060EE926000E8F
:10809000EA22F80EDB50EE26F90EDB50EE22FA0E45
:1080A000DB50EE22FB0EDB50EE22F80EDBCF1DF094
:1080B000F90EDBCF1EF0FA0EFB0E010E1E161F6A24
:1080C000206A1D501E101F1020106EE0D9501F0F87
:1080D000E96E000EDA20EA6EEECFE6FFEECFE6FFA5
:1080E000EECFE6FFEFCFE6FFFC0EDBCFE9FFFD0EA4
:1080F000DBCFEAFFEECFE6FFEFCFE6FFDCEC09F0E7
:108100001D6E060EE15C02E2E16AE552E16E1D5071
:10811000270E3BC0DBFF280E3CC0DBFF290E3DC015
:10812000DBFF2A0E3EC0DBFF270EDBCF1DF0280E43
:10813000DBCF1EF0290EDBCF1FF02A0EDBCF20F0A5
:108140001D501E101F1020100DE1FC0EDBCFE9FFAB
:10815000FD0EDBCFEAFF040EE926000EEA22EF8EC9
:10816000020EC6D0F80EDBCF1DF0F90EDBCF1EF0ED
:10817000FA0EDBCF1FF0FB0EDBCF20F0090ED890FC
:1081800020321F321E321D32E806F9E1D950270F86
:10819000E96E000EDA20EA6E1D50EE261E50EE2229
:1081A0001F50EE222050EE22FC0EDBCFE9FFFD0E29
:1081B000DBCFEAFF060EE926000EEA22EECF1DF025
:1081C000EECF1EF0010E1E161F6A206A1D501E10F3
:1081D0001F10201038E0270EDBCF21F0280EDBCF58
:1081E00022F0290EDBCF23F02A0EDBCF24F0FC0E89
:1081F000DBCFE9FFFD0EDBCFEAFF160EE926000E0E
:10820000EA222150EE1808E12250EE1805E1235031
:10821000EE1802E12450EE1816E0FC0EDBCFE9FF69
:10822000FD0EDBCFEAFF160EE926000EEA22270E2E
:10823000DBCFEEFF280EDBCFEEFF290EDBCFEEFF0C
:108240002A0EDBCFEEFFFC0EDBCFE9FFFD0EDBCF0E
:10825000EAFF0A0EE926000EEA22EECF1DF0EECF6D
:108260001EF0EECF1FF0EFCF20F0FC0EDBCFE9FFCA
:10827000FD0EDBCFEAFF060EE926000EEA22EE50E5
:108280001D5CEE501E58EE501F58EE5020582FE245
:10829000FC0EDBCFE9FFFD0EDBCFEAFF060EE92681
:1082A000000EEA22EECF1DF0EECF1EF0EECF1FF053
:1082B000EFCF20F0FC0EDBCFE9FFFD0EDBCFEAFFB6
:1082C0000A0EE926000EEA221DC0EEFF1EC0EEFFD8
:1082D0001FC0EEFF20C0EEFFFC0EDBCFE9FFFD0E5E
:1082E000DBCFEAFF040EE926000EEA22EF8ADF5018
:1082F0001D6E2F0EE15C02E2E16AE552E16E1D5057
:10830000E552E5CFDAFFE7CFD9FF1200D9CFE6FF7C
:10831000DACFE6FFE1CFD9FFE2CFDAFF0F0EE1249B
:1083200002E3E168E652E16ED950FC0FE96EFF0E00
:10833000DA20EA6EEE50ED1002E1090EEDD0E66AA9
:10834000FC0EDBCFE9FFFD0EDBCFEAFFE9CF1DF02E
:10835000EACF1EF0E9CFE6FFEACFE6FFD950FA0FE9
:10836000E66EFF0EDA20E66E9CEC22F01F6E050E24
:10837000E15C02E2E16AE552E16E1F50DF6EFC0E45
:10838000DBCFE9FFFD0EDBCFEAFF010EEECFDBFF17
:10839000020EEDCFDBFFDF5001E0B5D0D950030F67
:1083A0001D6E000EDA201E6EFC0EDBCFE9FFFD0E07
:1083B000DBCFEAFF140EE926000EEA221DC0EEFF15
:1083C0001EC0EDFFFA0EDBCFE6FFFB0EDBCFE6FFB4
:1083D000FC0EDBCFE6FFFD0EDBCFE6FFF3EC20F07B
:1083E000E552E552E552E552DF6EDF5001E084D000
:1083F000FC0EDBCFE9FFFD0EDBCFEAFF120EE92614
:10840000000EEA22EE50ED104AE0FC0EDBCFE9FF51
:10841000FD0EDBCFEAFF120EE926000EEA22EE5037
:10842000EFCFEAFFE96E0B0EE926000EEA22EF50CD
:10843000100B33E0FC0EDBCFE9FFFD0EDBCFEAFFD4
:10844000120EE926000EEA22EECFE6FFEFCFE6FF9E
:10845000010EDBCFE6FF020EDBCFE6FF0DEC1BF0DB
:10846000E552E552E552E5523CC01EF03DC01FF01A
:108470003EC020F0FC0EDBCFE9FFFD0EDBCFEAFFB4
:10848000060EE926000EEA223BC0EEFF1EC0EEFFFC
:108490001FC0EEFF20C0EEFF02D0050EDF6EDF50E2
:1084A0002BE1010EDBCFE9FF020EDBCFEAFF060E68
:1084B000E926000EEA22EECF1DF0EFCF1EF0FC0EF3
:1084C000DBCFE9FFFD0EDBCFEAFF020EE926000E4F
:1084D000EA221DC0EEFF1EC0EDFFE66EE66AFC0E4E
:1084E000DBCFE6FFFD0EDBCFE6FFD4EC14F0E55268
:1084F000E552E552E552DF6E040EDF5C02E1050E47
:10850000DF6EDF5008E0FC0EDBCFE9FFFD0EDBCFB6
:10851000EAFFEE6AED6ADF501D6E0F0EE15C02E2CB
:10852000E16AE552E16E1D50E552E5CFDAFFE7CF93
:10853000D9FF1200D9CFE6FFDACFE6FFE1CFD9FFAE
:10854000E2CFDAFF0D0EE12402E3E168E652E16ECC
:10855000FC0EDBCFE6FFFD0EDBCFE6FFCFEC29F014
:10856000E552E552DF6EDF5001E085D0D950FA0FB9
:10857000E96EFF0EDA20EA6EEE50ED1011E1000E0A
:10858000E66EE66AFC0EDBCFE6FFFD0EDBCFE6FF14
:10859000D4EC14F0E552E552E552E552DF6E6BD0B3
:1085A000D950010F1D6E000EDA201E6EFC0EDBCFBF
:1085B000E9FFFD0EDBCFEAFF140EE926000EEA22EA
:1085C0001DC0EEFF1EC0EDFFE66EE66AFC0EDBCFBF
:1085D000E6FFFD0EDBCFE6FF7BEC1CF0E552E5523B
:1085E000E552E552DF6E040EDF5C0FE1FC0EDBCFDF
:1085F000E9FFFD0EDBCFEAFF0E0EE926000EEA22B0
:10860000EE6AEE6AEE6AEE6ADF6ADF5034E1FA0E75
:10861000DBCFE6FFFB0EDBCFE6FFFC0EDBCFE6FF9A
:10862000FD0EDBCFE6FF92EC1FF0E552E552E5527E
:10863000E552000EE66EE66AFC0EDBCFE6FFFD0EAD
:10864000DBCFE6FF44EC17F0E552E552E552E55288
:10865000DF6E040EDF5C0FE1FC0EDBCFE9FFFD0EE9
:10866000DBCFEAFF0E0EE926000EEA22EE6AEE6A82
:10867000EE6AEE6ADF6ADF501D6E0D0EE15C02E20B
:10868000E16AE552E16E1D50E552E5CFDAFFE7CF32
:04869000D9FF1200FC
:0C869400D9CFE6FFDACFE6FFE1CFD9FF37
:1086A000E2CFDAFFE652E652E652E652E652D950FF
:1086B000030FE66E000EDA20E66E100EE66EE66A36
:1086C000000EE66E0A0EE66EB00EE66E060EE66E62
:1086D00072EC2DF01D6E080EE15C02E2E16AE552DB
:1086E000E16E1D50DF6EDF5001E0A0D0030EDBCF46
:1086F0001DF0040EDBCF1EF0100E1D5C000E1E5888
:1087000001E294D00A01005103E0FF0E005D48E150
:108710000C513AE10D5138E10E5136E10F5134E17F
:108720000251E66ED950010FE96E000EDA20EA6EB2
:10873000E552E750EE6EED6A03CA1DF003CA1EF063
:108740001D6AD950010FE96E000EDA20EA6E1D5045
:10875000EE121E50ED12010EDBCF1DF0020EDBCF2C
:108760001EF0100E1D5C000E1E580EE3D950010FB6
:10877000E96E000EDA20EA6E000ED880EE54400E4C
:10878000ED5402E3010E5DD0780E0C5D09E1560E4A
:108790000D5D06E1340E0E5D03E1120E0F5D46E045
:1087A000005105E1FE0E015D02E1030E4AD0E668CC
:1087B000210EE66EE66AE66AB00EE66E060EE66E1C
:1087C0001CEC39F01D6E060EE15C02E2E16AE55236
:1087D000E16E1D50DF6EDF501CE1D950030FE66ED5
:1087E000000EDA20E66E080EE66EE66A000EE66E11
:1087F0000A0EE66EB00EE66E060EE66E72EC2DF018
:108800001D6E080EE15C02E2E16AE552E16E1D5068
:10881000DF6EDF500BE1030EDBCF1DF0040EDBCF6C
:108820001EF0080E1D5C000E1E5802E2000E09D05C
:108830000A01005103E0FF0E005D02E1020E01D0CB
:10884000030E1D6E050EE15C02E2E16AE552E16E87
:108850001D50E552E5CFDAFFE7CFD9FF1200D9CF9F
:10886000E6FFDACFE6FFE1CFD9FFE2CFDAFFE6524B
:10887000E652E652E652126AD950FB0FE96EFF0E3D
:10888000DA20EA6EEE50ED1006E1FD0EDB50080135
:10889000F75D01E121D1FF0E0801F75D0AE0B00E9E
:1088A000E66E060EE66EF7EC38F0E552E55208018A
:1088B000F769D950FB0FE96EFF0EDA20EA6EEE5031
:1088C000ED1028E0FB0EDBCFE9FFFC0EDBCFEAFF6B
:1088D000EF5020E0FB0EDBCFE6FFFC0EDBCFE6FF28
:1088E000FD0EDB50190DF3CFE9FFF4CFEAFF2F0E99
:1088F000E926080EEA22EE52E9CF1DF0EACF1EF07B
:10890000E9CFE6FFEACFE6FF2FEC6EF0E552E55245
:10891000E552E552010EE66EFD0EDB50190DF3CF68
:10892000E9FFF4CFEAFF2F0EE926080EEA22EE5205
:10893000E9CF1DF0EACF1EF0E9CFE6FFEACFE6FF70
:10894000B00EE66E060EE66E8CEC2AF01F6E050E7B
:10895000E15C02E2E16AE552E16E1F50E76E030E50
:10896000E7CFDBFFDB5002E0180E48D0FD0EDBCF77
:10897000F7F8D950FB0FE96EFF0EDA20EA6EEE50E1
:10898000ED1001E1A9D0FD0EDBCFE6FF83DEE5525D
:10899000E66EFD0EDB50190DF3CFE9FFF4CFEAFFD1
:1089A0002F0EE926080EEA22E552E750EF6EE66A3E
:1089B000E66AE66AE66AB00EE66E060EE66E1CEC45
:1089C00039F01D6E060EE15C02E2E16AE552E16EED
:1089D0001D50FD0EDB50190DF3CFE9FFF4CFEAFF78
:1089E0002F0EE926080EEA22EF50030A3DE0010AA5
:1089F00021E0030A05E0010A54E1080E126E6CD072
:108A0000D950020FE66E000EDA20E66ED950010F43
:108A1000E66E000EDA20E66ED9CFE6FFDACFE6FF8B
:108A2000FD0EDBCFE6FF74EC49F01D6E070EE15C36
:108A300036E233D0D950020FE66E000EDA20E66E31
:108A4000D950010FE66E000EDA20E66ED9CFE6FFB0
:108A5000DACFE6FFFD0EDBCFE6FF18EC4EF01D6E21
:108A6000070EE15C1CE219D0D950020FE66E000E31
:108A7000DA20E66ED950010FE66E000EDA20E66EBF
:108A8000D9CFE6FFDACFE6FFFD0EDBCFE6FF8EECB7
:108A900051F01D6E070EE15C02E2E16AE552E16E03
:108AA0001D50DFCF00FA010EDBCF01FA020EDBCF43
:108AB00002FA0A01010E036FFD0EDB50190DF3CF10
:108AC000E9FFF4CFEAFF2F0EE926080EEA22EFCFE6
:108AD00004FA050E136E146A040EE15C02E2E16A08
:108AE000E552E16EE552E5CFDAFFE7CFD9FF12009C
:108AF000D9CFE6FFDACFE6FFE1CFD9FFE2CFDAFF49
:108B0000E65200CADFFFDF50070850E3156A0A018A
:108B10000151010A0AE0010A69E1020EE66E0A0E3D
:108B2000E66EDFCFE6FF9BDE5ED0DF500801F75D2B
:108B30002AE0000EE66EE66ADFCFE6FF90DEE55241
:108B4000E552E552DF50190DF3CFE9FFF4CFEAFF0C
:108B50002F0EE926080EEA22EF0413E1DF50190D6B
:108B6000F3CFE9FFF4CFEAFF2F0EE926080EEA2241
:108B70000E0EE926000EEA22020EE926000EEA2277
:108B8000EF68125033E1DF50190DF3CFE9FFF4CF56
:108B9000EAFF2F0EE926080EEA22EF50030A1BE037
:108BA000010A10E0030A05E0010A20E1050E126E39
:108BB0001DD003CAE6FF02CAE6FFDFCFE6FF38ECAE
:108BC0004AF011D003CAE6FF02CAE6FFDFCFE6FF94
:108BD00097EC50F008D003CAE6FF02CAE6FFDFCFE9
:108BE000E6FFB4EC51F0E552E552E552E552E552AC
:108BF000E5CFDAFFE7CFD9FF1200D9CFE6FFDACF12
:108C0000E6FFE1CFD9FFE2CFDAFF070EE12402E36E
:108C1000E168E652E16EFD0EDB50190DF3CFE9FF7E
:108C2000F4CFEAFF2F0EE926080EEA220E0EE926FF
:108C3000000EEA22E9CFDEFFEACFDDFFFC0EDB50BB
:108C4000E66ED950020FE96E000EDA20EA6EE552A8
:108C5000E750EE6EED6ADECFE9FFDDCFEAFF040EEE
:108C6000E926000EEA22EF500CE1D950020FE96E1E
:108C7000000EDA20EA6E010ED890EE36ED36E806E8
:108C8000FBE1FB0EDB501D6E1E6AD950020FE96E30
:108C9000000EDA20EA6E1D50EE261E50ED22020E66
:108CA000DBCF1DF0030EDBCF1EF01F6A206ADECF84
:108CB000E9FFDDCFEAFF070EE926000EEA221DC01C
:108CC000EEFF1EC0EEFF1FC0EEFF20C0EEFFDECFA6
:108CD000E9FFDDCFEAFFEECF1DF0EFCF1EF01F6AF8
:108CE000206ADECFE9FFDDCFEAFF070EE926000E9E
:108CF000EA221DC040F01EC041F01FC042F020C05B
:108D000043F0EECF3BF0EECF3CF0EECF3DF0EFCFB7
:108D10003EF0CEEC6FF03AC0EDFF39C0EDFF38C049
:108D2000EDFF37C0EFFFDECFE9FFDDCFEAFF070E33
:108D3000E926000EEA22100EEE26000EEE22EE22AA
:108D4000EE22DECFE9FFDDCFEAFF070EE926000EB7
:108D5000EA22EECFE6FFEECFE6FFEECFE6FFEFCF63
:108D6000E6FFB00EE66E060EE66E1CEC39F01D6EE8
:108D7000060EE15C02E2E16AE552E16E1D50E76E2B
:108D8000040EE7CFDBFFDB501FE1D950050FE66E85
:108D9000000EDA20E66E800EE66EE66AD20EE66E11
:108DA000060EE66EB00EE66E060EE66E72EC2DF066
:108DB0001D6E080EE15C02E2E16AE552E16E1D50B3
:108DC000E76E040EE7CFDBFF040EDB500BE1050E70
:108DD000DBCF1DF0060EDBCF1EF0800E1D5C000EFB
:108DE0001E5803E2050E126E17D0DECFE9FFDDCF6D
:108DF000EAFF020EE926000EEA22FC0EDBCFEFFFAF
:108E0000DECFE9FFDDCFEAFF030EE926000EEA22FE
:108E1000FB0EDBCFEFFF126A12501E6A12C0F3FF87
:108E20001EC0F4FF070EE15C02E2E16AE552E16E6A
:108E3000E552E5CFDAFFE7CFD9FF1200D9CFE6FF41
:108E4000DACFE6FFE1CFD9FFE2CFDAFF0F0EE12460
:108E500002E3E168E652E16EFD0EDB50190DF3CF3F
:108E6000E9FFF4CFEAFF2F0EE926080EEA220E0EE4
:108E7000E926000EEA22E9CFDEFFEACFDDFFFB0E96
:108E8000DBCFE9FFFC0EDBCFEAFF010EEF6EF90E40
:108E9000DBCFE9FFFA0EDBCFEAFF010EEF6EDECF8C
:108EA000E9FFDDCFEAFFEECF1DF0EFCF1EF0070E9A
:108EB0001DC0DBFF080E1EC0DBFF090EDB6A0A0EB9
:108EC000DB6AD950070FE96E000EDA20EA6E100E49
:108ED000EE26000EEE22EE22EE22D950070FE96EAA
:108EE000000EDA20EA6EEECFE6FFEECFE6FFEECF21
:108EF000E6FFEFCFE6FFB00EE66E060EE66E1CEC68
:108F000039F01D6E060EE15C02E2E16AE552E16EA7
:108F10001D50E76E060EE7CFDBFFDB501FE1D95097
:108F20000D0FE66E000EDA20E66E800EE66EE66A43
:108F3000D20EE66E060EE66EB00EE66E060EE66E1B
:108F400072EC2DF01D6E080EE15C02E2E16AE55262
:108F5000E16E1D50E76E060EE7CFDBFF060EDB501D
:108F60000CE00D0EDBCF1DF00E0EDBCF1EF0800EE1
:108F70001D5C000E1E5801E2ABD1DECFE9FFDDCF54
:108F8000EAFF060EE926000EEA22EF6A020EDB6A0D
:108F9000400EF36E020EDBCFF4FFF350F45C01E3FE
:108FA000FED0020EDB28EA6AD20FE96E060EEA2234
:108FB000EFCF1FF01FC020F01F6A020EDB50EA6ADD
:108FC000D20FE96E060EEA22EF5000011F241D6E3B
:108FD000000E20201E6E0B0E1DC0DBFF0C0E1EC0EF
:108FE000DBFFD9500B0FE96E000EDA20EA6EEE506F
:108FF000ED1001E1D4D00C0EDB50800B02E0010E2D
:1090000001D0000EE76E050EE7CFDBFFD9500B0F46
:10901000E96E000EDA20EA6EEE523F0EED16DECF5C
:10902000E9FFDDCFEAFF060EE926000EEA22EF2A6D
:10903000050EDB5007E0F90EDBCFE9FFFA0EDBCFC0
:10904000EAFFEF6ADECFE9FFDDCFEAFF050EE92692
:10905000000EEA22EF5005E1050EDB5002E1000EA2
:1090600001D0010E000902E0010E01D0020EE76EF0
:10907000040EE7CFDBFF0B0EDBCF1DF00C0EDBCFBA
:109080001EF01F6A206AD950070FE96E000EDA2021
:10909000EA6EEE501D26EE501E22EE501F22EE50BC
:1090A00020221DC0E6FF1EC0E6FF1FC0E6FF20C055
:1090B000E6FFB00EE66E060EE66E1CEC39F0216E91
:1090C000060EE15C02E2E16AE552E16E2150E76ED4
:1090D000060EE7CFDBFFDB501FE1D9500D0FE66E28
:1090E000000EDA20E66E0E0EE66EE66A000EE66E02
:1090F0000A0EE66EB00EE66E060EE66E72EC2DF00F
:109100001D6E080EE15C02E2E16AE552E16E1D505F
:10911000E76E060EE7CFDBFF060EDB5040E10D0EDB
:10912000DBCF1DF00E0EDBCF1EF01D5C000E1E58B7
:1091300036E3030EDB6ADB50EA6A000FE96E0A0EC3
:10914000EA22EF50FE0821E1030EDBCFE7FF040E19
:10915000DB50E726030EE7CFDBFFDBCFE7FF040E94
:10916000DB50E726030EE7CFDBFFDB50EA6A000F98
:10917000E96E0A0EEA22EF50010B07E0FB0EDBCF8F
:10918000E9FFFC0EDBCFEAFFEF6A020E1D6EDBCFBC
:10919000E7FFE850E726020EE7CFDBFFF9D6DECF88
:1091A000E9FFDDCFEAFF060EE926000EEA22EF50C6
:1091B0006BE1E66AE66AFD0EDBCFE6FF1EDDE552F7
:1091C000E552E552020EDB6A400EF36E020EDBCF73
:1091D000F4FFF350F45C58E2020EDB28EA6AD20F87
:1091E000E96E060EEA22EFCF1FF01FC020F01F6AC3
:1091F000020EDB50EA6AD20FE96E060EEA22EF5049
:109200001F241D6E000E20201E6E0B0E1DC0DBFFE6
:109210000C0E1EC0DBFFD9500B0FE96E000EDA20DA
:10922000EA6EEE50ED1030E00C0EDB50800B02E0E9
:10923000010E01D0000EE76E050EE7CFDBFFD9501F
:109240000B0FE96E000EDA20EA6EEE523F0EED16BD
:10925000DECFE9FFDDCFEAFF060EE926000EEA22A7
:10926000EF2A050EDB5007E0F90EDBCFE9FFFA0E1F
:10927000DBCFEAFFEF6A020EDBCFE7FFE850E7261D
:10928000020EE7CFDBFFA0D7DECFE9FFDDCFEAFF9D
:10929000050EE926000EEA22EF5008E0F90EDBCFBA
:1092A000E9FFFA0EDBCFEAFF010EEF6EDECFE9FF3A
:1092B000DDCFEAFF040EE926000EEA22EF5008E0B7
:1092C000FB0EDBCFE9FFFC0EDBCFEAFF010EEF6EFA
:1092D0000F0EE15C02E2E16AE552E16EE552E5CF94
:1092E000DAFFE7CFD9FF1200D9CFE6FFDACFE6FFEA
:1092F000E1CFD9FFE2CFDAFFE652E652E652E6527C
:10930000E652FD0EDB50190DF3CFE9FFF4CFEAFF73
:109310002F0EE926080EEA220E0EE926000EEA229A
:10932000E9CF1DF0EACF1EF0E9CFDEFFEACFDDFF87
:10933000D950030FE66E000EDA20E66E100EE66ED0
:10934000E66AD20EE66E060EE66EB00EE66E060E0B
:10935000E66E72EC2DF01D6E080EE15C02E2E16A31
:10936000E552E16E1D50E76E020EE7CFDBFFDB50EA
:109370000BE1030EDBCF1DF0040EDBCF1EF0100E51
:109380001D5C000E1E5803E2050E126E65D006012C
:10939000D305E66EFB0EDBCFE9FFFC0EDBCFEAFF69
:1093A000E552E750EF6E100ED615E66EDECFE9FF00
:1093B000DDCFEAFF040EE926000EEA22E552E7506F
:1093C000EF6E400ED615E66EDECFE9FFDDCFEAFF89
:1093D000050EE926000EEA22E552E750EF6ED5C6EB
:1093E0001FF0D5C620F01F6AD45100011F101D6E5A
:1093F000D5C61EF0DECFE9FFDDCFEAFFEE6E1EC060
:10940000EDFFDECFE9FFDDCFEAFF020EE926000E19
:10941000EA22EF68DECFE9FFDDCFEAFF030EE9269F
:10942000000EEA22EF68F70EDBCFE6FFF80EDBCF87
:10943000E6FFF90EDBCFE6FFFA0EDBCFE6FFFD0E0F
:10944000DBCFE6FFFBDC1D6E050EE15C02E2E16AAC
:10945000E552E16E1D50126A050EE15C02E2E16A1E
:10946000E552E16EE552E5CFDAFFE7CFD9FF120012
:10947000D9CFE6FFDACFE6FFE1CFD9FFE2CFDAFFBF
:10948000130EE12402E3E168E652E16EFD0EDB50CB
:10949000190DF3CFE9FFF4CFEAFF2F0EE926080EEE
:1094A000EA220E0EE926000EEA22EACF1EF0E9CFEC
:1094B000DEFFEACFDDFFDECFE9FFDDCFEAFF060EFC
:1094C000E926000EEA22EF50F36EFB0EDBCFF4FF2D
:1094D000F350F45C02E2000E01D0010EE76E020EC2
:1094E000E7CFDBFFDB5010E0DECFE9FFDDCFEAFFA7
:1094F000060EE926000EEA22FB0EDBCFE7FFEF5057
:10950000E75EFB0EE7CFDBFFDECFE9FFDDCFEAFF53
:10951000020EE926000EEA22EFCF1DF0FC0EDB5012
:109520001D5C0EE1DECFE9FFDDCFEAFF030EE92689
:10953000000EEA22EFCF1EF0020EDB501E5C14E09C
:10954000020EDBCFE6FFFC0EDBCFE6FFFD0EDBCF2E
:10955000E6FFFDEC45F0E552E552E552120EF3CF81
:10956000DBFFDB5001E056D3060EDB6A400EF36EE4
:10957000060EDBCFF4FFF350F45C01E34BD3060E91
:10958000DB28EA6AD20FE96E060EEA22EFCF1FF05F
:109590001FC020F01F6A060EDB50EA6AD20FE96E88
:1095A000060EEA22EF5000011F241D6E000E20203F
:1095B0001E6E030E1DC0DBFF040E1EC0DBFFD95064
:1095C000030FE96E000EDA20EA6EEE50ED1001E1B5
:1095D00021D3040EDB50800B02E0010E01D0000EFF
:1095E000E76E050EE7CFDBFFD950030FE96E000EE3
:1095F000DA20EA6EEE523F0EED16DECFE9FFDDCF48
:10960000EAFF050EE926000EEA22EF5005E1050EFD
:10961000DB5002E1000E01D0010E000902E0010E54
:1096200001D0020EE76E090EE7CFDBFF030EDBCFA2
:109630001DF0040EDBCF1EF01F6A206ADECFE9FFAB
:10964000DDCFEAFF070EE926000EEA22EE501D26C6
:10965000EE501E22EE501F22EE5020221DC0E6FFCB
:109660001EC0E6FF1FC0E6FF20C0E6FFB00EE66E9C
:10967000060EE66E1CEC39F0216E060EE15C02E28D
:10968000E16AE552E16E2150E76E120EE7CFDBFF93
:10969000DB501FE1D950100FE66E000EDA20E66EA7
:1096A0000E0EE66EE66A000EE66E0A0EE66EB00E6E
:1096B000E66E060EE66E72EC2DF01D6E080EE15C95
:1096C00002E2E16AE552E16E1D50E76E120EE7CF4D
:1096D000DBFF120EDB5001E09DD2100EDBCF1DF040
:1096E000110EDBCF1EF00E0E1D5C000E1E5801E2A7
:1096F00091D2070EDB6ADB50EA6A000FE96E0A0EB0
:10970000EA22EF50FE0801E07AD2070EDBCFE7FF36
:10971000090EDB50E726070EE7CFDBFFDB50EA6AD6
:10972000000FE96E0A0EEA22EFCF1DF0FC0EDB50AF
:109730001D5C01E064D2070EDBCFE7FF090EDB50B2
:10974000E726070EE7CFDBFFDB50EA6A000FE96E82
:109750000A0EEA22EF50010B1D6E020EDB501D5C5B
:1097600001E04DD2070EDBCFE7FF090EDB50E72605
:10977000070EE7CFDBFFDB50EA6A000FE96E0A0E47
:10978000EA22EFCF1DF0FB0EDB501D5C01E037D26B
:10979000070EDBCFE7FF090EDB50E726070EE7CF0A
:1097A000DBFFDBCFE7FF090EDB50E726070EE7CF35
:1097B000DBFFDBCFE7FF090EDB50E726070EE7CF25
:1097C000DBFFDBCFE7FF090EDB50E726070EE7CF15
:1097D000DBFF050EDB5002E02B0E01D01E0EE76E04
:1097E0000E0EE7CFDBFFDBCFE7FF090EDB50E70212
:1097F0000E0EF3CFDBFF070EDB50E76E030EDBCF61
:109800001DF0040EDBCF1EF0E7501D26000E1E22B9
:109810001F6A206ADECFE9FFDDCFEAFF070EE926E7
:10982000000EEA22EE501D26EE501E22EE501F22A0
:10983000EE5020221DC0E6FF1EC0E6FF1FC0E6FF5F
:1098400020C0E6FFB00EE66E060EE66E1CEC39F0A8
:10985000216E060EE15C02E2E16AE552E16E215002
:10986000E76E120EE7CFDBFFDB5020E1D950100F7F
:10987000E66E000EDA20E66E0E0EDBCFE6FFE66A3D
:10988000000EE66E0A0EE66EB00EE66E060EE66E90
:1098900072EC2DF01D6E080EE15C02E2E16AE55209
:1098A000E16E1D50E76E120EE7CFDBFF120EDB50AC
:1098B00001E0B0D1100EDBCF1DF0110EDBCF1EF09A
:1098C0000E0EDB50206AE8501D5C20501E5801E24D
:1098D000A1D10F0EDB68080EDB6A0E0EDB50F36EB3
:1098E000080EDBCFF4FFF350F45C2CE2F80E1D6E93
:1098F000080EDB50EA6A000FE96E0A0EEA22EF500A
:10990000D8801D5415E3080EDB50EA6A000FE96E9B
:109910000A0EEA22EF50FB080BE3080EDB50EA6A5E
:10992000000FE96E0A0EEA220F0EEFCFDBFF0AD01E
:10993000080EDBCFE7FF090EDB50E726080EE7CF66
:10994000DBFFCBD70F0EDB50FF0801E163D1080E20
:10995000DBCFE7FF090EDB50E726080EE7CFDBFF82
:10996000070EDB50E76E030EDBCF21F0040EDBCFDA
:1099700022F0E7502126000E2222080EDB500001C3
:1099800021241D6E000E22201E6E1F6A206ADECF6B
:10999000E9FFDDCFEAFF070EE926000EEA22EE50CE
:1099A0001D26EE501E22EE501F22EE5020221DC01A
:1099B000E6FF1EC0E6FF1FC0E6FF20C0E6FFB00EB8
:1099C000E66E060EE66E1CEC39F0236E060EE15CC8
:1099D00002E2E16AE552E16E2350E76E120EE7CF34
:1099E000DBFFDB5001E016D1090EDB0420E1D9508A
:1099F000100FE66E000EDA20E66EE66A010EE66EE5
:109A0000000EE66E0A0EE66EB00EE66E060EE66E0E
:109A100072EC2DF01D6E080EE15C02E2E16AE55287
:109A2000E16E1D50E76E120EE7CFDBFFD3D0D950A9
:109A30000A0FE96EDACFEAFF000EEA22000EEE6EA0
:109A40000A0EED6ED950100FE66E000EDA20E66EAB
:109A5000E66A010EE66E000EE66E090EE66EB00EC8
:109A6000E66E060EE66E72EC2DF01D6E080EE15CE1
:109A700002E2E16AE552E16E1D50E76E120EE7CF99
:109A8000DBFFDB5001E0C6D0100EDBCF1DF0110E66
:109A9000DBCF1EF0000E1D5C010E1E5801E2BAD095
:109AA000D9500C0FE96EDACFEAFF000EEA22000E61
:109AB000EE6E090EED6E080EDB6ADB501D6E1E6A3F
:109AC000D8901E5004E6800E1D5C000E1E581FE24A
:109AD0000C0EDBCFE9FFDB2A0D0EDBCFEAFF01E343
:109AE000DB2AEF50E66E0A0EDBCFE9FFDB2A0B0E16
:109AF000DBCFEAFF01E3DB2AE552E750EF6E0C0E05
:109B0000DB2A0D0E01E3DB2A080EDB2AD6D7D9505B
:109B1000100FE66E000EDA20E66EE66A010EE66EC3
:109B2000000EE66E090EE66EB00EE66E060EE66EEE
:109B300072EC2DF01D6E080EE15C02E2E16AE55266
:109B4000E16E1D50E76E120EE7CFDBFFDB5062E1E6
:109B5000100EDBCF1DF0110EDBCF1EF0000E1D5CD2
:109B6000010E1E5857E3D9500C0FE96EDACFEAFF09
:109B7000000EEA22000EEE6E090EED6E080EDB6A94
:109B8000DB501D6E1E6AD8901E5004E6800E1D5CD0
:109B9000000E1E581FE20C0EDBCFE9FFDB2A0D0E74
:109BA000DBCFEAFF01E3DB2AEF50E66E0A0EDBCFE4
:109BB000E9FFDB2A0B0EDBCFEAFF01E3DB2AE552EC
:109BC000E750EF6E0C0EDB2A0D0E01E3DB2A080EC8
:109BD000DB2AD6D70F0EDB50F80806E00F0EDB505D
:109BE000FA0802E0000E01D0010E000902E0060EA4
:109BF00001D0000E126E136A010E146E0DD0020E0B
:109C00001D6E060EDBCFE7FF1D50E726060EE7CFE1
:109C1000DBFFACD4050E126E130EE15C02E2E16ACA
:109C2000E552E16EE552E5CFDAFFE7CFD9FF12004A
:109C3000D9CFE6FFDACFE6FFE1CFD9FFE2CFDAFFF7
:109C4000080EE12402E3E168E652E16EFD0EDB500E
:109C5000190DF3CFE9FFF4CFEAFF2F0EE926080E26
:109C6000EA220E0EE926000EEA22060EE9CFDBFFFD
:109C7000070EEACFDBFFFB0EDBCFE9FFFC0EDBCFED
:109C8000EAFFEF6AF90EDBCFE9FFFA0EDBCFEAFF5E
:109C9000010EEF6EF70EDBCFE9FFF80EDBCFEAFF28
:109CA000010EEF6E060EDBCFE9FF070EDBCFEAFFFA
:109CB000EF6A010EDB6A020EDB6A010EDBCF1DF0DC
:109CC000020EDBCF1EF0550E1D5C0B0E1E5801E37D
:109CD000BFD0D950040FE66E000EDA20E66EFF0EFC
:109CE000E66EE66A000EE66E0A0EE66EB00EE66EF0
:109CF000060EE66E72EC2DF01D6E080EE15C02E2BF
:109D0000E16AE552E16E1D50E76E030EE7CFDBFF1F
:109D1000DB5001E0A4D0040EDBCF1DF0050EDBCF3D
:109D20001EF0FF0E1D5C000E1E5801E298D0DF6A87
:109D3000DF501D6E1E6AD8901E5004E6FF0E1D5C9B
:109D4000000E1E58BAE2010EDBCF1FF0020EDBCF71
:109D500020F0550E1F5C0B0E2058AFE2DF50EA6A70
:109D6000000FE96E0A0EEA22EF50FF0868E0DF50AC
:109D7000EA6A000FE96E0A0EEA22EFCF1DF0FB0E31
:109D8000DBCFE9FFFC0EDBCFEAFFEF50D8801D549C
:109D900011E2DF50EA6A000FE96E0A0EEA22EF5084
:109DA000E66EFB0EDBCFE9FFFC0EDBCFEAFFE552F0
:109DB000E750EF6EDF28EA6A000FE96E0A0EEA222A
:109DC000EFCF1DF0060EDBCFE9FF070EDBCFEAFF7A
:109DD000EF50D8801D5411E2DF28EA6A000FE96EC7
:109DE0000A0EEA22EF50E66E060EDBCFE9FF070E01
:109DF000DBCFEAFFE552E750EF6E020EDF24EA6A9E
:109E0000000FE96E0A0EEA22EF50800B07E0F70E12
:109E1000DBCFE9FFF80EDBCFEAFFEF6A020EDF24AB
:109E2000EA6A000FE96E0A0EEA22EF50100B07E013
:109E3000F90EDBCFE9FFFA0EDBCFEAFFEF6A030E84
:109E4000DF26010EDB2A020E01E272D7DB2A70D771
:109E5000060EDBCFE9FF070EDBCFEAFFEF2A080E85
:109E6000E15C02E2E16AE552E16EE552E5CFDAFF3C
:109E7000E7CFD9FF1200D9CFE6FFDACFE6FFE1CF77
:109E8000D9FFE2CFDAFF0A0EE12402E3E168E652ED
:109E9000E16EFD0EDB50190DF3CFE9FFF4CFEAFFC1
:109EA0002F0EE926080EEA220E0EE926000EEA22FF
:109EB000E9CF1DF0EACF1EF0E9CFDEFFEACFDDFFEC
:109EC000DECFE9FFDDCFEAFF020EE926000EEA222F
:109ED000EECFE6FFEECFE6FFEECFE6FFEFCFE6FFF9
:109EE000B00EE66E060EE66E1CEC39F01D6E060E28
:109EF000E15C02E2E16AE552E16E1D50E76E090E97
:109F0000E7CFDBFFDB504AE1DECFE9FFDDCFEAFF41
:109F1000020EE926000EEA22EE52220EEE26000E76
:109F2000EE22EE22020EDB6A030EDB6A020EDBCFAC
:109F30001DF0030EDBCF1EF0550E1D5C0B0E1E58E0
:109F400001E3E6D0D950070FE66E000EDA20E66E88
:109F5000FF0EE66EE66A000EE66E0A0EE66EB00EC4
:109F6000E66E060EE66E72EC2DF01D6E080EE15CDC
:109F700002E2E16AE552E16E1D50E76E090EE7CF9D
:109F8000DBFFDB500BE1070EDBCF1DF0080EDBCF54
:109F90001EF0FF0E1D5C000E1E5802E2000EB9D02E
:109FA000040EDB6A040EDB501D6E1E6AD8901E5034
:109FB00004E6FF0E1D5C000E1E58B8E2020EDBCF59
:109FC0001FF0030EDBCF20F0550E1F5C0B0E205848
:109FD000ADE2040EDB50EA6A000FE96E0A0EEA22D7
:109FE000EF50FF0847E0040EDB50EA6A000FE96E0D
:109FF0000A0EEA22EFCF1DF0FC0EDB501D5C3AE1A9
:10A00000040EDB28EA6A000FE96E0A0EEA22EFCF9F
:10A010001EF0FB0EDB501E5C2DE1040EDB50020F28
:10A02000EA6A000FE96E0A0EEA22EF50100B02E016
:10A03000010E01D0000EE76E060EE7CFDBFFDB500E
:10A04000F36EFA0EDB50F35C15E1040EDB50020FE9
:10A05000EA6A000FE96E0A0EEA22EF50E00BE66EA4
:10A06000DECFE9FFDDCFEAFFEE52E552E750EF6EBB
:10A07000010E4FD0040EDB50EA6A000FE96E0A0EA3
:10A08000EA22EF50FF0802E1020E01D0010E1D6E20
:10A09000040EDB50020FEA6A000FE96E0A0EEA2294
:10A0A000EF50030B1D18E76E050EE7CFDBFF800EA8
:10A0B0001D6E1E6A1F6A206A050EDB501F0B07E02B
:10A0C000D8901D361E361F362036E806F9E1DECF61
:10A0D000E9FFDDCFEAFF020EE926000EEA221D505D
:10A0E000EE261E50EE221F50EE222050EE22030ECE
:10A0F0001D6E040EDBCFE7FF1D50E726040EE7CFF1
:10A10000DBFF020EDB2A030E01E24CD7DB2A4AD723
:10A11000000E1D6E0A0EE15C02E2E16AE552E16E9C
:10A120001D50E552E5CFDAFFE7CFD9FF1200D9CFB6
:10A13000E6FFDACFE6FFE1CFD9FFE2CFDAFF060E86
:10A14000E12402E3E168E652E16EFD0EDB50190DF9
:10A15000F3CFE9FFF4CFEAFF2F0EE926080EEA223B
:10A160000E0EE926000EEA22E9CF1DF0EACF1EF01E
:10A17000E9CFDEFFEACFDDFFDECFE9FFDDCFEAFF8B
:10A18000EF50F36EFB0EDBCFF4FFF350F45C02E212
:10A19000000E01D0010EE76E050EE7CFDBFFDB50AE
:10A1A0000CE0DECFE9FFDDCFEAFFFB0EDBCFE7FF00
:10A1B000EF50E75EFB0EE7CFDBFFDECFE9FFDDCF41
:10A1C000EAFF020EE926000EEA22EE6AEE6AEE6A65
:10A1D000EE6A050EDBCFE6FFFB0EDBCFE6FFFC0EE3
:10A1E000DBCFE6FFFD0EDBCFE6FF45DEE552E552B5
:10A1F000E552E552000913E1050EDBCFE6FFFB0E49
:10A20000DBCFE6FFFC0EDBCFE6FFFD0EDBCFE6FF8C
:10A2100032DEE552E552E552E552000951E0DECF6B
:10A22000E9FFDDCFEAFF020EE926000EEA22EECFBB
:10A23000E6FFEECFE6FFEECFE6FFEFCFE6FFB00E94
:10A24000E66E060EE66E1CEC39F01D6E060EE15C45
:10A2500002E2E16AE552E16E1D50E76E020EE7CFC1
:10A26000DBFFDB501FE1D950030FE66E000EDA2052
:10A27000E66EE66A010EE66E000EE66E0A0EE66E09
:10A28000B00EE66E060EE66E72EC2DF01D6E080E38
:10A29000E15C02E2E16AE552E16E1D50E76E020EFA
:10A2A000E7CFDBFF020EDB500BE1030EDBCF1DF02F
:10A2B000040EDBCF1EF0000E1D5C010E1E5803E2E3
:10A2C000050E126E1FD0DECFE9FFDDCFEAFFEE52A2
:10A2D000EF50A00810E0DECFE9FFDDCFEAFFEE523D
:10A2E000EF50600808E0DECFE9FFDDCFEAFFEE5275
:10A2F000EF50200803E1060E126E01D0126A136AB5
:10A30000010E146E060EE15C02E2E16AE552E16EB6
:10A31000E552E5CFDAFFE7CFD9FF1200D9CFE6FF4C
:10A32000DACFE6FFE1CFD9FFE2CFDAFFFB0EDBCFDA
:10A33000E9FFFC0EDBCFEAFF230EEF6EF90EDBCF59
:10A34000E9FFFA0EDBCFEAFF010EEF6EF70EDBCF6F
:10A35000E9FFF80EDBCFEAFF010EEF6EE552E5CF25
:10A36000DAFFE7CFD9FF1200D9CFE6FFDACFE6FF59
:10A37000E1CFD9FFE2CFDAFFE652E652E652E652EB
:10A38000E652FD0EDB50190DF3CFE9FFF4CFEAFFE3
:10A390002F0EE926080EEA220E0EE926000EEA220A
:10A3A000E9CFDEFFEACFDDFF0A0EF36EFB0EDBCF57
:10A3B000F4FFF350F45C02E3050E9AD0FC0EDBCF01
:10A3C0001DF01E6A1F6A206ADECFE9FFDDCFEAFFBB
:10A3D0001DC0EEFF1EC0EEFF1FC0EEFF20C0EEFF4F
:10A3E000DECFE9FFDDCFEAFF0A0E406E416A426A26
:10A3F000436AEECF3BF0EECF3CF0EECF3DF0EFCF37
:10A400003EF0CEEC6FF03AC0EDFF39C0EDFF38C042
:10A41000EDFF37C0EFFFFB0EDBCF1DF01E6A1F6A9A
:10A42000206ADECFE9FFDDCFEAFF1D50EE261E5089
:10A43000EE221F50EE222050EE22DECFE9FFDDCFCC
:10A44000EAFFEF50EE6AEFCFF4FFEE6EEF50F4CF7D
:10A45000EEFFEF6EDECFE9FFDDCFEAFFEECFE6FFE6
:10A46000EECFE6FFEECFE6FFEFCFE6FFB00EE66EF3
:10A47000060EE66E1CEC39F01D6E060EE15C02E283
:10A48000E16AE552E16E1D50E76E020EE7CFDBFF99
:10A49000DB501FE1D950030FE66E000EDA20E66EA6
:10A4A000E66A010EE66E000EE66E0A0EE66EB00E6D
:10A4B000E66E060EE66E72EC2DF01D6E080EE15C87
:10A4C00002E2E16AE552E16E1D50E76E020EE7CF4F
:10A4D000DBFF020EDB500BE1030EDBCF1DF0040EA1
:10A4E000DBCF1EF0000E1D5C010E1E5803E2180E9D
:10A4F000126E0BD0136A010E146EFC0EDB501108A5
:10A5000002E1060E01D0000E126E050EE15C02E2C1
:10A51000E16AE552E16EE552E5CFDAFFE7CFD9FF18
:02A52000120027
:0EA52200D9CFE6FFDACFE6FFE1CFD9FFE2CFD7
:10A53000DAFFFD0EDB50C96EFD0EDB50046EC7A0C6
:10A54000FED78B80C9501C6E8B90E552E5CFDAFFA9
:10A55000E7CFD9FF1200D9CFE6FFDACFE6FFE1CF90
:10A56000D9FFE2CFDAFFE652E652010EDB6ADF6A7C
:10A57000040EDF5C15E2DF50B70DF3CFE9FFF4CF37
:10A58000EAFF320EE926030EEA222F0EE926000E1C
:10A59000EA22EF5003E0DE52010EDD6EDF2AE8D73B
:10A5A000010EDB50056EE552E552E552E5CFDAFFCC
:10A5B000E7CFD9FF1200D9CFE6FFDACFE6FFE1CF30
:10A5C000D9FFE2CFDAFFE652E652E652E652E65211
:10A5D000000EDE6E090EDD6EE66A010EE66EE66ABC
:10A5E000DECFE6FFDDCFE6FF15EC6EF01D6E050E4B
:10A5F000E15C02E2E16AE552E16E1D50DECFE9FF67
:10A60000DDCFEAFF560EEF6EDECFE9FFDDCFEAFFCA
:10A61000EE52CB0EEF6EDECFE9FFDDCFEAFF020E8A
:10A62000E926000EEA22100EEF6EDECFE9FFDDCF45
:10A63000EAFF040EE926000EEA22010EEF6EDECFDD
:10A64000E9FFDDCFEAFF050EE926000EEA22010E42
:10A65000EF6EDECFE9FFDDCFEAFF0A0EE926000E3E
:10A66000EA22430EEF6EF29CDECFE9FFDDCFEAFF78
:10A670000C0EE926000EEA228DC0EFFFDECFE9FFC7
:10A68000DDCFEAFF0D0EE926000EEA228CC0EFFFB7
:10A69000640E00018E25E66EDECFE9FFDDCFEAFF16
:10A6A0000E0EE926000EEA22E552E750EF6EF28C1C
:10A6B000DECFE9FFDDCFEAFF1B0EE926000EEA221E
:10A6C000030EEF6EDECFE9FFDDCFEAFF1C0EE926B9
:10A6D000000EEA22480EEF6EDECFE9FFDDCFEAFF83
:10A6E0001D0EE926000EEA22C00EEF6EDECFE9FF56
:10A6F000DDCFEAFF1E0EE926000EEA22080EEF6EFD
:10A70000DECFE9FFDDCFEAFF1F0EE926000EEA22C9
:10A71000010EEF6E530E1D6EE10E1E6E1F6A1DC000
:10A72000E6FFE66E1FC0E6FFDECFE9FFDDCFEAFF02
:10A73000200EE926000EEA22E9CF20F0EACF21F030
:10A74000E9CFE6FFEACFE6FF50EC6EF0226E050E91
:10A75000E15C02E2E16AE552E16E2250D950030F5A
:10A76000E66E000EDA20E66EE66A010EE66E000E78
:10A77000E66E090EE66EFC0EDBCFE6FFFD0EDBCFCC
:10A78000E6FF0DEC32F01D6E080EE15C02E2E16ABC
:10A79000E552E16E1D50E76E020EE7CFDBFFDB50A6
:10A7A00028E1FC0EDBCFE6FFFD0EDBCFE6FFD1ECB0
:10A7B00037F0E552E552E76E020EE7CFDBFFDB50E4
:10A7C00018E1E66AE66AE66AE66AFC0EDBCFE6FFB7
:10A7D000FD0EDBCFE6FF1CEC39F01D6E060EE15CD2
:10A7E00002E2E16AE552E16E1D50E76E020EE7CF2C
:10A7F000DBFF000E1D6E050EE15C02E2E16AE55230
:10A80000E16E1D50E552E5CFDAFFE7CFD9FF120028
:10A81000D9CFE6FFDACFE6FFE1CFD9FFE2CFDAFF0B
:10A820000C0EE12402E3E168E652E16EFD0EDB501E
:10A83000B70DF3CF1DF0F4CF1EF0320E1D26030E20
:10A840001E220A0E1DC0DBFF0B0E1EC0DBFF0A0E10
:10A85000DBCFE9FF0B0EDBCFEAFF2F0EE926000E60
:10A86000EA22EF5002E0000E84D2FD0EDB50B70D5D
:10A87000F3CFE9FFF4CFEAFF320EE926030EEA2216
:10A88000220EE926000EEA22E9CFDEFFEACFDDFF45
:10A89000DECFE9FFDDCFEAFFEF5030E14B0E1D6E5A
:10A8A000E10E1E6E1F6A1DC0E6FFE66E1FC0E6FFCA
:10A8B000DECFE6FFDDCFE6FF50EC6EF0206E050E3A
:10A8C000E15C02E2E16AE552E16E2050FD0EDB50F0
:10A8D000300FE66EDECFE9FFDDCFEAFF070EE92697
:10A8E000000EEA22E552E750EF6EDECFE9FFDDCF42
:10A8F000EAFF080EE926000EEA22EF6A030EF36E65
:10A90000070EF3CFDBFFFC0EDBA203D0070EF36EC6
:10A9100005D0DBA405D0010EF36E070EF3CFDBFFED
:10A92000070EDBCFE6FFDECFE6FFDDCFE6FF0A0E48
:10A93000DBCFE9FF0B0EDBCFEAFFE9CF1DF0EACF5B
:10A940001EF0E9CFE6FFEACFE6FF8CEC2AF01F6E9F
:10A95000050EE15C02E2E16AE552E16E1F50E76E2E
:10A96000020EE7CFDBFFDB5001E001D2FC0EDB5033
:10A97000030B58E10A0EDBCFE9FF0B0EDBCFEAFF3A
:10A98000370EE926000EEA22E9CF1DF0EACF1EF0CD
:10A990000A0EDBCFE9FF0B0EDBCFEAFF200EE92624
:10A9A000000EEA221DC0EEFF1EC0EDFF0A0EDBCF37
:10A9B000E9FF0B0EDBCFEAFF370EE926000EEA2295
:10A9C000200EEE6EEE6AEE6AEE6AE668E668E6680B
:10A9D000E6680A0EDBCFE9FF0B0EDBCFEAFFE9CF1B
:10A9E0001DF0EACF1EF0E9CFE6FFEACFE6FF1CEC50
:10A9F00039F01F6E060EE15C02E2E16AE552E16E9B
:10AA00001F50E76E020EE7CFDBFFDB500BE10A0EB3
:10AA1000DBCFE9FF0B0EDBCFEAFF2F0EE926000E9E
:10AA2000EA22EF82FC0EDBA218D00A0EDBCFE9FF90
:10AA30000B0EDBCFEAFFE9CF1DF0EACF1EF0E9CF26
:10AA4000E6FFEACFE6FFB7DDE552E552E76E020E1C
:10AA5000E7CFDBFFDB5001E078D1D950030FE66E82
:10AA6000000EDA20E66EE66A010EE66E000EE66E75
:10AA7000090EE66E0A0EDBCFE9FF0B0EDBCFEAFF15
:10AA8000E9CF1DF0EACF1EF0E9CFE6FFEACFE6FFFF
:10AA900072EC2DF01F6E080EE15C02E2E16AE552F5
:10AAA000E16E1F50E76E020EE7CFDBFFDB5001E0E7
:10AAB0004CD1D950030FE96E000EDA20EA6EEE5049
:10AAC00001E027D1010EED1801E023D1D950080F84
:10AAD000E96EDACFEAFF000EEA22000EEE6E090EF2
:10AAE000ED6E080EDBCFE9FF090EDBCFEAFFEF507A
:10AAF000560801E00ED1080EDBCFE9FF090EDBCFCF
:10AB0000EAFFEE52EF50CB0801E003D1080EDBCF95
:10AB1000E9FF090EDBCFEAFF020EE926000EEA226A
:10AB2000EF5010080EE0080EDBCFE9FF090EDBCF77
:10AB3000EAFF020EE926000EEA22EF50110801E0BA
:10AB4000E8D0FC0EDBA40CD00A0EDBCFE9FF0B0E25
:10AB5000DBCFEAFF320EE926000EEA22010E1DD0FD
:10AB6000080EDBCFE9FF090EDBCFEAFF070EE9266F
:10AB7000000EEA22EF50800B02E0010E01D0000E21
:10AB8000E66E0A0EDBCFE9FF0B0EDBCFEAFF320EDB
:10AB9000E926000EEA22E552E750EF6E080EDBCF01
:10ABA000E9FF090EDBCFEAFF1B0EE926000EEA22C1
:10ABB000EF50030B1E6E1D6A0A0EDBCFE9FF0B0E72
:10ABC000DBCFEAFF330EE926000EEA221DC0EEFFBE
:10ABD0001EC0EDFF080EDBCFE9FF090EDBCFEAFF59
:10ABE0001C0EE926000EEA22EF501D6E1E6A0A0EA8
:10ABF000DBCFE9FF0B0EDBCFEAFF330EE926000EB9
:10AC0000EA221D50EE261E50ED220A0EDBCFE9FF90
:10AC10000B0EDBCFEAFF360EE926000EEA22200EED
:10AC2000EF6E080EDBCFE9FF090EDBCFEAFF1D0E4A
:10AC3000E926000EEA22EF500EE0080EDBCFE9FF16
:10AC4000090EDBCFEAFF1D0EE926000EEA22EF50C7
:10AC50001D6E1E6A03D01D6A010E1E6E050E1DC0FC
:10AC6000DBFF060E1EC0DBFF0A0EDBCFE9FF0B0E7B
:10AC7000DBCFEAFF360EE926000EEA22EF501D6E0A
:10AC80001E6A050EDBCF3DF0060EDBCF3EF01DC089
:10AC900042F01EC043F088EC70F03D50E66E0A0EA4
:10ACA000DBCFE9FF0B0EDBCFEAFF350EE926000E06
:10ACB000EA22E552E750EF6E080EDBCFE9FF090EFE
:10ACC000DBCFEAFF1D0EE926000EEA22EFCF1DF0D2
:10ACD0000A0EDBCFE9FF0B0EDBCFEAFF360EE926CB
:10ACE000000EEA22EFCF1EF01EC043F01DC03EF062
:10ACF000CCEC70F03A500DE10A0EDBCFE9FF0B0E01
:10AD0000DBCFEAFF350EE926000EEA22EF500808F5
:10AD100006E2090EF36E020EF3CFDBFF16D00A0E29
:10AD2000DBCFE9FF0B0EDBCFEAFF300EEB6A310E13
:10AD3000EB6A0A0EDBCFE9FF0B0EDBCFEAFF2F0E2B
:10AD4000E926000EEA22EF8014D00A0EDBCFE9FFDD
:10AD50000B0EDBCFEAFFE9CF1DF0EACF1EF0E9CF03
:10AD6000E6FFEACFE6FFF7EC38F0E552E552020ED7
:10AD7000DB501D6E0C0EE15C02E2E16AE552E16E11
:10AD80001D50E552E5CFDAFFE7CFD9FF1200D9CF4A
:10AD9000E6FFDACFE6FFE1CFD9FFE2CFDAFFE652F6
:10ADA0000E6ADF6A040EDF5C27E2E66ADFCFE6FFA9
:10ADB0002FDDE552E55200091DE1010E056EDF5061
:10ADC000B70DF3CFE9FFF4CFEAFF320EE926030E09
:10ADD000EA22320EE926000EEA22EF500BE0800E46
:10ADE000DF5206E0DFCFF3FFE8327F0BF306FCE132
:10ADF00002090E6EDF2AD6D7ABEC52F0055002E006
:10AE0000000E01D0010EE552E552E5CFDAFFE7CFA3
:10AE1000D9FF1200D9CFE6FFDACFE6FFE1CFD9FFA5
:10AE2000E2CFDAFFE652E652FD0EDB50B70DF3CF6C
:10AE3000E9FFF4CFEAFF320EE926030EEA222F0ED5
:10AE4000E926000EEA22EF5037E0FD0EDB50B70D89
:10AE5000F3CFE9FFF4CFEAFF320EE926030EEA2230
:10AE6000E9CF1DF0EACF1EF0E9CFE6FFEACFE6FF1B
:10AE7000F7EC38F0E552E552FD0EDB50B70DF3CF9D
:10AE8000E9FFF4CFEAFF320EE926030EEA222F0E85
:10AE9000E926000EEA22EF6AFD0EDB50B70DF3CF74
:10AEA000E9FFF4CFEAFF320EE926030EEA22220E72
:10AEB000E926000EEA22EF6AABEC52F0E552E552C9
:10AEC000E552E5CFDAFFE7CFD9FF1200D9CFE6FF91
:10AED000DACFE6FFE1CFD9FFE2CFDAFFE652DF6A51
:10AEE000040EDF5C06E2DFCFE6FF94DFE552DF2AE7
:10AEF000F7D7E552E552E5CFDAFFE7CFD9FF1200E9
:10AF0000D9CFE6FFDACFE6FFE1CFD9FFE2CFDAFF14
:10AF1000070EE12402E3E168E652E16E0C50B70D42
:10AF2000F3CF1DF0F4CF1EF0320E1D26030E1E22AD
:10AF30001DC0DEFF1EC0DDFFDECFE9FFDDCFEAFF73
:10AF4000350EE926000EEA22EF500D5C0CE2DECF52
:10AF5000E9FFDDCFEAFF360EE926000EEA22EF50C8
:10AF6000D880095402E2130E12D1DECFE9FFDDCF03
:10AF7000EAFF360EE926000EEA22EFCF29F02A6A10
:10AF80002B6A2C6ADECFE9FFDDCFEAFF350EE9261A
:10AF9000000EEA22EFCF25F0266A276A286A0AC047
:10AFA00021F00BC022F0236A246A0AC03BF00BC0D8
:10AFB0003CF023C03DF024C03EF025C040F026C048
:10AFC00041F027C042F028C043F0CEEC6FF037C00C
:10AFD0001DF038C01EF039C01FF03AC020F037C055
:10AFE0003BF038C03CF039C03DF03AC03EF029C0DB
:10AFF00040F02AC041F02BC042F02CC043F0CEEC10
:10B000006FF0020E37C0DBFF030E38C0DBFF040E0B
:10B0100039C0DBFF050E3AC0DBFFDECFE9FFDDCF35
:10B02000EAFF360EE926000EEA22EFCF25F0266A67
:10B03000276A286A0D50216E226A236A246A0DC08D
:10B040003BF022C03CF023C03DF024C03EF025C0C0
:10B0500040F026C041F027C042F028C043F0CEECBB
:10B060006FF037C01DF038C01EF039C01FF03AC075
:10B0700020F0D950020FE96E000EDA20EA6E375048
:10B08000EE261E50EE221F50EE222050EE22DECF82
:10B09000E9FFDDCFEAFF360EE926000EEA22EFCF08
:10B0A00025F0266A276A286A0950216E226A236AD7
:10B0B000246A09C03BF022C03CF023C03DF024C00C
:10B0C0003EF025C040F026C041F027C042F028C025
:10B0D00043F02BEC70F038C01EF039C01FF03AC0BE
:10B0E00020F0D950020FE96E000EDA20EA6E3750D8
:10B0F000EE261E50EE221F50EE222050EE22D95096
:10B10000020FE96E000EDA20EA6EEF50EE6AEFCF22
:10B11000F4FFEE6EEF50F4CFEEFFEF6ED950020F5A
:10B12000E96E000EDA20EA6EEE52EE2A000EEE22F2
:10B13000EE22D950020FE96E000EDA20EA6EEECF51
:10B14000E6FFEECFE6FFEECFE6FFEFCFE6FFDECF86
:10B15000E9FFDDCFEAFFE9CF1DF0EACF1EF0E9CF2E
:10B16000E6FFEACFE6FF1CEC39F01F6E060EE15C4D
:10B1700002E2E16AE552E16E1F50E76E060EE7CF8C
:10B18000DBFFDB5003E0060EDB5001D0000E1D6E2E
:10B19000070EE15C02E2E16AE552E16E1D50E55204
:10B1A000E5CFDAFFE7CFD9FF1200D9CFE6FFDACF3C
:10B1B000E6FFE1CFD9FFE2CFDAFFE652E652E652F0
:10B1C000E652E6520C50B70DF3CF1DF0F4CF1EF04F
:10B1D000320E1D26030E1E221DC0DEFF1EC0DDFF27
:10B1E000D950020FE66E000EDA20E66EE66A010E16
:10B1F000E66E000EE66E090EE66EDECFE9FFDDCFED
:10B20000EAFFE9CF1DF0EACF1EF0E9CFE6FFEACF73
:10B21000E6FF72EC2DF01F6E080EE15C02E2E16ABF
:10B22000E552E16E1F50E76E040EE7CFDBFFDB5007
:10B2300017E1DECFE9FFDDCFEAFF300EE926000E91
:10B24000EA22EE50ED100CE0DECFE9FFDDCFEAFFA1
:10B25000300EE926000EEA22580EEE6E020EED6E5A
:10B26000040EDB501D6E050EE15C02E2E16AE55260
:10B27000E16E1D50E552E5CFDAFFE7CFD9FF1200AE
:10B28000D9CFE6FFDACFE6FFE1CFD9FFE2CFDAFF91
:10B29000E652E652E652E652E6520C50B70DF3CFB4
:10B2A0001DF0F4CF1EF0320E1D26030E1E221DC00F
:10B2B000DEFF1EC0DDFFD950020FE66E000EDA2061
:10B2C000E66EE66A010EE66E000EE66E090EE66EAA
:10B2D000DECFE9FFDDCFEAFFE9CF1DF0EACF1EF0B8
:10B2E000E9CFE6FFEACFE6FF0DEC32F01F6E080E65
:10B2F000E15C02E2E16AE552E16E1F50E76E040E86
:10B30000E7CFDBFFDB500FE1DECFE9FFDDCFEAFF68
:10B31000300EE926000EEA22580EEE6E020EED6E99
:10B320000801010EF96F040EDB501D6E050EE15C85
:10B3300002E2E16AE552E16E1D50E552E5CFDAFF27
:10B34000E7CFD9FF1200D9CFE6FFDACFE6FFE1CF92
:10B35000D9FFE2CFDAFFE652E652E652E652E65273
:10B36000DE52010EDD6E020EDB6ADF6A040EDF5C68
:10B3700065E2DF50B70DF3CF1DF0F4CF1EF0320EB3
:10B380001D26030E1E22030E1DC0DBFF040E1EC071
:10B39000DBFF030EDBCFE9FF040EDBCFEAFF2F0E4E
:10B3A000E926000EEA22EF5047E0010EF36E020E8E
:10B3B000F3CFDBFF030EDBCFE9FF040EDBCFEAFFA9
:10B3C000300EE926000EEA22EE50ED1035E0030EB5
:10B3D000DBCFE9FF040EDBCFEAFF300EE926000EDB
:10B3E000EA22EE06000EEF5A030EDBCFE9FF040E51
:10B3F000DBCFEAFF300EE926000EEA22EE50ED1018
:10B4000019E1F29E030EDBCFE9FF040EDBCFEAFF6A
:10B41000E9CF1DF0EACF1EF01DC0E6FF1EC0E6FF1B
:10B42000D1EC37F0E552E55281B202D006ED04F0DE
:10B43000F28E02D0010EDB6ADF2A98D7020EDB50B3
:10B4400005E0010EDB5002E00801F96B050EE15C3E
:10B4500002E2E16AE552E16EE552E5CFDAFFE7CFBD
:10B46000D9FF1200D9CFE6FFDACFE6FFE1CFD9FF4F
:10B47000E2CFDAFFE652DF6A040EDF5C1EE2B70EAF
:10B48000E66EE66AE66ADF50B70DF3CF1DF0F4CF43
:10B490001EF0320E1D26030E1E221DC0E6FF1EC02A
:10B4A000E6FF15EC6EF01F6E050EE15C02E2E16A4C
:10B4B000E552E16E1F50DF2ADFD7400EE66E91ECB9
:10B4C00052F0E552E552E552E5CFDAFFE7CFD9FF7A
:10B4D00012000150030A28E0010A1DE0030A16E0E9
:10B4E00001AC39D00F0E0114F66EF76AD890F6361B
:10B4F000F7365C0EF626E10EF7220900F5CF1DF0B7
:10B500000800F5CF1EF0010EE66E23D0F9DC00092D
:10B5100010E1500E3BD0580E026EF2DC000909E13A
:10B5200044DE000934E00CD0500E026EE9DC000964
:10B5300004E0510E026E100E06D0A2DE000927E0D4
:10B54000510E026E400E076E22D01EC0FAFF1D5033
:10B55000F96EFBDF1AD001AE1AD00F0E0114F66E91
:10B56000F76AD890F636F7365C0EF626E10EF7222B
:10B570000900F5CF1DF00800F5CF1EF0E66A04D0F3
:10B580001EC0FAFF1D50F96EFBDFE552026E02503D
:0AB59000E66E91EC52F0E552120055
:06B59A00D9CFE6FFDACF75
:10B5A000E6FFE1CFD9FFE2CFDAFFFD0EDB50C96E37
:10B5B000C7A0FED7C950E552E5CFDAFFE7CFD9FFE4
:10B5C0001200D9CFE6FFDACFE6FFE1CFD9FFE2CF15
:10B5D000DAFFE6520001640EA16FE668DEDFE55295
:10B5E000E668DBDFE552DF6EFF0EDF5C03E00001A3
:10B5F000A151F6E1DF50E552E552E5CFDAFFE7CFA2
:10B60000D9FF1200898AE668C8DFE55212001200ED
:10B61000899AD7DFF7DF0001CD811200D9CFE6FF8D
:10B62000DACFE6FFE1CFD9FFE2CFDAFF0801FC8FE6
:10B630000001280EA06FE668B0DFE5520001A56F9B
:10B64000FF0EA55D02E1A051F6E1FE0EA55D40E111
:10B6500000011A6B1B6BE668A0DFE552E66EFC0E7C
:10B66000DBCFE9FFFD0EDBCFEAFFE552E750EF6EDF
:10B67000FC0EDBCFE9FFFD0EDBCFEAFFEF50E66EFD
:10B6800018EC70F0E552FC0EDB2AFD0E01E3DB2A1C
:10B69000FA0EDB06DBCF1DF0FB0E01E2DB06DBCF93
:10B6A0001EF01D501E10D7E1E66877DFE55200015D
:10B6B000A66FE66872DFE5520001A76F1BC01DF0A0
:10B6C0001D50A65D05E100011A510001A75D02E0D1
:10B6D000000E01D0010EE552E5CFDAFFE7CFD9FF2A
:10B6E0001200D9CFE6FFDACFE6FFE1CFD9FFE2CFF4
:10B6F000DAFF67DFFF0857E1FB0EDBCFE6FF4DDF28
:10B70000E552FB0EDB50FD0850E00801F98F000107
:10B71000A96B020EAA6FFC0EDBCFABF0FD0EDBCFE8
:10B72000ACF000011A6B1B6B0001ABC0E9FFACC0B1
:10B73000EAFFAB2B000EAC23EF50E66E18EC70F076
:10B74000E5520001A907000EAA5BA951AA11ECE17C
:10B75000A96B020EAA6FFC0EDBCFE9FFDB2AFD0E00
:10B76000DBCFEAFF01E3DB2AEF50E66E16DFE5529E
:10B770000001A907000EAA5BA951AA11ECE11BC0A8
:10B780001DF01E6A1D50E66E08DFE5521AC0E6FF86
:10B7900004DFE552E66801DFE5520001A86F1F0EE5
:10B7A000A815050802E0000E01D0010EE552E5CF14
:10B7B000DAFFE7CFD9FF1200D9CFE6FFDACFE6FFF5
:10B7C000E1CFD9FFE2CFDAFFFD0EDBAE18D0FD0EE0
:10B7D000DB9EE66AE66AE66AE66A770EE66EECDF0C
:10B7E0001D6E050EE15C02E2E16AE552E16E1D505C
:10B7F0000001AE6F1D50010802E2AE519AD0898A55
:10B80000899ADFDEFF0802E0FF0E93D00001196B7A
:10B81000FD0EDBCFE6FFC1DEE552FD0EDBCFE6FF1E
:10B8200006EC70F0E552F90EDBCF1DF0FA0EDBCF1F
:10B830001EF0FB0EDBCF1FF0FC0EDBCF20F0180E4E
:10B84000D89020321F321E321D32E806F9E11DC0A9
:10B85000ADF01DC0E6FFA1DEE552ADC0E6FF06EC8F
:10B8600070F0E552F90EDBCF1DF0FA0EDBCF1EF0C3
:10B87000FB0EDBCF1FF0FC0EDBCF20F0100ED890BC
:10B8800020321F321E321D32E806F9E11DC0ADF034
:10B890001DC0E6FF82DEE552ADC0E6FF06EC70F0AB
:10B8A000E552F90EDBCF1DF0FA0EDBCF1EF0FB0EDA
:10B8B000DBCF1FF0FC0EDBCF20F0080ED89020323B
:10B8C0001F321E321D32E806F9E11DC0ADF01DC069
:10B8D000E6FF63DEE552ADC0E6FF06EC70F0E55230
:10B8E000F90EDBCFADF0ADC0E6FF57DEE552ADC0DF
:10B8F000E6FF06EC70F0E5520001199F1947198127
:10B9000019C0E6FF4ADEE552FD0EDB504C0803E1AC
:10B91000E66843DEE55200010A0EAD6FE6683DDEE3
:10B92000E5520001AE6F800EAE1502E0AD07F6E104
:10B93000AE51E552E5CFDAFFE7CFD9FF1200D9CFFC
:10B94000E6FFDACFE6FFE1CFD9FFE2CFDAFF070E5D
:10B95000E12402E3E168E652E16EFD0EDB5002E015
:10B96000010E20D10001CDB31CD151DE220EC66ED6
:10B970000A0EDF6EDF5005E0E6680FDEE552DF06F7
:10B98000F9D7020EDB6AE66AE66AE66AE66A400E04
:10B99000E66E12DF1D6E050EE15C02E2E16AE55221
:10B9A000E16E1D50010801E0D4D00001C80EA06F67
:10B9B000AA0EE66E010EE66EE66AE66A480EE66ECE
:10B9C000FBDE1D6E050EE15C02E2E16AE552E16E0E
:10B9D0001D50010873E1DF6A040EDF5C16E2E668C1
:10B9E000DCDDE552E66ED950030F1D6E000EDA2045
:10B9F0001E6EDF500F011D24E96E000E1E20EA6E40
:10BA0000E552E750EF6EDF2AE7D7050EDB0401E0D1
:10BA1000A0D0060EDB50AA0801E09BD00001A05187
:10BA200012E0E66AE66AE66A400EE66EE90EE66E47
:10BA3000C3DE1D6E050EE15C02E2E16AE552E16ED5
:10BA40001D500009EBE10001A05101E182D0E66A3E
:10BA5000E66AE66AE66A7A0EE66EAEDE1D6E050EF0
:10BA6000E15C02E2E16AE552E16E1D50000971E11C
:10BA7000DF6A040EDF5C16E2E6688FDDE552E66EF3
:10BA8000D950030F1D6E000EDA201E6EDF500F011D
:10BA90001D24E96E000E1E20EA6EE552E750EF6E9F
:10BAA000DF2AE7D7030EDB50400B02E00C0E01D07B
:10BAB000040EE76E020EE7CFDBFF4BD0E66AE66AC4
:10BAC000E66AE66AE90EE66E77DE1D6E050EE15C5B
:10BAD00002E2E16AE552E16E1D50010806E3020E42
:10BAE000F36EDB6EDE52E90E07D0010EF36E020E2E
:10BAF000F3CFDBFFDE52410EDD6E0001A05112E0FC
:10BB0000E66AE66AE66AE66A010EDBCFE6FF54DE25
:10BB10001D6E050EE15C02E2E16AE552E16E1D5028
:10BB20000009EBE10001A05112E0E66A020EE66EA8
:10BB3000E66AE66A500EE66E3FDE1D6E050EE15CBB
:10BB400002E2E16AE552E16E1D50000902E0020ED8
:10BB5000DB6A020EDB500001A26FA36B53DD020E05
:10BB6000DB501AE0200EC66E010EE66EE66AE66A4B
:10BB7000E66A7B0EE66E20DE1D6E050EE15C02E2DB
:10BB8000E16AE552E16E1D50DF6EDF5003E1000116
:10BB9000CD9102D0020EDB6A020EDB5001E138DDEE
:10BBA0000001CD511D6E070EE15C02E2E16AE55233
:10BBB000E16E1D50E552E5CFDAFFE7CFD9FF120065
:10BBC000D9CFE6FFDACFE6FFE1CFD9FFE2CFDAFF48
:10BBD000FD0EDB5002E0010E02D00001CD51E55216
:10BBE000E5CFDAFFE7CFD9FF1200D9CFE6FFDACFF2
:10BBF000E6FFE1CFD9FFE2CFDAFFFD0EDB5003E134
:10BC0000F60EDB0402E0040E5AD00001CDA102D0F2
:10BC1000030E55D00001A251080B12E1D950F70FC5
:10BC2000E96EFF0EDA20EA6E090EE76ED890EF3665
:10BC3000010EEB36020EEB36030EEB36E706F6E1AD
:10BC40000001200EA46FD950F70FE96EFF0EDA2025
:10BC5000EA6EEECFE6FFEECFE6FFEECFE6FFEFCFE8
:10BC6000E6FF510EE66EA8DD1D6E050EE15C02E2F8
:10BC7000E16AE552E16E1D50000912E1E66A020E2A
:10BC8000E66EFB0EDBCFE6FFFC0EDBCFE6FFC6DC8D
:10BC9000E552E552E552E552000902E0F60EDB6A94
:10BCA000B1DCF60EDB5005E00001A451A40700084A
:10BCB000CAE3F60EDB5002E0010E01D0000EE552A1
:10BCC000E5CFDAFFE7CFD9FF1200D9CFE6FFDACF11
:10BCD000E6FFE1CFD9FFE2CFDAFFFD0EDB5003E153
:10BCE000F60EDB0402E0040E5CD00001CDA102D010
:10BCF000030E57D0CDA502D0020E53D00001A251A1
:10BD0000080B12E1D950F70FE96EFF0EDA20EA6E48
:10BD1000090EE76ED890EF36010EEB36020EEB36C9
:10BD2000030EEB36E706F6E10001200EA46FD950B2
:10BD3000F70FE96EFF0EDA20EA6EEECFE6FFEECFE8
:10BD4000E6FFEECFE6FFEFCFE6FF580EE66E34DDFE
:10BD50001D6E050EE15C02E2E16AE552E16E1D50E6
:10BD6000000910E1FE0EE66EFB0EDBCFE6FFFC0ED7
:10BD7000DBCFE6FFB6DCE552E552E552000902E012
:10BD8000F60EDB6A3FDCF60EDB5005E00001A45145
:10BD9000A4070008CCE3F60EDB5002E0010E01D050
:10BDA000000EE552E5CFDAFFE7CFD9FF1200D9CF79
:10BDB000E6FFDACFE6FFE1CFD9FFE2CFDAFF180ED8
:10BDC000E12402E3E168E652E16EFA0EDBCF3DF0DA
:10BDD000FB0EDBCF3EF0120E3DC0DBFF130E3EC06C
:10BDE000DBFFFD0EDB5002E0040EE2D20001CDA12C
:10BDF00002D0030EDDD2010EDF6EFC0EDB500E0A08
:10BE000001E1A4D2030A01E16DD2010A01E146D2A7
:10BE1000070A01E11DD2010A01E111D2090A01E17B
:10BE20001CD1010A01E10FD1030A0AE0010A01E075
:10BE3000BAD2899AE1EC5AF0FF0801E0B6D2B1D249
:10BE4000E66AE66AE66AE66A490EE66EB5DC1D6EEB
:10BE5000050EE15C02E2E16AE552E16E1D50000967
:10BE600001E0A3D2100EE66EE66AD950020FE66E2C
:10BE7000000EDA20E66E0EEC5BF0E552E552E5527C
:10BE8000E552000901E191D2060E1D6E020EDB5053
:10BE90001DC0E7FFE75204E0E8427F0BE706FCE144
:10BEA000010856E10A0EDBCF25F025C026F0256AF1
:10BEB0000B0EDB5000012524216E000E2620226E81
:10BEC000236A246A090EDB503F0B276E286A296A11
:10BED0002A6A100E1F0B07E0D8902736283629361D
:10BEE0002A36E806F9E1215027241D6E2250282029
:10BEF0001E6E235029201F6E24502A20206E1D2ADA
:10BF0000000E1E221F222022140E1DC0DBFF150E64
:10BF10001EC0DBFF160E1FC0DBFF170E20C0DBFFAD
:10BF2000140EDBCF1DF0150EDBCF1EF0160EDBCF8F
:10BF30001FF0170EDBCF20F00A0E1F0B01E170D1AE
:10BF4000D8901D361E361F362036E806F9E168D136
:10BF50000C0EDB50216E226A800E2116000E221676
:10BF6000070ED89022322132E804FBE1070EDB50A5
:10BF70000F0B21241F6E000E2220206E0B0EDB50B3
:10BF8000030BE8241F241D6E000E20201E6E020EDF
:10BF90001D26000E1E22010E1DC0DBFF090EDB5008
:10BFA000226E236AD89022362336D8902236233642
:10BFB000060E216E0A0EDB5021C0E7FFE75204E0B7
:10BFC000E8427F0BE706FCE1000122241F6E000E11
:10BFD0002320206E080EDB50030B246E256A0A0E08
:10BFE000D89024362536E804FBE11F5024241D6E2A
:10BFF000205025201E6E010E1D26000E1E22140E3E
:10C000001DC0DBFF150E1EC0DBFF160EDB6A170E10
:10C01000DB6A140EDBCF1DF0150EDBCF1EF0160E03
:10C02000DBCF1FF0170EDBCF20F0010EDB50F70F38
:10C030001F0B01E1F5D0D8901D361E361F36203675
:10C04000E806F9E1EDD0FA0EDBCFE9FFFB0EDBCF1E
:10C05000EAFFEE6A020EED6EA4D10001A251040BBC
:10C0600049E0E66AE66AE66AE66ACD0EE66EDCEC70
:10C070005BF01D6E050EE15C02E2E16AE552E16EE5
:10C080001D50000901E091D1E668CDEC5AF0E5526F
:10C09000100EE66EE66AD950020FE66E000EDA2048
:10C0A000E66E0EEC5BF0E552E552E552E552000912
:10C0B00001E17BD1DE52300EDD6E010EDB5007E078
:10C0C000E668CDEC5AF0E552010EDB06F6D7100E0D
:10C0D0001D6E1E6A1F6A206A0C0EDB380F0B1F0BC9
:10C0E00001E19ED0D8901D361E361F362036E80658
:10C0F000F9E196D0E66AE66AE66AE66A490EE66E15
:10C10000DCEC5BF01D6E050EE15C02E2E16AE552DB
:10C11000E16E1D50000901E048D1100EE66EE66A9E
:10C12000D950020FE66E000EDA20E66E0EEC5BF0E0
:10C13000E552E552E552E552000901E136D1000130
:10C14000A251020B34E00D0EDB50236E246A800EE8
:10C150002316000E2416070ED89024322332E8044A
:10C16000FBE10C0EDB503F0BE82400012324216E81
:10C17000000E2420226E010E2126000E2222060E21
:10C18000256E0F0EDB5025C0E7FFE75204E0E842C2
:10C190007F0BE706FCE1FF0F21C01DF022C01EF05F
:10C1A0003DE0D8901D361E36E804FBE137D00D0E79
:10C1B000DB50256E266AE00E2516000E2616050EAB
:10C1C000D89026322532E804FBE10D0EDB50030B3C
:10C1D000080DF35000012524236E000E2620246E46
:10C1E000010E2326000E24220C0EDB507C0BE840AF
:10C1F000E8403F0B216E226A010E2126000E22220A
:10C2000021C03DF022C03EF023C042F024C043F0E4
:10C210004FEC70F03BC01DF03CC01EF01F6A206A5E
:10C22000FA0EDBCFE9FFFB0EDBCFEAFF1DC0EEFF0E
:10C230001EC0EEFF1FC0EEFF20C0EEFFB2D0120EF8
:10C24000DBCFE9FF130EDBCFEAFFA2C0EFFFA9D0DF
:10C25000E66AE66AE66AE66A490EE66EDCEC5BF0E0
:10C260001D6E050EE15C02E2E16AE552E16E1D50D1
:10C27000000901E09AD0100EE66EE66AFA0EDBCFF6
:10C28000E6FFFB0EDBCFE6FF0EEC5BF0E552E5527E
:10C29000E552E552000901E188D083D0E66AE66AFA
:10C2A000E66AE66A4A0EE66EDCEC5BF01D6E050E91
:10C2B000E15C02E2E16AE552E16E1D50000975E1C0
:10C2C000100EE66EE66AFA0EDBCFE6FFFB0EDBCF62
:10C2D000E6FF0EEC5BF0E552E552E552E55200094F
:10C2E00064E05FD0E66AE66AE66AE66A7A0EE66EBF
:10C2F000DCEC5BF01D6E050EE15C02E2E16AE552EA
:10C30000E16E1D50000951E1010EDB6A040EF36E6F
:10C31000010EDBCFF4FFF350F45C43E2E668CDECB2
:10C320005AF0E552E66E010EDB50E76EFA0EDBCFF7
:10C33000E9FFFB0EDBCFEAFFE750E926000EEA2219
:10C34000E552E750EF6E010EDB2AE0D70001A25163
:10C35000040B2BE0E66AE66AE66AE66ACD0EE66E54
:10C36000DCEC5BF01D6E050EE15C02E2E16AE55279
:10C37000E16E1D50000919E1E668CDEC5AF0E55276
:10C38000400EE66EE66AFA0EDBCFE6FFFB0EDBCF71
:10C39000E6FF0EEC5BF0E552E552E552E55200098E
:10C3A00004E0DF6A02D0040EDF6E02EC5BF0DF50C7
:10C3B0001D6E180EE15C02E2E16AE552E16E1D506D
:10C3C000E552E5CFDAFFE7CFD9FF1200D9CFE6FF7C
:10C3D000DACFE6FFE1CFD9FFE2CFDAFFE652E6524D
:10C3E000E6520001A05101E0A007A15101E0A10720
:10C3F0000801F82BAFC0DEFFB0C0DDFF300E8114A6
:10C400000001AF6FB06BDECF1DF0DDCF1EF0E85046
:10C410001D1819E1B0511E1816E1020ECDC0DBFF48
:10C42000DF50200B03E0020EDB8402D0020EDB940F
:10C43000DF50100B04E0020EDB80DB8202D0020E24
:10C44000DB92DBCFCDF0E552E552E552E552E5CF88
:10C45000DAFFE7CFD9FF1200020E0001CD1501E08F
:04C46000000C010CBF
:0CC46400D9CFE6FFDACFE6FF580EE55214
:10C47000E5CFDAFFE7CFD9FF1200D9CFE6FFDACF59
:10C48000E6FF060E136E146A0A01020E006F0D0E0F
:10C49000016F060EF66EF76A0800F5CF02FA070E76
:10C4A000F66EF76A0800F5CF03FAFE0EF66EF7682F
:10C4B0000800F5CF04FAF668F7680800F5CF05FA2A
:10C4C000580EE552E5CFDAFFE7CFD9FF1200D9CFFA
:10C4D000E6FFDACFE6FF060E136E146AF29C88C000
:10C4E00000FA89C001FA8AC002FA8EC003FA8CC031
:10C4F00004FA8DC005FAF28C580EE552E5CFDAFF4A
:10C50000E7CFD9FF1200D9CFE6FFDACFE6FFE1CFC0
:10C51000D9FFE2CFDAFFFD0EDB5004E1060E136E09
:10C52000146A18D000CA92F001CA93F002CA94F0BB
:10C5300003CA98F004CA96F005CA97F00001010EEC
:10C54000956F920EE66E000EE66EDAEC67F0E5523D
:10C55000E5520080580EE552E5CFDAFFE7CFD9FF6C
:10C560001200D9CFE6FFDACFE6FFE1CFD9FFE2CF65
:10C57000DAFFFD0EDB0442E108012D510AE00E0E48
:10C58000E66E060EE66EF7EC38F0E552E55208016D
:10C590002D6B00CAE6FF010EE66E0A0EE66E0E0E69
:10C5A000E66E060EE66E8CEC2AF01D6E050EE15C62
:10C5B00002E2E16AE552E16E1D50126E1D5004E088
:10C5C000136A146A510E1BD00801010E2D6F040E60
:10C5D000136E146AE66EE66A180EE66E060EE66ED6
:10C5E000000EE66E0A0EE66EEAEC6DF01D6E060EAB
:10C5F000E15C02E2E16AE552E16E1D50580EE5523F
:10C60000E5CFDAFFE7CFD9FF1200D9CFE6FFDACFC7
:10C61000E6FFE1CFD9FFE2CFDAFFE652E6520801AA
:10C620002D512AE0D9CFE6FFDACFE6FF13C0E6FFAF
:10C6300014C0E6FF000EE66E0A0EE66E0E0EE66E03
:10C64000060EE66E72EC2DF01D6E080EE15C02E245
:10C65000E16AE552E16E1D50126E1D500FE1DECF12
:10C6600013F0DDCF14F0D9CFE9FFDACFEAFFEE50B7
:10C67000ED1006E1500E05D0040E126E510E01D0E1
:10C68000580EE552E552E552E5CFDAFFE7CFD9FF84
:10C690001200D9CFE6FFDACFE6FFE1CFD9FFE2CF34
:10C6A000DAFFE652E652FD0EDB5009E108012D519A
:10C6B00004E0136A010E146E2CD0040E27D0D9CFDB
:10C6C000E6FFDACFE6FF13C0E6FF14C0E6FF000E78
:10C6D000E66E0A0EE66E0E0EE66E060EE66E0DECC9
:10C6E00032F01D6E080EE15C02E2E16AE552E16E95
:10C6F0001D50126E1D500BE1DECF1DF0DDCF1EF080
:10C7000013501D5C14501E5804E2140E126E510E8C
:10C7100001D0580EE552E552E552E5CFDAFFE7CFFA
:10C72000D9FF1200D9CFE6FFDACFE6FFE1CFD9FF7C
:10C73000E2CFDAFFE652E652E652E652FD0EDB5059
:10C740002AE108012D5124E0040E136E146A14C668
:10C75000DFFF010E15C6DBFF020E16C6DBFF030E60
:10C7600017C6DBFF040EE66EE66AD9CFE6FFDACF26
:10C77000E6FF000EE66E0A0EE66EEAEC6DF01D6E48
:10C78000060EE15C02E2E16AE552E16E1D5037D02F
:10C79000040E126E32D0040EE66EE66A000EE66EED
:10C7A0000A0EE66ED9CFE6FFDACFE6FFEAEC6DF0CF
:10C7B0001D6E060EE15C02E2E16AE552E16E1D507B
:10C7C000D9CFE9FFDACFEAFFEECFE6FFEECFE6FF03
:10C7D000EECFE6FFEFCFE6FF0E0EE66E060EE66E3C
:10C7E0001CEC39F01D6E060EE15C02E2E16AE552D6
:10C7F000E16E1D50126E1D5002E0510E01D0580E18
:10C800001D6E040EE15C02E2E16AE552E16E1D502C
:10C81000E552E5CFDAFFE7CFD9FF1200D9CFE6FF27
:10C82000DACFE6FFE1CFD9FFE2CFDAFF08012D51E1
:10C830000FE00E0EE66E060EE66EF7EC38F0E552EF
:10C84000E552126EE85002E0510E03D008012D6B44
:10C85000500EE552E5CFDAFFE7CFD9FF1200D9CF6E
:10C86000E6FFDACFE6FFE1CFD9FFE2CFDAFFFD0E38
:10C87000DB5004E1020E136E146A1CD0150E0A017F
:10C88000005D18E1040E0A01015D14E1E668FE0E88
:10C89000E66E030EE66E07EC6FF0E552E552E552E8
:10C8A000E668E668030EE66E07EC6FF0E552E552C7
:10C8B000E552FF00580E00D0E552E5CFDAFFE7CF92
:10C8C000D9FF1200D9CFE6FFDACFE6FFE1CFD9FFDB
:10C8D000E2CFDAFFFD0EDB041AE1000EE66E0A0E6F
:10C8E000E66E000EE66E080EE66E86EC41F0E5524E
:10C8F000E552E552E552126EE85006E0136A146AFA
:10C9000008012C6B510E04D00801010E2C6F580E3B
:10C91000E552E5CFDAFFE7CFD9FF1200D9CFE6FF26
:10C92000DACFE6FFE1CFD9FFE2CFDAFF08012C51E1
:10C9300003E1050E126E11D0160EE66E080EE66EBD
:10C94000000EE66E080EE66E9AEC42F0E552E552F5
:10C95000E552E552126EE85002E0510E1ED0080179
:10C960001F5102E1500E19D0160E136E146AE66EB6
:10C9700014C0E6FF160EE66E080EE66E000EE66EBA
:10C980000A0EE66EEAEC6DF01D6E060EE15C02E248
:10C99000E16AE552E16E1D50580EE552E5CFDAFF2F
:10C9A000E7CFD9FF1200D9CFE6FFDACFE6FFE1CF1C
:10C9B000D9FFE2CFDAFFE652FD0EDB043FE1030EC2
:10C9C000135C000E145805E300CADFFF040EDF5CA1
:10C9D00003E3130E126E30D0DFCFE6FF0AEC57F000
:10C9E000E552020EE66E0A0EE66EDF50B70DF3CF8B
:10C9F000E9FFF4CFEAFF320EE926030EEA22220E07
:10CA0000E926000EEA22E9CF1DF0EACF1EF0E9CFB9
:10CA1000E6FFEACFE6FF2FEC6EF0E552E552E55275
:10CA2000E55201CAE6FF00CAE6FF08EC54F0E55201
:10CA3000E552126EE85002E0510E01D0580EE55258
:10CA4000E552E5CFDAFFE7CFD9FF1200D9CFE6FFF5
:10CA5000DACFE6FFE1CFD9FFE2CFDAFFE652E652C6
:10CA6000E652FD0EDB5001E0E8D0136A146ADF6A7B
:10CA7000040EDF5C01E3E1D0DF50B70DF3CF1DF012
:10CA8000F4CF1EF0320E1D26030E1E22010E1DC015
:10CA9000DBFF020E1EC0DBFF010EDBCFE9FF020E43
:10CAA000DBCFEAFF2F0EE926000EEA22EF50E66EFA
:10CAB00013C0E9FF14C0EAFF132A000E1422000E6F
:10CAC000E9260A0EEA22E552E750EF6E010EDBCFAF
:10CAD000E9FF020EDBCFEAFF320EE926000EEA2262
:10CAE000EF50E66E13C0E9FF14C0EAFF132A000EF0
:10CAF0001422000EE9260A0EEA22E552E750EF6EF4
:10CB0000010EDBCFE9FF020EDBCFEAFF330EE92691
:10CB1000000EEA22EECF1DF0EFCF1EF01EC01DF07A
:10CB20001E6A13C0E9FF14C0EAFF132A1422000E84
:10CB3000E9260A0EEA221DC0EFFF010EDBCFE9FF56
:10CB4000020EDBCFEAFF330EE926000EEA22EECF1B
:10CB50001DF0EFCF1EF0FF0E1D16000E1E1613C0A7
:10CB6000E9FF14C0EAFF132A1422000EE9260A0E78
:10CB7000EA221DC0EFFF010EDBCFE9FF020EDBCF83
:10CB8000EAFF350EE926000EEA22EF50E66E13C0EA
:10CB9000E9FF14C0EAFF132A000E1422000EE92652
:10CBA0000A0EEA22E552E750EF6E010EDBCFE9FFF5
:10CBB000020EDBCFEAFF360EE926000EEA22EF5026
:10CBC000E66E13C0E9FF14C0EAFF132A000E142218
:10CBD000000EE9260A0EEA22E552E750EF6E0D0E2E
:10CBE000E66EE66A010EDBCFE9FF020EDBCFEAFF5D
:10CBF000220EE926000EEA22E9CF1DF0EACF1EF050
:10CC0000E9CFE6FFEACFE6FF000E13241F6E0A0EFF
:10CC10001420206E1FC0E6FFE66EEAEC6DF0216E78
:10CC2000060EE15C02E2E16AE552E16E21500D0E72
:10CC30001326000E1422DF2A1BD7580EE552E552A8
:10CC4000E552E552E5CFDAFFE7CFD9FF1200D9CFA1
:10CC5000E6FFDACFE6FFE1CFD9FFE2CFDAFFFD0E44
:10CC6000DB0402E178EC45F0580EE552E5CFDAFF3F
:10CC7000E7CFD9FF1200D9CFE6FFDACFE6FFE1CF49
:10CC8000D9FFE2CFDAFFE652E652E652E652FD0E57
:10CC9000DB5063E10C50B70DF3CF1DF0F4CF1EF065
:10CCA000320E1D26030E1E221DC0DEFF1EC0DDFF3C
:10CCB000DECFE9FFDDCFEAFF2F0EE926000EEA22E4
:10CCC000EF5043E0E66AE66AE66AE66ADECFE9FF2D
:10CCD000DDCFEAFFE9CF1DF0EACF1EF0E9CFE6FF96
:10CCE000EACFE6FF1CEC39F01F6E060EE15C02E2B3
:10CCF000E16AE552E16E1F50126E1F502EE1D950CD
:10CD0000020FE66E000EDA20E66EE66A010EE66EAF
:10CD1000000EE66E0A0EE66EDECFE9FFDDCFEAFF1B
:10CD2000E9CF1DF0EACF1EF0E9CFE6FFEACFE6FF3C
:10CD300072EC2DF01F6E080EE15C02E2E16AE55232
:10CD4000E16E1F50126E1F5002E0510E07D0020E0E
:10CD5000DBCF13F0030EDBCF14F0580E1D6E040E64
:10CD6000E15C02E2E16AE552E16E1D50E552E5CF79
:08CD7000DAFFE7CFD9FF120042
:08CD7800D9CFE6FFDACFE6FF98
:10CD8000E1CFD9FFE2CFDAFFE652E652DF6AFD0ECD
:10CD9000DB50F00BE8380F0BE76E010EE7CFDBFF3F
:10CDA000DBCF1DF0000EE76E1D18E8AE02D01D347B
:10CDB00003D0E750D8801D5405E20A0EDF26010E8D
:10CDC000DB06EED7FD0EDB500F0BDF26DF50E55202
:10CDD000E552E552E5CFDAFFE7CFD9FF1200D9CF10
:10CDE000E6FFDACFE6FFE1CFD9FFE2CFDAFFE65286
:10CDF000DF6AFD0EDBCF1DF00A0EE76E1D18E8AEF0
:10CE000002D0E73402D0E7501D5C0CE30A0E1D6E21
:10CE1000FD0EDBCFE7FF1D50E75EFD0EE7CFDBFF2A
:10CE2000DF2AE7D7DF38F00BDF6EFD0EDB50DF12B5
:10CE3000DF50E552E552E5CFDAFFE7CFD9FF120028
:10CE4000D9CFE6FFDACFE6FFE1CFD9FFE2CFDAFFB5
:10CE50002DEC6BF0D00EE66E58EC6CF0E55200094C
:10CE600010E1FD0EDBCFE6FF58EC6CF0E552000957
:10CE700008E1FC0EDBCFE6FF58EC6CF0E552000950
:10CE800002E0FF0E03D035EC6BF0000EE552E5CF6B
:10CE9000DAFFE7CFD9FF1200D9CFE6FFDACFE6FFFE
:10CEA000E1CFD9FFE2CFDAFFE652010EDF6E2DECC3
:10CEB0006BF0D00EE66E58EC6CF0E55200091DE107
:10CEC000E66A58EC6CF0E552000917E148EC6BF0AB
:10CED000D10EE66E58EC6CF0E55200090EE10A0E38
:10CEE000E66E920EE66E000EE66ECCEC6BF0E5524E
:10CEF000E552E552000901E1DF6A35EC6BF0DF50E5
:10CF000051E1F29CDF6ADFCF1DF0060EE76E1D18BF
:10CF1000E8AE02D01D3403D0E750D8801D541CE386
:10CF2000DFCFE9FFEA6AE9BEEA68920EE926000E61
:10CF3000EA22EF50E66E20DFE552E66EDFCFE9FF32
:10CF4000EA6AE9BEEA68880EE926000EEA22E5529E
:10CF5000E750EF6EDF2AD7D7DFCF1DF00A0EE76E5E
:10CF60001D18E8AE02D0E73402D0E7501D5C19E28C
:10CF7000DFCFE9FFEA6AE9BEEA68920EE926000E11
:10CF8000EA22EF50E66EDFCFE9FFEA6AE9BEEA681F
:10CF9000880EE926000EEA22E552E750EF6EDF2AFE
:10CFA000DBD7F28C000EE552E552E5CFDAFFE7CF92
:10CFB000D9FF1200D9CFE6FFDACFE6FFE1CFD9FFE4
:10CFC000E2CFDAFFE652E652DF6ADFCF1DF0060E4F
:10CFD000E76E1D18E8AE02D01D3403D0E750D880AC
:10CFE0001D5420E3DFCF1DF01E6A1DBE1E68FC0E1F
:10CFF000DB501D24E96EFD0EDB501E20EA6EEF5063
:10D00000E66EEDDEE552E66EDFCFE9FFEA6AE9BEE5
:10D01000EA68920EE926000EEA22E552E750EF6E2A
:10D02000DF2AD3D70001100E996F150E9A6F040EE8
:10D030009B6FDE52010EDD6E2DEC6BF0D00EE66EB6
:10D0400058EC6CF0E552000915E1E66A58EC6CF01A
:10D05000E55200090FE10A0EE66E920EE66E000E32
:10D06000E66E73EC6CF0E552E552E552000902E120
:10D07000010EDB6A35EC6BF0010EDB50E552E55238
:10D08000E552E5CFDAFFE7CFD9FF1200100EE66ECA
:10D09000070EE66ED5DEE552E552FEDE150E000106
:10D0A000905D03E1040E915D12E0926B936B946BC3
:10D0B000010E956F966F040E976F0C0E986F920E7F
:10D0C000E66E000EE66E76DFE552E552E5DE120012
:10D0D0000001882B3C0E885D0CE3886B892B3C0E8D
:10D0E000895D07E3896B8A2B180E8A5D02E38A6BE0
:10D0F00000801200F29C8EC01DF01E6A1F6A206A1A
:10D10000140E1D26000E1E221F222022190E1F0B98
:10D1100007E0D8901D361E361F362036E806F9E1A6
:10D120008DC021F0226A236A246A150E1F0B07E0C6
:10D13000D8902136223623362436E806F9E12150EC
:10D140001D1222501E1223501F12245020128CC078
:10D1500025F0266A276A286A100E1F0B07E0D89070
:10D160002536263627362836E806F9E125501D12E1
:10D1700026501E1227501F122850201200018A51DB
:10D18000296E2A6A2950296AE834E834E834F80B11
:10D190002A6E2B6A2C6A29501D122A501E122B50FF
:10D1A0001F122C50201289512D6E2E6A050ED89018
:10D1B0002D362E36E804FBE12F6A306A2D501D1201
:10D1C0002E501E122F501F12305020120001885175
:10D1D000316E326AD89032323132336A346A1D503D
:10D1E00031109C6F1E5032109D6F1F5033109E6F78
:10D1F000205034109F6FF28C9CC03BF09DC03CF0DF
:08D200009EC03DF03E6E1200DD
:08D20800949C948E969096828E
:10D21000AC6AAC8AAC84AB6AAB8EAB889F9A9F98A1
:10D220002A0EAF6EAC84B86A9D8A0001BB6BBC6BE2
:10D23000BD6BBE6BBF6BC06B12000001BB5102E146
:10D240009D981200BD51EA6A000FE96E0B0EEA22AA
:10D25000EF50AD6EBD2BBD511D6E1E6A800E1D18A8
:10D2600003E11E5001E1BD6BBB0712000001BB5181
:10D270001D6E1E6AD8901E5004E6800E1D5C000EC6
:10D280001E5801E3000C010CD9CFE6FFDACFE6FF10
:10D29000E1CFD9FFE2CFDAFF0001BB511D6E1E6A5C
:10D2A000D8901E5004E6800E1D5C000E1E58F4E25D
:10D2B000F29CBC51EA6A000FE96E0B0EEA22FD0EE9
:10D2C000DBCFEFFFBC2BBC511D6E1E6A800E1D18FC
:10D2D00003E11E5001E1BC6BBB2B9D88F28CE55233
:10D2E000E5CFDAFFE7CFD9FF12000001BB51FDE126
:10D2F0001200ABA202D0AB98AB88ABB420D0000137
:10D30000BE511D6E1E6AD8901E5004E6800E1D5C34
:10D31000000E1E5814E2BF51EA6A800FE96E0B0E30
:10D32000EA22AECFEFFFBF2BBF511D6E1E6A800EEB
:10D330001D1803E11E5001E1BF6BBE2B1200AECFE2
:10D34000C1F01200D9CFE6FFDACFE6FFE1CFD9FF77
:10D35000E2CFDAFF0001BE5102E1000E1FD0F29CC5
:10D36000C051EA6A800FE96E0B0EEA22EF50E66EBA
:10D37000FC0EDBCFE9FFFD0EDBCFEAFFE552E75005
:10D38000EF6EC02BC0511D6E1E6A800E1D1803E18A
:10D390001E5001E1C06BBE07F28C010EE552E5CFD5
:10D3A000DAFFE7CFD9FF1200D9CFE6FFDACFE6FFE9
:10D3B000E1CFD9FFE2CFDAFFFC0EDBCFF6FFFD0EA7
:10D3C000DBCFF7FF0800F5500FE0FC0EDBCFF6FFD8
:10D3D000DB2AFD0EDBCFF7FF01E3DB2A0800F55067
:10D3E000E66E52DFE552E8D7E552E5CFDAFFE7CF48
:10D3F000D9FF1200D9CFE6FFDACFE6FFE1CFD9FFA0
:10D40000E2CFDAFFFC0EDBCFE6FFFD0EDBCFE6FF5F
:10D41000CBDFE552E5520D0EE66E36DFE5520A0E21
:10D42000E66E32DFE552E552E5CFDAFFE7CFD9FF0E
:10D430001200D9CFE6FFDACFE6FFE1CFD9FFE2CF86
:10D44000DAFFFC0EDBCFE9FFFD0EDBCFEAFFEF508A
:10D450000EE0FC0EDBCFE9FFDB2AFD0EDBCFEAFF9F
:10D4600001E3DB2AEF50E66E0FDFE552EAD7E55223
:10D47000E5CFDAFFE7CFD9FF1200D9CFE6FFDACF49
:10D48000E6FFE1CFD9FFE2CFDAFFFC0EDBCFE6FF0C
:10D49000FD0EDBCFE6FFCDDFE552E5520D0EE66E69
:10D4A000F3DEE5520A0EE66EEFDEE552E552E5CF19
:10D4B000DAFFE7CFD9FF1200D9CFE6FFDACFE6FFD8
:10D4C000E1CFD9FFE2CFDAFFE652FD0EDB50F00BE1
:10D4D000E8380F0BDF6EDFCF1DF0090EE76E1D1869
:10D4E000E8AE02D01D3403D0E750D8801D5402E2CC
:10D4F000370E01D0300EDF26DFCFE6FFC5DEE55266
:10D50000FD0EDB500F0BDF6EDFCF1DF0090EE76E57
:10D510001D18E8AE02D01D3403D0E750D8801D544A
:10D5200002E2370E01D0300EDF26DFCFE6FFACDEA1
:10D53000E552E552E552E5CFDAFFE7CFD9FF120019
:10D54000D9CFE6FFDACFE6FFE1CFD9FFE2CFDAFFAE
:10D55000FD0EDBCF1EF01EC01DF01E6A1D50E66ED4
:10D56000ABDFE552FF0EE76EFC0EDBCF1DF0E750A0
:10D570001D161E6A1D50E66E9FDFE552E552E5CF8F
:10D58000DAFFE7CFD9FF1200D9CFE6FFDACFE6FF07
:10D59000E1CFD9FFE2CFDAFFFA0EDBCF1DF0FB0EB1
:10D5A000DBCF1EF0FC0EDBCF1FF0FD0EDBCF20F03B
:10D5B000180ED89020321F321E321D32E806F9E1D3
:10D5C0001D50E66E79DFE552FA0EDBCF1DF0FB0E43
:10D5D000DBCF1EF0FC0EDBCF1FF0FD0EDBCF20F00B
:10D5E000100ED89020321F321E321D32E806F9E1AB
:10D5F0001D50E66E61DFE552FA0EDBCF1DF0FB0E2B
:10D60000DBCF1EF0FC0EDBCF1FF0FD0EDBCF20F0DA
:10D61000080ED89020321F321E321D32E806F9E182
:10D620001D50E66E49DFE552FA0EDBCF1DF0FB0E12
:10D63000DBCF1EF0FC0EDBCF1FF0FD0EDBCF20F0AA
:10D640001D50E66E39DFE552E552E5CFDAFFE7CF50
:04D65000D9FF1200EC
:0CD654009482948412008B9294920A0E2F
:10D66000E66EDAEC70F0E55212008B9494948B9293
:10D6700094920A0EE66EDAEC70F0E55294840A0E8B
:10D68000E66EDAEC70F0E5529482000000001200C1
:10D690008B94949494820A0EE66EDAEC70F0E55264
:10D6A00094840A0EE66EDAEC70F0E5528B92949256
:10D6B0000A0EE66EDAEC70F0E55212008B94949448
:10D6C00094820A0EE66EDAEC70F0E5529484320E23
:10D6D000E66EDAEC70F0E55282B2FF0C000C1E0E22
:10D6E000E66EDAEC70F0E55282A4FE0C000C00014C
:10D6F000080ECC6F8B94949494820A0EE66EDAEC4A
:10D7000070F0E5529484010EE66EDAEC70F0E552AA
:10D7100082B407D0E4DF000904E0FE0EF36EF46883
:10D720001200010E0001D890CA37E806FCE10001A2
:10D73000CA91CB6B82B2CA81CC07DDE1CAC0F3FFCC
:10D74000CBC0F4FF1200D9CFE6FFDACFE6FFE1CF7E
:10D75000D9FFE2CFDAFFE652E652C9DFF3CFDEFFB0
:10D76000F4CFDDFF010EDB50FF0B03E1A7DF000963
:10D7700003E1F368F46808D0DECF1DF0DDCF1EF0C2
:10D780001DC0F3FF1EC0F4FFE552E552E552E5CFA0
:10D79000DAFFE7CFD9FF1200D9CFE6FFDACFE6FFF5
:10D7A000E1CFD9FFE2CFDAFFE652E652FB0EDBCF44
:10D7B000F3FFDB06F35000092BE099DFF3CFDEFF28
:10D7C000F4CFDDFF010EDB50FF0B02E0FF0E21D096
:10D7D000FC0EDBCFE9FFDB2AFD0EDBCFEAFF01E326
:10D7E000DB2ADFCFEFFFFB0EDB5003E19494948242
:10D7F00003D094948B9294920A0EE66EDAEC70F059
:10D80000E55294840A0EE66EDAEC70F0E552CED75B
:10D81000000EE552E552E552E5CFDAFFE7CFD9FF3A
:10D820001200D9CFE6FFDACFE6FFE1CFD9FFE2CF92
:10D83000DAFF0001080ECC6FFD0EDB500001CA6F4D
:10D84000CB6B8B9482B406D04ADF000902E0FF0E56
:10D8500029D023D00001CB6BCA37D8A00ED0949426
:10D8600094820A0EE66EDAEC70F0E55294840A0EA9
:10D87000E66EDAEC70F0E5520ED094948B929492AE
:10D880000A0EE66EDAEC70F0E55294840A0EE66E4B
:10D89000DAEC70F0E5520001CC070001CC51D2E186
:10D8A000000E00D0E552E5CFDAFFE7CFD9FF120036
:10D8B000D9CFE6FFDACFE6FFE1CFD9FFE2CFDAFF3B
:10D8C000FD0EDBCFE6FFADDFE552000903E1F6DE3A
:10D8D000000902E0FF0E01D0000EE552E5CFDAFFAD
:10D8E000E7CFD9FF1200D9CFE6FFDACFE6FFE1CFCD
:10D8F000D9FFE2CFDAFFFB0EDB5017E0FC0EDBCFE7
:10D90000E9FFDB2AFD0EDBCFEAFF01E3DB2AEF5064
:10D91000E66E87DFE552000903E1D0DE000902E090
:10D92000FF0E04D0FB0EDB06E6D7000EE552E5CF76
:08D93000DAFFE7CFD9FF120076
:08D93800D8CFE4FFE0CFE4FFCB
:10D94000E46EE9CFE4FFEACFE4FFF6CFE4FFF7CFE0
:10D95000E4FFF5CFE4FFF3CFE4FFF4CFE4FFFACF29
:10D96000E4FF00EE35F0140EE80403E3EECFE4FF2D
:10D97000FBD700EE1DF0180EE80403E3EECFE4FF42
:10D98000FBD7E6529EA204D09E92E6EC61F00082A4
:10D99000F0A203D0F09268EC68F09EA803D09E98A5
:10D9A0001DEC69F09EAA03D09E9A79EC69F0E552CD
:10D9B00000EE34F0180EE80403E3E5CFEDFFFBD7EB
:10D9C00000EE48F0140EE80403E3E5CFEDFFFBD7CB
:10D9D000E5CFFAFFE5CFF4FFE5CFF3FFE5CFF5FFA5
:10D9E000E5CFF7FFE5CFF6FFE5CFEAFFE5CFE9FFAB
:10D9F000E550E5CFE0FFE5CFD8FF1000D9CFE6FF37
:10DA0000DACFE6FFE1CFD9FFE2CFDAFFE652929A12
:10DA1000938A938894969488949A898A94908B9008
:10DA20000F0EC16E921293968A9692889382F08618
:10DA3000F08CF19A9384F088F09EF198939E939CD9
:10DA40008A9E8A9CFE0EE66E6DEC70F0E552C30E67
:10DA5000CB6E9F92400EC76E210EC66ED08E1F0EEB
:10DA6000186E006A08012E6B2D6B2C6BDF6A040E9A
:10DA7000DF5C11E2DF50B70DF3CFE9FFF4CFEAFF2F
:10DA8000320EE926030EEA22220EE926000EEA22D1
:10DA9000EF6ADF2AECD7E552E552E5CFDAFFE7CFB0
:10DAA000D9FF1200D9CFE6FFDACFE6FFE1CFD9FFE9
:10DAB000E2CFDAFFE652E6520801FC8F020E2E6F2B
:10DAC000DE52030EDD6EE66A9FEC5CF0E552DF6E1F
:10DAD000DF5007E0010EDBCFF3FFDB06F350000859
:10DAE000F2E3DF5013E1000EE66E010EE66EE66A29
:10DAF00035EC2AF0E552E552E552DF6EDF5006E1E3
:10DB00000801010E2E6FC7EC56F0DF6E020E080101
:10DB10002E5D02E1020EF96FDF50126EE552E55202
:10DB2000E552E5CFDAFFE7CFD9FF120066EC57F0F8
:10DB3000000EE66EE66AE66A35EC2AF0E552E5523A
:10DB4000E55208012E6BF96B120058DF69EC6EF09C
:10DB50002AEC6BF046EC68F032EC5AF004EC69F019
:10DB60008CEC6FF0036A400EE66E91EC52F0E552D9
:10DB7000F28EF28C00A003D04CEC67F0009000A273
:10DB800023D00092F90EE66E080EE66E73EC6EF08E
:10DB9000E552E552FC0EE66E080EE66E73EC6EF092
:10DBA000E552E552A3EC59F02CEC62F0000904E0D8
:10DBB00008012E5101E176DF2CEC62F0000904E14E
:10DBC00008012E5101E0B2DF00A4D4D7009469EC23
:04DBD0005AF0D0D760
:0CDBD400D9CFE6FFDACFE6FFFA0EE3CF70
:10DBE000D9FFFB0EE3CFDAFFFC0EE3CFE9FFFD0E1A
:10DBF000E3CFEAFFE9CFF3FFEACFF4FFF80EE350FB
:10DC000003E1F90EE35008E0F80EE30602E2F90E34
:10DC1000E306DECFEEFFF2D7FF0EE3CFDAFFE552E9
:10DC2000FF0EE3CFD9FFE5521200FE0EE3CFE9FF6E
:10DC3000FF0EE3CFEAFFE9CFF3FFEACFF4FFFB0EDD
:10DC4000E35003E1FC0EE35009E0FB0EE30602E2C1
:10DC5000FC0EE306FD0EE350EE6EF1D71200D9CFB5
:10DC6000E6FFDACFE6FFFA0EE3CFD9FFFB0EE3CFF4
:10DC7000DAFFFC0EE3CFE9FFFD0EE3CFEAFFE9CFC9
:10DC8000F3FFEACFF4FFDECFEFFFEE66FCD7FF0E27
:10DC9000E3CFDAFFE552FF0EE3CFD9FFE5521200E2
:10DCA000FB0EE3CFF6FFFC0EE3CFF7FFFD0EE3CF55
:10DCB000F8FFFE0EE3CFE9FFFF0EE3CFEAFFE9CF67
:10DCC000F3FFEACFF4FF0900F5CFEFFFEE66FBD7D5
:02DCD000120040
:0EDCD2000801010EFB6FFA6BF96B0801FE6B87
:10DCE000FD6BFC6B1200D9CFE6FFDACFE6FFE1CF88
:10DCF000D9FFE2CFDAFFFC0EDBCFE9FFFD0EDBCF71
:10DD0000EAFFEF50030B030A0EE0010A0AE0030AE0
:10DD100005E0010A0DE10801FF6B0AD00801010EC0
:10DD200006D0400E01D0800E0801F8150801FF6FE3
:10DD3000FC0EDBCFE9FFFD0EDBCFEAFFEF50800BDF
:10DD400010E0FC0EDBCFE9FFFD0EDBCFEAFFEF9E1C
:10DD5000FC0EDBCFE9FFFD0EDBCFEAFFEE52080E33
:10DD6000EF6EFC0EDBCFE9FFFD0EDBCFEAFFEE52DC
:10DD7000EF500AE0FC0EDBCFE9FFFD0EDBCFEAFF40
:10DD8000EE52EF060801FF71FC0EDBCFE9FFFD0E3E
:10DD9000DBCFEAFF020EE926000EEA22EF5008E090
:10DDA0000801FF51E8B08A8CE8B008D08A9C06D000
:10DDB0000801FF51E8B08A8EE8A08A9EE552E5CFBF
:08DDC000DAFFE7CFD9FF1200E2
:08DDC800D9CFE6FFDACFE6FF38
:10DDD000E1CFD9FFE2CFDAFFFF0EE76EFC0EDBCF1B
:10DDE0001DF0E7501D161D50A96EFD0EDBCF1EF075
:10DDF0001EC01DF01E6A1D50AA6EA69EA69CA6807F
:10DE0000A850E552E5CFDAFFE7CFD9FF1200D9CF0E
:10DE1000E6FFDACFE6FFE1CFD9FFE2CFDAFFFF0E70
:10DE2000E76EFC0EDBCF1DF0FD0EDBCF1EF0E750E2
:10DE30001D161E6A1D50A96EFC0EDBCF1DF0FD0ED7
:10DE4000DBCF1EF01EC01DF01E6A1D50AA6EFB0E19
:10DE5000DB50A86EA69CA69EA684F29E550EA76EC9
:10DE6000AA0EA76EA682F28EA6B2FED7A694E5529F
:0ADE7000E5CFDAFFE7CFD9FF12007B
:06DE7A00CA0EF66E0A0E4E
:10DE8000F76E000EF86E00010900F550B66F09003C
:10DE9000F550B76F03E1B66701D03DD00900F550EA
:10DEA000B16F0900F550B26F0900F550B36F09006A
:10DEB0000900F550E96E0900F550EA6E0900090005
:10DEC0000900F550B46F0900F550B56F090009005D
:10DED000F6CFB8F0F7CFB9F0F8CFBAF0B1C0F6FF8F
:10DEE000B2C0F7FFB3C0F8FF0001B45302E1B5536D
:10DEF00007E00900F550EE6EB407F8E2B507F9D770
:10DF0000B8C0F6FFB9C0F7FFBAC0F8FF0001B60706
:08DF1000000EB75BBFD7120041
:08DF18000001C46B400EC56F4F
:10DF200012000001C45107E0C2C0E6FF44EC69F0F2
:10DF3000E5520001C46B36EC69F0000903E0000112
:10DF4000C58D02D00001C59DC5B90CD0C30EE66ECB
:10DF5000000EE66EA2EC69F0E552E552000902E01F
:10DF60000001C58912000001C45106E183CFC2F04F
:10DF7000010EC46FC59D1200C58F12000001C5A916
:10DF800004D0C3C08CFFC59902D0C58B8C68956A3C
:0CDF90001200C5C08CFF956A1200120040
:04DF9C003B504002B4
:10DFA000F3CF37F0F4CF38F04102F3503826000EAB
:10DFB000F420396E3B504202F3503926000EF42013
:10DFC0003A6E3B504302F3503A263C504002F35025
:10DFD0003826F4503922000E3A223C504102F350C8
:10DFE0003926F4503A223C504202F3503A263D5032
:10DFF0004002F3503926F4503A223D504102F3508A
:0CE000003A263E504002F3503A2612002F
:04E00C00E550080EC5
:10E010001C6ED8901936E7AE02D0090E191A19AE47
:10E0200002D0090E191AE7461C2EF3D7E65012004B
:10E03000FF0EE3501B181C6EF00B1C3A1C1A1C50F0
:10E04000F00B1A181B6E1C441B1AE00B1B1A1C3A0F
:06E050001C181A6E000C02
:0AE056003A6A396A386A376A200E08
:10E06000E76ED8903B363C363D363E36373638364E
:10E0700039363A364050375C41503858425039585A
:10E0800043503A5809E34050375E4150385A4250A5
:0EE09000395A43503A5A3B2AE72EE4D7120081
:02E09E003DC083
:10E0A00047F03D504202F4CF3CF0F3CF3BF03E50FE
:10E0B0004302F4CF3EF0F3CF3DF04202F3503C2652
:10E0C000F4503D22E86A3E2247504302F3503C267A
:0AE0D000F4503D22E86A3E22000CE5
:06E0DA00D9CFE6FFDACF0A
:10E0E000E6FFE1CFD9FFE2CFDAFFFD0EDB50FB0BFD
:10E0F000CA6ECC6A9E92FD0EDBAE02D09D8201D02C
:10E100009D92CA84E552E5CFDAFFE7CFD9FF12002E
:10E110003A6A396A100EE76ED8903D363E36393687
:10E120003A364250395C43503A5805E34250395E22
:0CE1300043503A5A3D2AE72EF0D7120067
:04E13C00222A2B2C3C
:10E140003A3B3C3D3E3F5B5D7C7F002F68617264E3
:0CE15000342D0065747273686172640005
:04E15C007AC4CEC4EF
:10E1600006C562C50AC692C61CC85EC8C4C81CC91A
:0CE17000A6C924C74CCA4ECC76CC64C4AF
:04E17C001CEE00F0A5
:10E180002CEE00F0F86A369C3DEC6FF0ECEC70F091
:08E19000A5EC6DF0FBD71200B5
:08E198003A6A080EE76ED89008
:10E1A0003E363A3643503A5C02E33A6E3E2AE72E58
:04E1B000F7D712008B
:0CE1B400FF0EE350E84E1200000000D007
:0AE1C00000D000D0E82EFAD71200BC
:06E1CA0000EE00F00F0E54
:08E1D000EE6AEA62FDD71200BD
:02E1D800120033
:01E1DA000143
:02FFFE0007FA00
:020000040030CA
:0100010006F8
:0100020018E5
:010003001EDE
:010005008179
:010006008178
:01000B00A054
:0200000400F00A
:10000000FEFEFF180218193A4038E680C01116505B
:100010000609CD1F50C0E946524548442E524F4D67
:1000200021000039E5DDE1EB3E03D3C4CDA45078D7
:100030003C3CD3C30EC23E01ED79EDB3AFED79CDBB
:10004000A450C00EFFCD7F503D200CCD7050CD7F11
:1000500050772310F918EE3D280BCD7F5047CD7F08
:100060005010FB18E0CD70503E06D3C4CDA450AF65
:10007000C9CD7F5047CD7F506F05CD7F506705C9F3
:100080000C2003CD8850DBC2C9AFD3C33E04D3C418
:10009000CDA4502005DBCFE608C03E06D3C4CDA4D6
:1000A00050DDF93CC9DBCF0738FBDBCFE601C9FFE8
:1000B000FFFFFFFFFFFFFFFFFFFFFFFFFFFFFFFF50
:1000C000FFFFFFFFFFFFFFFFFFFFFFFFFFFFFFFF40
:1000D000FFFFFFFFFFFFFFFFFFFFFFFFFFFFFFFF30
:1000E000FFFFFFFFFFFFFFFFFFFFFFFFFFFFFFFF20
:1000F000FFFFFFFFFFFFFFFFFFFFFFFFFFFFFFFF10
:0203FE0007FAFC
:00000001FF
